:020000040800F2
:100000000000011089D90308C9B503088DCA00088A
:100010008DDA03088DDA03088DDA0308000000008A
:10002000000000000000000000000000C5B503084B
:10003000C1B5030800000000BDB50308E5EC0008E9
:100040008DDA03088DDA03088DDA03088DDA0308E8
:100050008DDA03088DDA0308C59C0008B59D0008F9
:100060008DDA0308799D00083D9D000865BF0008F2
:1000700055BF000845BF000835BF000825BF000870
:1000800011BF0008FDBE00088DDA03088DDA0308F1
:100090008DDA03088DDA03088DDA0308019D000864
:1000A0008DDA03085DD000088DDA03086DD00008F2
:1000B0008DDA03084DD000083DD0000841C5000886
:1000C00049C5000835C500083DC500088DDA03089C
:1000D0008DDA0308699400080DEE00088DDA030834
:1000E000899C00088DDA030819B903088DDA030822
:1000F0000DD000088DDA03081DD00008E9BE000805
:100100008DDA03088DDA03082DD000088DDA030894
:1001100071ED00088DDA03088DDA03088DDA030823
:10012000D5BE0008C1BE0008ADBE000899BE0008DB
:1001300085BE00088DDA03088DDA03088DDA03081E
:100140008DDA03088DDA03088DDA030881AF03081E
:1001500071BE00085DBE000849BE00088DDA0308C4
:1001600029C5000831C500088DDA03088DDA0308B7
:100170008DDA03088DDA03088DDA03088DDA0308B7
:080180008DDA03088DDA030893
:0801880020D503000100000076
:10019000020203008C1E0020881E002000000000C8
:1001A0000000000016000800901E0020981E00208D
:1001B00000000000F00500081D000100D82200200A
:1001C0006823002000000000F80500082700040054
:1001D000F82200206C23002000000000FA0500082F
:1001E0000300010038250020402500200000000009
:1001F00000000000031232006C2600205C27002063
:10020000000000000000000025005A00A826002081
:10021000022700200000000000000000F601080096
:1002200044250020A026002000000000000000005F
:1002300012001600FC270020E0280020000000002B
:10024000FE0500080C00240012280020F8280020D9
:10025000000000000984010800020500D4270020E6
:100260001C29002000000000000000002C001000ED
:10027000E82C0020D82C002000000000653E020879
:100280002B0024001C2D0020F82C00200000000072
:10029000353E02081E000400142F0020FC30002010
:1002A000000000001406000822000C00802E002030
:1002B0000031002000000000180600080400C00003
:1002C00068530020285500200000000000000000B6
:1002D000F90104001C360020E85500200000000051
:1002E000C981000818002C00E8350020EC550020DA
:1002F000000000000547020806001A000C3100202B
:1003000018560020000000007D00030801010400D1
:100310007C5600201C65002000000000000000004A
:1003200008020900C06400202065002000000000D1
:10033000D981000806020C00C96400202C65002049
:10034000000000007D90000807020200FC6400200D
:10035000386500200000000024060008FF010100AD
:10036000186500203C6500200000000026060008FB
:10037000FA01010010650020406500200000000027
:100380002806000802000C00D86400204465002004
:1003900000000000000000001B00F400EC6E0020D4
:1003A000E06F002000000000217902080B100C0013
:1003B000586D0020D4700020000000002A060008BC
:1003C00001000A000C7A0020187A002000000000CA
:1003D000360600081A000800F4790020247A00206C
:1003E00000000000400600082A0060008C7A00200F
:1003F0002C7A002000000000F1FF020815007000B8
:10040000B8720020EC7A002000000000000000001C
:1004100029005000007E0020547E002000000000D3
:100420000000000014000200FC7D0020A47E0020DB
:10043000000000004806000810000300F07D0020C6
:10044000A87E0020000000004A06000828000C00DA
:10045000E47D0020AC7E0020000000004E06000875
:1004600026000800DC7D0020B87E0020000000008F
:100470005A06000823000E00CC7D0020C07E00201C
:1004800000000000A932020819000500C47D002008
:10049000D07E00200000000062060008F801010084
:1004A000C07D0020D87E0020000000006806000803
:1004B00000010400BC7D0020DC7E00200000000064
:1004C0006A0600080D003400408600207486002073
:1004D0000000000025D40208FD012400507F002008
:1004E000A88600200000000059810008FE010800D5
:1004F0003C7F0020CC8600200000000051C6000890
:100500000500050001880020F49400200000000090
:10051000700600080E00DE00E8860020FC94002033
:10052000000000005D00030813000400FC870020A9
:10053000DC9500200000000078060008020103009E
:10054000D7860020E09500200000000049A802089E
:1005500003010600889700209C97002000000000FF
:100560007C0600083400100010A60020E4A600203D
:100570000000000019000308FB010100ECA40020AA
:10058000F4A600200000000049C60008FC01090094
:10059000B4A30020F8A600200000000015C6000843
:1005A000F7010600ACA3002004A700200000000013
:1005B000820600080A001200149800200CA70020F0
:1005C00000000000880600081F000E0030A8002070
:1005D00058A80020000000009A060008050201004B
:1005E0001CA8002068A8002000000000A806000841
:1005F000C4090000190128280000200300000000A1
:1006000000010000000000000000000000000000E9
:100610000000000000000100C800141E010064007A
:100620002C012800013C01002C002B21231E00027C
:10063000000001000A010A0AE8030000640001004A
:100640007E05EA05B4053200030000010500000044
:100650000001000000000000000001155802D9034D
:10066000C503000028010000040065FDC409000066
:100670000101020001000000180100000401010056
:1006800000003D010000000000300100005A0000A1
:10069000000090012C01C800640000000000000070
:0906A0000100000000050000004B
:1006A9000000803F0000803F0000803F0000803F45
:1006B9000000803F0000803F50010000070000005B
:1006C9000200000000000000000000000102030415
:1006D90006070809FF0100000000803F0000803F75
:1006E900006002401060024000000000000B0000A2
:1006F900000020000000000000000000006002402F
:100709002860024000000000060C000000002000E4
:10071900000000000000000000600240406002404C
:1007290000000000100D0000000020000000000083
:100739000000000000600240586002400000000014
:10074900160E00000000200000000000000000005C
:10075900006002407060024000000000200F0000AD
:1007690000002000000000000000000000600240BE
:1007790088600240000000002610000000002000F0
:10078900000000000000000000600240A06002407C
:1007990000000000301100000000200000000000EF
:1007A9000000000000600240B86002400000000044
:1007B900362F0000000020000000000000000000AB
:1007C900006402401064024000000000003800008C
:1007D900000040000000000000000000006402402A
:1007E90028640240000000000639000000004000B3
:1007F9000000000000000000006402404064024064
:1008090000000000103A0000000040000000000055
:10081900000000000064024058640240000000002B
:10082900163B00000000400000000000000000002E
:10083900006402407064024000000000203C000097
:1008490000004000000000000000000000640240B9
:1008590088640240000000002644000000004000B7
:10086900000000000000000000640240A064024093
:1008790000000000304500000000400000000000BA
:100889000000000000640240B8640240000000005B
:100899003646000000004000000000000000000093
:1008A900FFFFFFFF01000000010100001D390208E0
:1008B900000000000000000001000000000001012C
:1008C900FFFF00000000803F5419040805080400D8
:1008D900000000006C3204080832040840190408BA
:1008E900000000008019040805080A000000000043
:1008F9006C32040808320408703104080000000052
:10090900104A0408D0490408000000000000000053
:10091900204A0408284A04080000000001200000B9
:100929002C4A0408344A0408000000000140000071
:10093900384A0408E05D04080000000001200000B6
:10094900444A0408504A040800000000040000005A
:10095900544A0408604A040800000000040000002A
:10096900644A040860540408000000000100000003
:10097900010200002D800308E57F0308357F030885
:1009890000000000317D0308697E0308097F030820
:10099900D17D03080000000000000000257D030848
:1009A90001AE0308FDAD0308F9AD0308EDAD030879
:1009B900E9AD0308F5AD0308F1AD030875AE030809
:1009C90069AE030841AE030855AE03082DAE03080E
:1009D90019AE030805AE0308010000000840040829
:1009E900000000000000000059A80208A0860100CC
:1009F90004000000000000000000000000000000EA
:100A090000000000000000000000000000000000DD
:100A1900C06304086C3F0408000000003D9A010807
:100A29007D0000000600000000000000000000003A
:100A390000000000000000000000000000000000AD
:100A490000000000704A04080000000000000000D7
:100A59006D140108E8030000030000000000000015
:100A6900000000000000000000000000000000007D
:100A79000000000000000000784A0408000000009F
:100A890000000000B1010308102700000300000066
:100A9900000000000000000000000000000000004D
:100AA900000000000000000000000000B048040839
:100AB900000000000D3D0208A9EE0008204E0000CC
:100AC9000500000000000000000000000000000018
:100AD900000000000000000000000000000000000D
:100AE900604104080000000000000000210F010817
:100AF90010270000010000000000000000000000B5
:100B090000000000000000000000000000000000DC
:100B190000000000844A04080000000000000000F2
:100B2900E1C50008E803000005000000000000001E
:100B390000000000000000000000000000000000AC
:100B49000000000000000000904A040800000000B6
:100B5900000000007DAA0208204E000003000000EA
:100B6900000000000000000000000000000000007C
:100B7900000000000000000000000000A04A040876
:100B8900000000000000000087A80208204E0000B5
:100B99000300000000000000000000000000000049
:100BA900000000000000000000000000000000003C
:100BB900B04A04080000000000000000790D010897
:100BC900400D0300030000000000000000000000C9
:100BD900000000000000000000000000000000000C
:100BE9000000000038350408000000000000000083
:100BF90005E70208102700000100000000000000BE
:100C090000000000000000000000000000000000DB
:100C19000000000000000000783F04080000000008
:100C290000000000811C02081027000003000000DA
:100C390000000000000000000000000000000000AB
:100C4900000000000000000000000000C04A040885
:100C590000000000000000003DC50308A086010057
:100C6900010000000000000000000000000000007A
:100C7900000000000000000000000000000000006B
:100C8900D8340408000000000000000065C403080F
:100C990050C3000001000000000000000000000037
:100CA900000000000000000000000000000000003B
:100CB90000000000C84A040800000000000000000D
:100CC900D5BF0308A8610000010000000000000072
:100CD900000000000000000000000000000000000B
:100CE9000000000000000000D44A040800000000D1
:100CF90000000000A9270208A086010001000000E9
:100D090000000000000000000000000000000000DA
:100D19000000000000000000000000007C3504080D
:100D29000000000000000000C1310108A00F000010
:100D390001000000000000000000000000000000A9
:100D4900000000000000000000000000000000009A
:100D5900E04A04080000000000000000397302089E
:100D69001027000001000000000000000000000042
:100D7900000000000000000000000000000000006A
:100D890000000000C041040800000000000000004D
:100D99006D9D0308102700000100000000000000FD
:100DA900000000000000000000000000000000003A
:100DB9000000000000000000603F0408000000007F
:100DC90000000000896003081A41000001000000CA
:100DD900000000000000000000000000000000000A
:100DE900000000000000000000000000EC4A0408B8
:100DF900000000000000000001D40208400D0300BB
:100E090000000000000000000000000000000000D9
:100E190000000000000000000000000000000000C9
:100E2900F44A0408000000000000000071AC020848
:100E3900A08601000300000000000000000000007F
:100E49000000000000000000000000000000000099
:100E5900000000000000803F20700020702D72000B
:100E69000000000000010000000000000000000078
:100E7900B86904080E00000000000000000000002E
:100E890000000000CC140020FFFFFFFFFA00000063
:100E99000100000001000000746504080000000062
:100EA9000000000000000000000000006B6504085D
:100EB900040000009D70030800000000000000000D
:100EC9007C6504080100000000000000000000002B
:100ED90000000000000000000D00000000000000FC
:100EE9000000000000000000DA5400200100C409DD
:100EF90000000000D85400200100C40900000000CF
:100F0900D65400200100C40900000000D454002078
:100F19000100C40900000000D05400200100C409E8
:100F290000000000D25400200100C40900000000A4
:100F3900CE5400200100C40900000000CC54002058
:100F49000100C409000000009C6504080E000000AF
:100F5900000000000000000000000000F807002069
:100F6900849700209CFF2C010000000080150020C0
:100F79000A0000007031040828970020E0150C17BA
:100F89000000000082150020080000000832040853
:100F990081150020050000006C3204082A97002002
:100FA90002000000883104080788002001200100A0
:100FB900068800200200000094310408CE87002032
:100FC9000000F40101000000CC8700200000F401BA
:100FD90001000000CA8700200000F40101000000A0
:100FE900C88700200000F40101000000C687002026
:100FF90000FF0100E2870020E803D0070A00000093
:10100900E0870020006401000A000000E187002059
:10101900006401000A000000DA8700200064010072
:101029000A000000DF870020006401000A000000B8
:10103900DE870020006401000A000000DD8700202F
:10104900006401000A000000D987002000FF0100A8
:101059000A000000D887002000FF01000A000000F4
:10106900E48600200000F40101000000E28600206F
:101079000000F40101000000E08600200000F401F6
:1010890001000000DE8600200000F40101000000DC
:10109900D587002000C80100D487002000C80100BE
:1010A900D387002000C80100D28700200064010016
:1010B9000A000000D187002000FF01000A0000009B
:1010C900ED87002000C80100EC87002000C801005E
:1010D900EB87002000C80100EA87002000C8010052
:1010E900E987002000C80100E887002000C8010046
:1010F900E787002000C80100E687002000C801003A
:10110900E587002000C80100A4650408000000006C
:10111900000000000000000000000000B4650408A1
:1011290009000000000000009C08002004000000E5
:10113900BC650408090000000000000090080020B8
:10114900040000007868040809000000000000009D
:1011590084080020040000009848040809000000E1
:10116900000000007808002004000000C46504089D
:1011790009000000000000006C08002004000000C5
:10118900CC65040809000000000000006008002088
:1011990004000000D46504080900000000000000F4
:1011A9005408002004000000DC6504080900000060
:1011B9000000000048080020040000007C650408C5
:1011C9000100000000000000000000000000000015
:1011D900000000000D0000000000000000000000F9
:1011E90000000000E46504080000000000000000A1
:1011F9000000000000000000F4650408050000007C
:1012090000000000DD860020000000007C65040865
:1012190001000000000000000000000000000000C4
:10122900000000000D0000000000000000000000A8
:1012390000000000FC650408000000000000000038
:101249000000000000000000D04904080000000070
:1012590000000000801700200400000094480408E2
:101269000C00000035710308FC0800200000000094
:10127900CC6A04080C000000016F0308F008002084
:1012890000000000086604080C000000E56E030871
:10129900E4080020000000001066040808000000AF
:1012A90000000000D80800200400000018660408A7
:1012B9000C000000516E0308CC080020000000005B
:1012C900206604080900000000000000C008002092
:1012D900040000002866040803000000555F0308A5
:1012E900A8080020000000007C6504080100000037
:1012F90000000000000000000000000000000000E5
:101309000D000000000000000000000000000000C7
:101319002C66040800000000000000000000000026
:10132900000000003C6604080C00000000000000FA
:101339001009002000000000446604080A000000AB
:101349000000000008880020000000005066040822
:101359000A000000000000001088002000000000C2
:10136900586604080A0000000000000018880020E0
:10137900000000006066040807000000000000008B
:1013890008090020000000006C6604080400000041
:101399004D54030800000000000000007C650408AB
:1013A9000100000000000000000000000000000033
:1013B900000000000D000000000000000000000017
:1013C900000000007866040800000000000000002A
:1013D90000000000000000008C66040807000000FF
:1013E900000000004C090020000000009866040875
:1013F9000800000000000000400900200000000073
:10140900A466040808000000000000003409002058
:1014190000000000B0660408080000000000000099
:101429002809002000000000BC660408080000002C
:10143900000000001C090020000000007C65040871
:101449000100000000000000000000000000000092
:10145900000000000D000000000000000000000076
:1014690000000000C8660408000000000000000039
:10147900BB07002000000000D46604080B00000030
:1014890000000000B409002000000000DC66040828
:101499000B00000000000000A80900200000000067
:1014A900E86604080B000000000000009C09002009
:1014B90000000000F46604080B00000000000000B2
:1014C9009009002000000000006704080B000000DC
:1014D9000000000084090020000000000C670408D7
:1014E9000B00000000000000780900200000000047
:1014F900146704080B000000000000006C090020BC
:1015090000000000206704080B0000000000000034
:1015190060090020000000002C6704080800000092
:101529000000000054090020000000007C65040848
:1015390001000000000000000000000000000000A1
:10154900000000000D000000000000000000000085
:1015590000000000386704080000000000000000D7
:1015690000000000000000004C67040808000000AB
:1015790000000000E409002000000000586704088A
:101589000800000000000000D80900200000000049
:10159900646704080800000000000000CC0900206E
:1015A9000000000070670408080000000000000047
:1015B900C0090020000000007C650408010000004B
:1015C9000000000000000000000000000000000012
:1015D9000D000000000000000000000000000000F5
:1015E900786704080000000000000000B807002028
:1015F90000000000886704080B00000000000000DC
:10160900140A002000000000946704080B00000081
:1016190000000000080A002000000000A06704087C
:101629000700000000000000000A00200000000080
:10163900AC6704080700000000000000F80900205A
:1016490000000000B867040807000000000000005F
:10165900F0090020000000007C650408010000007A
:101669000000000000000000000000000000000071
:101679000D00000000000000000000000000000054
:10168900C46704080000000000000000B80700203B
:1016990000000000D06704080700000000000000F7
:1016A900600A002000000000D86704080700000055
:1016B90000000000580A002000000000E06704084C
:1016C9000700000000000000500A00200000000090
:1016D900E86704080700000000000000480A00202D
:1016E90000000000F0670408070000000000000087
:1016F900400A002000000000F86704080700000005
:1017090000000000380A00200000000000680408FA
:101719000700000000000000300A0020000000005F
:10172900086804080700000000000000280A0020DB
:101739000000000010680408070000000000000015
:10174900200A0020000000007C6504080100000058
:101759000000000000000000000000000000000080
:101769000D00000000000000000000000000000063
:10177900186804080E00000000000000054E030868
:1017890000000000680A0020DB8600200A32010000
:10179900DA86002001FA0100D686002000C801007F
:1017A900D4860020E803D00701000000414C4945D8
:1017B9004E464C4947485446340000002068040806
:1017C9000E0000001B4E030800000000EB51030847
:1017D900440B0020286804080E0000008D6E0308E1
:1017E9000000000000000000940B0020306804088D
:1017F9000E0000002D540308E15203083950030874
:10180900700C0020386804080E000000B54E03086B
:10181900854E030800000000240D002040680408DC
:101829000E0000002D4F0308714F0308000000004F
:10183900C40D0020D6870020010301004C6804086C
:101849000E000000614E03083D4E03080000000031
:10185900B40E0020546804080E000000E54E030889
:101869001552030800000000400F002060680408BA
:101879000E000000A14F03085D520308000000009C
:10188900E00F0020D08700200103010068680408E8
:10189900000000000000000000000000000000003F
:1018A900746804080800000000000000001100200E
:1018B900000000007C680408070000000000000028
:1018C900F8100020000000008C68040807000000E0
:1018D90000000000F01000200000000098680408D3
:1018E9000700000000000000E810002000000000D0
:1018F900A468040803000000555F0308D010002005
:10190900000000007C6504080100000000000000E0
:101919000000000000000000000000000D000000B1
:10192900000000000000000000000000AC6804088E
:10193900000000000000000000000000000000009E
:10194900BC6804080A000000000000009034040884
:1019590000000000C46804080A000000000000003C
:10196900A862040800000000CC6804080A0000000E
:1019790000000000EE87002000000000D468040881
:101989000A000000000000000C1100200000000007
:101999007C65040801000000000000000000000050
:1019A90000000000000000000D0000000000000021
:1019B9000000000000000000DC68040800000000CE
:1019C900000000000000000000000000B03504081D
:1019D90003000000555F03084C11002000000000BF
:1019E900F068040803000000555F0308841500200F
:1019F90000000000F868040803000000555F0308B0
:101A090034110020000000000069040803000000F0
:101A1900555F03081C110020000000007C650408C4
:101A290001000000000000000000000000000000AC
:101A3900000000000D000000000000000000000090
:101A4900000000000C69040800000000000000000C
:101A590000000000000000001869040807000000E9
:101A6900A9520308E411002000000000C063040823
:101A790003000000555F0308CC110020000000009E
:101A89002469040803000000555F0308B41100200D
:101A9900000000002C69040803000000555F0308DA
:101AA9009C110020000000003469040807000000B0
:101AB9008D5203089411002000000000E86A040810
:101AC90003000000555F03087C110020000000009E
:101AD9004069040803000000555F030864110020F1
:101AE900000000007C6504080100000000000000FF
:101AF9000000000000000000000000000D000000D0
:101B09000000000000000000000000004C6904080B
:101B19000E000000D94D0308AB4D0308000000007A
:101B2900EC110020546904080E0000000D50030850
:101B390000000000000000008C1200206069040809
:101B49000E0000000000000000000000000000007E
:101B590018130020706904080E000000E54F0308FF
:101B6900C552030800000000A41300207869040886
:101B7900000000000000000000000000000000005C
:101B8900A848040803000000555F0308B4140020A6
:101B9900000000006469040803000000555F0308A1
:101BA9009C14002000000000846904080300000060
:101BB900555F0308841400200000000090690408A0
:101BC90003000000555F03086C14002000000000AA
:101BD90098690408020000006D5E03080000000017
:101BE90000000000A0690408020000006D5E0308FF
:101BF9000100000000000000AC69040802000000B8
:101C09006D5E0308020000000000000000000000F3
:101C19000D000000000000000000000000000000AE
:101C2900010101006C6B04080E000000856F0308B8
:101C3900000000000000000004170020406B0408A9
:101C4900000000000000000000000000000000008B
:101C5900D04904080000000000000000BC1B00205F
:101C690004000000CC6A04080C00000001A9030864
:101C7900981B002000000000086604080C00000002
:101C8900D9A803088C1B0020000000001066040876
:101C99000800000000000000801B00200400000074
:101CA900186604080C00000063A30308741B0020D5
:101CB900000000002866040803000000555F0308BF
:101CC9005C1B002000000000506B040803000000AA
:101CD900555F0308441B0020000000007C650408D0
:101CE90001000000000000000000000000000000EA
:101CF900000000000D0000000000000000000000CE
:101D090000000000406B0408000000000000000013
:101D19000000000000000000D04904080000000095
:101D290000000000BC1B002004000000786A0408C1
:101D3900030000003B7003082C1B00200800000072
:101D4900186604080C00000063A30308741B002034
:101D5900000000002866040803000000555F03081E
:101D69005C1B002000000000506B04080300000009
:101D7900555F0308441B0020000000007C6504082F
:101D89000100000000000000000000000000000049
:101D9900000000000D00000000000000000000002D
:101DA90000000000586B040800000000000000005B
:101DB9000000000000000000D049040800000000F5
:101DC90000000000BC1B002004000000806A040819
:101DD90003000000555F0308A41B00200000000059
:101DE9007C650408010000000000000000000000FC
:101DF90000000000000000000D00000000000000CD
:101E0900000000000000000000FFFF0000000000CB
:101E19000000000001020304010203040607080987
:101E29002D202D2D202D2D2D2D202D2D2D2D00005A
:101E39000000000000000000000000000000000099
:101E49004097002088130C170100000042970020DA
:101E590088130C1700000000D06904080000000076
:101E6900000000000000000000000000E069040814
:101E79000800000000000000AC170020040000006A
:101E8900EC6904080800000000000000A017002009
:101E990000000000286604080400000075710308AA
:101EA90000000000000000007C650408010000003B
:101EB9000000000000000000000000000000000019
:101EC9000D000000000000000000000000000000FC
:101ED900C01200003E97002088130C170100000073
:101EE9003C97002088130C1700000000286A04089A
:101EF9000E000000D96F0308000000000000000078
:101F0900B81700206F970020010000002C32040848
:101F19003A97002001000000383204086C9700202D
:101F29000200000040320408225500200000000091
:101F39000000000020550020000000000000000003
:101F49001E55002000000000000000001C55002064
:101F590000000000000000001A55002000000000E9
:101F690000000000185500200000000000000000DB
:101F79003018002000000000000000003997002000
:101F8900020000004C320408306A04080000000016
:101F9900000000000000000000000000E0690408E3
:101FA90008000000000000004018002004000000A4
:101FB900EC69040808000000000000003418002043
:101FC900000000002866040804000000B96F030837
:101FD90000000000000000007C650408010000000A
:101FE90000000000000000000000000000000000E8
:101FF9000D000000000000000000000000000000CB
:10200900406A040800000000000000000000000011
:1020190000000000506A04080C000000EDA103084C
:102029007C180020040000005C6A04080C00000011
:10203900519F03087018002004000000686A040812
:102049000C000000B9A1030864180020000000007A
:10205900746A040803000000597003084C18002032
:1020690008000000806A040803000000555F0308A7
:10207900A41B0020000000007C650408010000008A
:102089000000000000000000000000000000000047
:102099000D0000000000000000000000000000002A
:1020A9007465040800000000000000000000000042
:1020B90000000000886A0408040000009171030808
:1020C90000000000000000007C6504080100000019
:1020D90000000000000000000000000000000000F7
:1020E9000D000000000000000000000000000000DA
:1020F900D46A04080000000000000000000000008D
:1021090000000000544204080C0000000000000018
:10211900DC18002004000000E46A0408080000003C
:1021290000000000D018002004000000F06A040834
:102139000800000000000000C4180020040000008E
:10214900F86A04080800000000000000B818002020
:1021590004000000006B04080800000000000000F3
:10216900AC18002004000000086B040808000000F7
:1021790000000000A018002004000000106B0408F3
:10218900080000000000000094180020040000006E
:10219900186B0408080000000000000088180020DF
:1021A900040000007C650408010000000000000034
:1021B9000000000000000000000000000D00000009
:1021C900000000000000000000000000206B04086F
:1021D9000E000000C96F03080000000000000000A5
:1021E900E8180020286B04080E0000000000000019
:1021F900000000000000000060190020306B040896
:102209000E000000000000000000000000000000B7
:10221900001A0020709700200400000058320408BA
:1022290098970020E0150C17000000006D9700201A
:1022390008000000083204086E970020050000001D
:102249006C320408386B04080E000000000000001E
:102259000000000000000000501A00202D202D2D44
:10226900202D2D2D2D202D2D2D00000000000000EA
:102279000000000000000000000000000902430007
:10228900020100C032090400000102020100052414
:10229900001001052401000104240202052406009E
:1022A90001070582030800FF09040100020A000072
:1022B90000070501024000000705810240000000F7
:1022C900FF0000000001010101000000AA55030000
:1022D9009FAA5505010000AA550701000001AA554A
:1022E9000B010000AA5509020000000001000000CE
:1022F900040309041201000202020040830440574A
:102309000002010203010000AD830308AD82030846
:10231900298403088D7D0308C18003089D7D030876
:10232900B97D0308657D0308557D03080000000099
:1023390000000000685E0C0043000000000000007F
:102349000000000000000000000000000000000084
:102359000000000000000000430000000000000031
:102369000000000000000000000000000000000064
:102379000000000000000000430000000000000011
:102389000000000000000000000000000000000044
:1023990000000000000000004300000000000000F1
:1023A9000000000000000000000000000000000024
:1023B90000000000000000004300000000000000D1
:1023C9000000000000000000000000000000000004
:1023D90000000000000000004300000000000000B1
:1023E90000000000000000000000000000000000E4
:1023F9000000000000000000430000000000000091
:1024090000000000000000000000000000000000C3
:10241900000000000000000069DF0308A9DD0308CF
:1024290000000000C96B040866650408F946040841
:10243900F9460408F9460408F9460408F946040867
:10244900F9460408F9460408F9460408F946040857
:10245900FFFFFFFFFFFFFFFFFFFFFFFFFFFF000081
:1024690001004153434949000000000000000000F9
:102479000000000000000000000000000000000053
:1024890000004153434949000000000000000000DA
:102499000000000000000000000000000000000033
:1024A90000000000081E00200000000000000000DD
:1024B9000000000000000000000000000000000013
:1024C9000000000000000000000000000000000003
:1024D90000000000000000000000000000000000F3
:1024E90000000000000000000000000000000000E3
:1024F90000000000000000000000000000000000D3
:0C250900000000000000000001000000C5
:10800000436B826A816930B41C68456A24F00104BC
:108010001144AA421C60D9600DD3016900248A1A58
:108020005A6084621A68002142F0010280F84C1004
:1080300030BC1A607047AA1A5A608562F2E700BF26
:10804000436A8269F0B4D154436A0469426B0133D4
:10805000A34228BF00234362FAB1116811F0010165
:1080600001D0F0BC7047856A1768866927F0010760
:108070002E449D421760D6600BD3641B546081620E
:108080001368002143F0010380F84C10F0BC13602A
:1080900070475D1B55608362F2E7826DD36843F0E1
:1080A0008003D360DDE700BF026B10B462B1836C64
:1080B000C2684469D11A013B615C5DF8044B08BF9A
:1080C00013468364C8B27047016A4369C4685B5C45
:1080D0000131A14228BF114601625DF8044BD8B2BC
:1080E000704700BF436B13B190F84C007047836A30
:1080F000406A181AB0FA80F040097047416A836AF2
:1081000099420AD3CB1A416B026961B14968501E8A
:108110000B4483420AD2C01A704702691144CB1A39
:10812000416B0029F2D1501EC01A704700207047E1
:10813000036B43B1826C5B6893422FBF981AC0688F
:108140009B1AC0187047C269036A9A422FBFD01A9F
:10815000C0688018C01A70470A4B30B503F1140488
:1081600093F900205D78072AC8BF143A81180433B8
:108170000D7313F8025C855413F8012C0A76A342A0
:10818000EED130BD3404040803682DE9F041DF6905
:108190001FB13B46BDE8F0411847002A164611DDE5
:1081A00004460D460E4400E023689B68204698472D
:1081B0000028F9D0236815F8011B1B682046984752
:1081C000AE42F1D1BDE8F08100233C214222017092
:1081D00042708370C370704710B5084B03F10C01F7
:1081E00093F900205C78845402449C78D470DC7845
:1081F000947104338B42F3D110BD00BF48040408CE
:1082000030B4446814B12368A5885D83036840F2E4
:10821000E93001E0002833D01D89013815F0020F44
:1082200080B2F7D089B2998140F2E93101E00029AA
:1082300050D01889013910F0010F89B2F7D099890F
:1082400040F2E93101E000292FD01889013910F0FE
:10825000020F89B2F7D092B29A8140F2E93201E07E
:10826000002A4BD01989013A11F0010F92B2F7D0D0
:108270009B8914B12368A2881A83012030BC7047FF
:108280002C498B4208D0A1F578418B424CD001F5A6
:1082900080618B42D4D10220274901EB0010418933
:1082A000013189B241814189CAE7224A934208D00B
:1082B000A2F57842934235D002F580629342D8D13C
:1082C00002211D4B03EB01114B8901339BB24B8102
:1082D0004B89CEE71748834207D018498B4227D0F5
:1082E00001F580618B42ABD10221134800EB0111F3
:1082F0004889013080B248814989A1E70D498B4204
:1083000007D00E4A934211D002F580629342B0D159
:108310000222094B03EB0212538901339BB25381B2
:108320005389A6E70121CCE70120B5E70122F0E758
:108330000121DAE7003001403CB90020003800405C
:10834000002870B51EDB0928044620DD012303EB5D
:1083500083035B00B0FBF3F2092AF8D87BB10E4E21
:10836000B4FBF3F00928CCBF57223022A6FB03E56B
:10837000024403FB1044EB0801F8012BF0D1002369
:108380000B7070BD2D230B7040420131DBE73030A4
:1083900001F8010BF3E700BFCDCCCCCC884230B460
:1083A0004FF001042ED301FB04F4B0FBF4F58D4231
:1083B000F9D284B1AAB901E0B0FBF4F5092DCCBF24
:1083C000572230222A4404FB150003F8012BB4FB8A
:1083D000F1F4002CF0D100221A7030BC7047B0FBD1
:1083E000F4F5092DCCBF372230222A4404FB1500B6
:1083F00003F8012BB4FBF1F4002CF0D100221A7029
:1084000030BC70470546002AEBD1D7E703685A1CF9
:1084100002601970704700BF2DE9F047089C25786D
:10842000002B804689460CBF4FF0200A4FF0300ADF
:10843000661C35B3002A29DD334601E0024698B1B7
:1084400013F8011B501E0029F8D1971E60B13D465C
:10845000013D51464046C8476B1C002BF8DC25788F
:1084600027EAE770013055B1041B29464046C8474A
:10847000301916F8015B002DF7D1BDE8F087BDE893
:10848000F087002A04DC2846BDE8F0870020EBE7EF
:10849000571EDCE70A44914251D030B441F2210426
:1084A00011F8013B80EA0320430010F4004F84EAF6
:1084B00003059BB2ADB208BF1D466B0015F4004F1B
:1084C00084EA03009BB280B208BF1846430010F450
:1084D000004F84EA03059BB2ADB208BF1D466B0096
:1084E00015F4004F84EA03009BB280B208BF18461F
:1084F000430010F4004F84EA03059BB2ADB208BFFD
:108500001D466B0015F4004F84EA03009BB280B255
:1085100008BF1846430010F4004F84EA03059BB2DD
:10852000ADB208BF1D466B0084EA030015F4004F8E
:1085300085B298B218BF28468A42B1D130BC704784
:1085400083684268D0ED037A00EB830101339342E4
:1085500081ED040A836004BF0023836000EB830382
:1085600093ED047A036870EE277A9A42C0ED037A9D
:1085700077EEC77AC0ED037A0CDA013307EE103AD2
:10858000F8EEC76AB7EE007A87EEA60A036030EE0F
:10859000070A704707EE102AB8EEC77A87EE870AF7
:1085A000704700BF90ED097A90ED004AD0ED0A6A5D
:1085B000D0ED014AD0ED047A90ED035AD0ED025A85
:1085C000A4EE007AB0EE406AB0EE470AB0EE667AEA
:1085D000A6EE247A67EEC07AA0EE457AE6EE257A1A
:1085E00080ED097AC0ED0A7A704700BFD0ED057AB8
:1085F00090ED013AD0ED003AD0ED064A90ED024AF6
:1086000090ED077A90ED035A90ED086AD0ED045A88
:10861000C0ED067AF0EE406A27EE830AC0ED056AE7
:10862000A3EEA60A80ED087AA4EE240AA5EE470A76
:10863000A5EEC60A80ED070A704700BFD0ED007AAC
:1086400090ED017A30EE670AE7EE007AB0EE670A45
:10865000C0ED007A704700BF704700BF2DE9F04FB2
:10866000DFF8F8C1DFF8F8E1BCF80A70DEF8006066
:10867000BCF80C30BCF808A03C028BB0361B4FF0A5
:108680000004CDE90034009CBCF806304FEA1765C1
:108690004FF0000767EB0507B946B046A4FB066735
:1086A0000024CDE90634009C002304FB0977002454
:1086B000CDE90034AAFB0823CDE90223039AF30D88
:1086C00000930AFB09230393009B43EA472300938B
:1086D000029B4FEAD31AFB150193039B4AEA436AB4
:1086E000DDE9002344464D46CDE90845069C12F5D8
:1086F000FA62A4FB086743F1000304FB0977CDE9A4
:108700000623BCF80440039BBCF802204FEAE31B9D
:10871000230C059323040493340A44EA07643D12AE
:10872000DDE904674FEAC23816EB0A0647EB0B0790
:1087300018EB0408DDE906344FEA524949EB050914
:10874000B3F5FA6F74F10004B246BB463CDADDE9DA
:108750000067BC00B20044EA9673B41847EB030507
:1087600022463C462B4602FB04F406FB0344A2FBD4
:1087700006232344940844EA83749D105B104FEA57
:108780003202B8EB040869EB0509BAEB020A6BEB9D
:10879000030BDDE90623304C4FF0FF35A242AB411D
:1087A0002CDBDDE90856A5FB052305FB06F403EBEE
:1087B0004403D40F44EA4304DD17DDE90623121B0A
:1087C00063EB0503CDE90623DEF80440A4FB082390
:1087D00004FB0933540D44EAC3245D15B4EB0A0AC3
:1087E00065EB0B0B4FEADA3343EA4B4300B103600E
:1087F00009B1069B0B600BB0BDE8F08F40F6AC52A0
:10880000B4184FF0000347EB03052246A2FB0223F6
:1088100004FB05F403EB4403941843EB0305A4188D
:108820005D414FEA850CA6004CEA947CB41A6CEBCF
:108830000305DF00D6006D104FEA340447EA527793
:10884000921B63EB0703B8EB040869EB05091AEB0D
:10885000020A4BEB030BA4E724FAFFFF242C0020B1
:108860006C1E00202DE9F04FDFF81CB2DFF81CE28F
:10887000BBF80020DEF80860BBF90430BBF90250F9
:10888000BBF90A80C2EB261404FB04F42413520043
:10889000C2EBE60203FB04F305FB02F29B1303EBBE
:1088A000E223B3F5FA364FEAE37589B045F1FF37B5
:1088B0003246A6FB0645CDE9024502FB07F205EB71
:1088C0004202CDE90467029EBBF90840039208FB0F
:1088D00002FC4FEAE87906FB09CC3A46A8FB068978
:1088E000049ECBF81830E51704FB02F206FB0522C4
:1088F000A4FB0667E14417444FEA182242EA0962E2
:1089000000924FEA292201923D03DDE90078340309
:1089100045EA16553F19BBF80660069048EB050876
:108920003C1C48F5004503EB8302A4FB068906FBCB
:108930000599803213124FEA69064FEAE9770793E7
:1089400056EA07038A4600F09280DDE90489BBF904
:108950000E20DEF80C40BBF910004946C4F5801E1D
:10896000D317DDE9024502FB01F108FB0311A2FB6D
:1089700008230B444FEA43492B46C11700FB03F37E
:1089800004FB0133A0FB0401BBF90C401944E300D4
:1089900001937346DC170023009349EAD2394FEA6A
:1089A0004248DDE9002310EB080041EB0901E5072F
:1089B00012184FEACE744B4145EA5E05A41A65EBE6
:1089C0000305221945EB050312196B41990190012A
:1089D000801841EA926159418B00820043EA90730A
:1089E000101943EB05018B00820043EA9073104697
:1089F0000019194632463B46694134F0F1FDBBF996
:108A000016204C13450B45EAC14502FB04F6D3176B
:108A100005FB0366A2FB05233344BBF9146002FB8C
:108A200004F405FB034406FB01FEA2FB0523F71734
:108A3000234400FB07EE540EA6FB0067774444EA8C
:108A4000C3144FEAD64800194FEA636548EA47382D
:108A500069414FEAE74918EB0008BBF9124049EBBE
:108A600001094FEA182646EA096620013618069BD6
:108A70000BB1360A1E60BAF1000F02D0079BCAF88C
:108A8000003009B0BDE8F08F382C00206C1E0020AB
:108A9000704700BF704700BF4FF400630382704708
:108AA0004FF400630382704750F8043C012280F8C1
:108AB0003520143803B11847704700BFBFF34F8FFC
:108AC0000549064BCA6802F4E0621343CB60BFF36A
:108AD0004F8F00BFFDE700BF00ED00E00400FA0586
:108AE000F8B5027B466903681F2A2DD9A2F120053B
:108AF0005F682024AC402742114617D01022AA40BC
:108B0000DC60DA605A68EA40D40749D4716B756A50
:108B10000A68B46A22F00102A5420A6037D1012234
:108B200086F84C20027B11461F2A20D920390822C2
:108B300058688A40024200D0DA600422586802FA7B
:108B400001F1014221D1F8BD20241D689440254245
:108B500011460CD0102191409C6099601968D14059
:108B6000C907D3D5012101FA02F29A60CEE70822A3
:108B700018688A40024200D09A600422186802FAFB
:108B800001F101420BD09960F8BDD960F8BD0446EF
:108B90003046FFF735FA227B23681146C4E7F8BD5B
:108BA000012202FA05F5DD60B0E700BF70B4037B77
:108BB00004681F2B08D9203B2021626801FA03F3C7
:108BC0001A421CD170BC70472021226801FA03F3BD
:108BD0001A42F7D042691449582000FB021251682A
:108BE0005689CD680868296821F0010129608289C9
:108BF00092B222EA06028281A36070BC7047426989
:108C00000949582000FB021251685689CD6808684E
:108C1000296821F001012960828992B222EA0602C4
:108C20008281E36070BC70473831002030B4094B5A
:108C30001C786CB1084A002502EBC40411689388C3
:108C40004D628889083203439BB2A2428B81F5D1E1
:108C500030BC7047583500205C35002010B4037BD1
:108C600001681F2B09D9203B20224C6802FA03F32C
:108C70001C4214D15DF8044B704720220C6802FAA4
:108C800003F31C42F6D00C4A4068002414700268BA
:108C90005DF8044B22F0010202608B607047064AC7
:108CA00040680024147002685DF8044B22F0010251
:108CB0000260CB60704700BF8E2D0020F0B5C4006D
:108CC00022189200AE498B585B689D8AADB2EEB215
:108CD000F7070A445CD4B70732D5BFF35F8F167E1F
:108CE000F6B2012E00F0C780A64D1A8BBFF35F8F3E
:108CF000221801EB8202167E022E00F0D580221887
:108D000001EB8202167E032E00F088809A8895F986
:108D1000106092B242F480629A80221801EB8202C3
:108D2000127E013296425BD1AA7C00266E74002A24
:108D300040F09580204401EB800000234375F0BD96
:108D400077074ED416F0400600F0C9808D4D1E8A7C
:108D500095F910E0176AF6B207F80E605FFA8EFE1A
:108D60000EF1010C4FFA8CFC177E85F810C00CF147
:108D700003029742664600F01C81221801EB820232
:108D8000127E9445C9D10EF1020676B22E74C4E764
:108D90001E887C4D26F400663604360C1E801E8824
:108DA000B6B246F480661E80967E00272F74002E91
:108DB00048D06E7C002E42D0221801EB82020126A0
:108DC000127E6E74022A00F0B980221801EB820232
:108DD000927D42F001021A82204401EB8000037E62
:108DE000F0BD684D967E0127AF74002E73D06E7C67
:108DF000002E7BD1221801EB8202527E002A00F065
:108E0000A3801A882E7C92B2013642F4007276B2A8
:108E10001A802E741A88D205FCD47EE7927E002A2E
:108E20003FF474AF6A7C002A3FF470AF9A8895F9DA
:108E3000106022F480621204120C9A806DE7D27DD9
:108E4000FF2AB9D0221801EB8202967D06F0FE06B9
:108E50001E82D37DFF2BBFD0FF232B74BCE79A88E3
:108E600022F4407212042044120C01EB80009A801C
:108E700000234375F0BD927E424D002A3FF435AF8A
:108E80006A7C002A3FF431AF1A8822F4806212040F
:108E9000120C1A80BFF35F8F1A8B1A88AE7492B2CD
:108EA00042F400721A8031E7927E002A3FF427AF25
:108EB0006A7C002A3FF423AF1A8895F9106022F4E7
:108EC00080621204120C1A809A8822F480621204C2
:108ED000120C9A8021E76A7C002A8BD091E715F06A
:108EE000800F284D3AD195F9106016E7167ED2F81A
:108EF00020E01F88022E95F9106045D927F480677D
:108F00003F043F0C1F801F8AFFB20EF806701F88B7
:108F1000D2F820E0BFB247F400771F80F2B21F8A78
:108F2000561C76B2FFB20EF806709F88961CBAB235
:108F300076B242F480622E749A806BE71A8892B2FD
:108F400042F400621A8040E71A8895F9106092B2E4
:108F500042F4807201271A806F745BE795F91070F4
:108F6000B7F1FF3F2CD0D669F65D1E8292F818E06B
:108F700001377AB2964516462A747FF4CEAEA3E73F
:108F8000CCB800206C1E0020BFB247F400771F80D1
:108F90001F8AFFB20EF80670F6B21F8AD2F820E0E0
:108FA000721C52B20336FFB276B20EF802702E7403
:108FB00030E79A8822F480621204120C9A80DCE670
:108FC000D77D1F822E74957E1DB9127E002A7FF4F4
:108FD00003AF9A8822F480621204120C9A80FBE696
:108FE00090F8493013B1002280F8492018467047A4
:108FF00070B5044682B01830256D94F85C106B464D
:109000000622A847A8B19DF804009DF800609DF8CD
:1090100001109DF802509DF803209DF8053041EAAB
:10902000062143EA002342EA0522A184E284238543
:10903000012002B070BD00BF70B5044682B0083098
:10904000256A6B4606223B21A847A8B19DF804007B
:109050009DF800609DF801109DF802509DF80320D6
:109060009DF8053041EA062143EA002342EA052241
:109070006182A282E382012002B070BD00230360FE
:1090800043608360262303702723C3700123837109
:1090900043727047F8B50468C4F30D0405460E46E4
:1090A00004B32F682EF070FA092840F08880454CF0
:1090B000236923F440732361236943F4007323611C
:1090C000236943F0010323613E602EF05DFA2369BA
:1090D000092823F00103236171D12B6804332B602D
:1090E0000020F8BD384B394A93422BD902F5804213
:1090F000934226D902F5804293422AD902F5804252
:10910000934228D902F58032934226D902F50032E3
:10911000934224D902F50032934222D902F500325B
:10912000934220D902F5003293421ED902F58022E3
:1091300093421CD9B3F1016F1BD3052004F0AEF9A3
:10914000FBE708242EF020FA092814D04FF0FF3056
:10915000F8BD1024F6E71824F4E72024F2E72824C9
:10916000F0E73024EEE73824ECE74024EAE748242F
:10917000E8E75824E6E7134F3B6923F440733B616B
:109180003B6943F400733B613B6923F0F8033B61A7
:109190003B6943F002031C433C613B6943F4803369
:1091A0003B612EF0F1F93B6923F002033B613B691F
:1091B000092823F0F8033B613FF473AFC6E76FF073
:1091C0000100F8BD003C024000400008FF3F0008DD
:1091D000F8B504460D468E180027B54201D1206926
:1091E000F8BDE368591CE160234415F8012B1A729D
:1091F0000429F2D1206918B9A1682046FFF74AFF77
:109200002061E760E9E700BFF0B583B004466B4634
:10921000062203211E2032F037FC00283CD09DF8A6
:1092200000509DF801109DF802709DF803209DF8F4
:1092300004609DF8053041EA052142EA072243EA2D
:10924000062309B212B21BB2144D06EE901A07EEB5
:10925000102A07EE903AF8EEE66A95ED005AD5ED41
:10926000025A95ED016AB8EEC77AF8EEE77A66EE33
:10927000856A27EE257A67EE867AFDEEE66ABDEE10
:10928000C77AFDEEE77A16EE901A17EE102A17EE5F
:10929000903A2180A280638003B0F0BD00000020DE
:1092A00000B583B001AB03220021772032F0ECFB44
:1092B0009DF805309DF804209DF806001B0243EA46
:1092C0000243184303B05DF804FB00BF08B5FFF785
:1092D000E7FF014B586008BD6C1E002008B5FFF782
:1092E000DFFF014B186008BD6C1E002070B582B016
:1092F0006B460622F721762032F0C6FB9DF801204E
:109300009DF804309DF800609DF803509DF80240E0
:109310009DF80500074912011B0142EA063243EAA3
:10932000053342EA141243EA1013CA608B6002B09C
:1093300070BD00BF6C1E0020682032F0A5BB00BFCE
:1093400008B505F08BFB044B5B68C01AC0F5FA50FA
:1093500020EAE07008BD00BF787F002000B5002142
:1093600083B00A202AF0B2FF0F210A202AF0AEFFB4
:1093700001AA032110202AF0D1FF9DF90430DFED6E
:10938000277ADFED275A06EE103A9DF9053006EEF2
:10939000903A9DF9063007EE103AB8EEC66AF8EE3C
:1093A000E66AB8EEC77A76EEE76A36EE676A37EEB7
:1093B000677AF7EE007AB0EE675AA6EE255A194B97
:1093C0000021B0EE456AB0EE675AA6EEA55A0A2013
:1093D000E7EE257AF3EE0E5A26EE256A25EE257A7B
:1093E00067EEA57A83ED036A83ED047AC3ED057A0F
:1093F0002AF06CFF0DF10302012102202AF08EFFFA
:109400000DF10302012109202AF088FF01210A2021
:109410002AF05CFF012003B05DF804FB000000436C
:109420000000803B0000002070B582B00446694611
:1094300018302AF0C9FCA8B19DF805009DF801601C
:109440009DF802109DF803509DF804209DF8063009
:1094500041EA062143EA002342EA0522A184E2848C
:109460002385012002B070BD38B5254B1C68236BE5
:1094700073B1A36D626BCAB1998A1A88C90592B299
:1094800001D5D20700D438BD4FF6F7721A8038BD27
:10949000A36D99891A88890692B2EBD59206E9D50F
:1094A000E26ACAB1988880B29047E2E799891A883F
:1094B0000D0692B2E0D51006DED5A26A616A8A4234
:1094C00019D0A1692569885C98800132B2FBF5F159
:1094D00005FB1122A262CFE79B88E2696169DBB2DA
:1094E0008B54E269E068A36D0132B2FBF0F100FB3E
:1094F0001122E261BEE7DA6822F08002DA60BBE79F
:10950000A864002003685B6A03B11847704700BF76
:1095100003681B6A03B11847704700BF03682DE951
:10952000F041DF691FB13B46BDE8F0411847002A12
:10953000164611DD04460D460E4400E023689B6884
:10954000204698470028F9D0236815F8011B1B68AE
:1095500020469847AE42F1D1BDE8F08103689B698F
:10956000184700BF03685B69184700BF03681B69A1
:10957000184700BF0368DB68184700BF03689B6893
:10958000184700BF03685B68184700BF03681B6883
:10959000184700BF014B1868F8E700BF941F002070
:1095A00038B50C46097849B1054601342B68284680
:1095B0001B68984714F8011B0029F7D138BD00BF7C
:1095C000064B53F820302BB11A689B8851690B4227
:1095D00001D1138370475383704700BFF8BA00204E
:1095E00010B50409013C032C17D80D4B33F8142097
:1095F00000F00F0042FA00F313F001030DD0012335
:1096000003FA00F00138104034F03AF8054A064BEE
:10961000125D104403EBC00010BD002010BD00BF60
:10962000E4330408E03304086CB900202DE9F04F5E
:109630004A484B494B4B4C4C4FF0010A4FF0020942
:109640004FF004084FF0080C4FF0100E2027402672
:10965000802530F8022B12F0010F03D01960A3F817
:1096600004A0083312F0020F03D01960A3F804908D
:10967000083312F0040F03D01960A3F804800833F4
:1096800012F0080F03D01960A3F804C0083312F0D9
:10969000100F03D01960A3F804E0083312F0200F74
:1096A00002D019609F80083312F0400F02D0196079
:1096B0009E80083312F0800F02D019609D8008331D
:1096C00012F4807F05D04FF4807B1960A3F804B0BA
:1096D000083312F4007F05D04FF4007B1960A3F823
:1096E00004B0083312F4806F05D04FF4806B19601A
:1096F000A3F804B0083312F4006F05D04FF4006BE8
:109700001960A3F804B0083312F4805F05D04FF459
:10971000805B1960A3F804B0083312F4005F05D031
:109720004FF4005B1960A3F804B0083312F4804FC3
:1097300005D04FF4804B1960A3F804B00833D20B66
:1097400004D04FF4004219609A80083301F580611B
:10975000A1427FF47EAFBDE8F08F00BFE433040880
:10976000000002406CB900200010024000286AD0BE
:1097700003682DE9F04F03F13F4404F57E045F4E8A
:10978000A40A0125345D04F01F066409032C05FAC0
:1097900006F559D0042C00F0AC80022C59D08588F5
:1097A000B5FA85F0C0F11F0080B2C40803EB840451
:1097B00000F00700266A80000F27874026EA070688
:1097C0002662276A01F003068240701E3A43012890
:1097D000C1F3810CC1F300182262C1F341113DD9DC
:1097E0000024224601274FF0030E03E0102A04F163
:1097F000020426D007FA02F0A84302F10102F5D1D3
:10980000D3F800C00EFA04F0C04300EA0C0CC3F811
:1098100000C0D3F8008006FA04FC4CEA080CC3F838
:1098200000C0D3F80CC000EA0C00D860D3F80CC01C
:1098300001FA04F040EA0C00102AD86004F1020496
:10984000D8D1BDE8F08F70472D4C266C3543256488
:10985000A5E72B4C666C35436564A0E70020024603
:109860004FF0010E4FF0030904E00132102A00F11D
:1098700002003CD00EFA02F737EA0504F5D1D3F81E
:1098800000A009FA00F4E4430AEA040AC3F800A0BD
:10989000D3F800B006FA00FA4AEA0B0AC3F800A0AF
:1098A000D3F808A004EA0A0AC3F808A0D3F808B05D
:1098B0000CFA00FA4AEA0B0AC3F808A0D3F804A08D
:1098C0002AEA07075F60D3F804A008FA02F747EA1C
:1098D0000A075F60DF683C40DC60DF6801FA00F483
:1098E00001323C43102ADC6000F10200C2D1BDE825
:1098F000F08F034C266B3543256350E7B0330408E3
:1099000000380240002855D0026802F13F4303F5B9
:109910007E032DE9F04F9B0A544DEB5C03F01F05CD
:109920005B090124032B04FA05F444D0042B00F056
:109930009780022B44D001F00306731E012BC1F364
:10994000810CC1F300188588C1F341113DD9002471
:10995000234601274FF0030E03E0102B04F102040D
:1099600026D007FA03F0A84303F10103F5D1D2F89A
:1099700000C00EFA04F0C04300EA0C0CC2F800C0AC
:10998000D2F8008006FA04FC4CEA080CC2F800C0C9
:10999000D2F80CC000EA0C00D060D2F80CC001FA7A
:1099A00004F040EA0C00102BD06004F10204D8D17E
:1099B000BDE8F08F70472E4B1D6C2C431C64BAE73A
:1099C0002B4B5D6C2C435C64B5E7002003464FF0E5
:1099D000010E4FF0030904E00133102B00F10200E7
:1099E0003CD00EFA03F737EA0504F5D1D2F800A00F
:1099F00009FA00F4E4430AEA040AC2F800A0D2F823
:109A000000B006FA00FA4AEA0B0AC2F800A0D2F83F
:109A100008A004EA0A0AC2F808A0D2F808B00CFAB2
:109A200000FA4AEA0B0AC2F808A0D2F804A02AEA0F
:109A300007075760D2F804A008FA03F747EA0A07B5
:109A40005760D7683C40D460D76801FA00F401330E
:109A50003C43102BD46000F10200C2D1BDE8F08F6E
:109A6000034B1D6B2C431C6365E700BFB033040838
:109A70000038024010B1036882885A83704700BFE3
:109A800010B1036882881A83704700BF10B5014681
:109A900000BF064C2068FFF7EDFF084632F082F861
:109AA0002068FFF7EDFF00BF10BD00BF1465002068
:109AB00018B10368828809B95A8370471A837047BE
:109AC00010B40A4B0A4A1C7801238340234052F801
:109AD000200029B9B3FA83F149095DF8044BE7E79F
:109AE000191C18BF01215DF8044BE1E7F4BA00200E
:109AF000F8BA002030B1036882881B691A4214BF8B
:109B000001200020704700BF38B5044690F84D0092
:109B100000285AD104F11805636D80226B21284674
:109B20009847642005F040F8636D072268212846B5
:109B30009847642005F038F8636D00226B212846B1
:109B40009847642005F030F8636D01226B212846A8
:109B500098470F2005F028F894F84720636D022AF3
:109B60008CBF1A2218221B21284698470F2005F087
:109B70001BF8636D18221C21284698470F2005F01A
:109B800013F8636D94F846201A21284698470F2051
:109B900005F00AF8636D94F8482019212846984783
:109BA000642005F001F8636D10223721284698479C
:109BB0000F2004F0F9FF2846636D012238219847F1
:109BC0000F20BDE8384004F0EFBFFFF709FD054660
:109BD000FFF790FF014600289CD1D5B12023E87102
:109BE000AB712846FFF78EFE21460F4B41F8143F1C
:109BF00028462AF07FF8AB88B3FA83F3C3F11F033A
:109C0000012212FA03F385D008490A6813430B6056
:109C100080E72946FFF776FE2146034B41F8143FC3
:109C200028462AF067F875E7A98A0008003C014039
:109C300010B504460120A269138823F040031B04D9
:109C40001B0C138013889BB223F0380343F03003BE
:109C5000138013889BB243F04003138004F04AFF43
:109C60002046FFF751FF10226A2104F11800FEF789
:109C7000C7FA642004F098FFA06932F007F80120C9
:109C8000BDE8104004F036BF2DE9F0410B4E3468BA
:109C900073691C400FD0DFF828800127B4FA84F3E1
:109CA000C3F11F0307FA03F558F823000368984728
:109CB000AC437561F2D1BDE8F08100BF003C0140CA
:109CC000E07E00202DE9F0410B4E346873691C40A2
:109CD0000FD0DFF828800127B4FA84F3C3F11F0303
:109CE00007FA03F558F8230003689847AC437561F9
:109CF000F2D1BDE8F08100BF003C0140E07E0020D1
:109D00002DE9F0410B4E346873691C400FD0DFF829
:109D100028800127B4FA84F3C3F11F0307FA03F57F
:109D200058F8230003689847AC437561F2D1BDE849
:109D3000F08100BF003C0140E07E00202DE9F041B1
:109D40000B4E346873691C400FD0DFF82880012760
:109D5000B4FA84F3C3F11F0307FA03F558F823009C
:109D600003689847AC437561F2D1BDE8F08100BF4C
:109D7000003C0140E07E00202DE9F0410B4E3468AC
:109D800073691C400FD0DFF828800127B4FA84F3F0
:109D9000C3F11F0307FA03F558F823000368984737
:109DA000AC437561F2D1BDE8F08100BF003C0140D9
:109DB000E07E00202DE9F0410B4E346873691C40B1
:109DC0000FD0DFF828800127B4FA84F3C3F11F0312
:109DD00007FA03F558F8230003689847AC43756108
:109DE000F2D1BDE8F08100BF003C0140E07E0020E0
:109DF000084A094808B5536C43F480435364002172
:109E0000402236F062FA054B4FF0FF321A60C3F879
:109E1000032008BD00380240E07E0020207F0020A3
:109E200003685B6A184700BF2DE9F04104461846F5
:109E30000D461646984632F029FF2768E6722844F8
:109E4000A07229467D69434632462046AC46BDE8AD
:109E5000F0416047036810B504461B6898472368C3
:109E600020469B689847A37B0133A37310BD00BFB6
:109E700010B5036804469B689847FF23012263736B
:109E8000227310BD08B5FFF7ABFB38B12C228271ED
:109E90000022C2712021BDE8084033E508BD00BFA3
:109EA000F0B484894FF6FF764FF47A7463B3002AD6
:109EB0003CD01778013201E0B4421AD00589013C48
:109EC00015F00205A4B2F7D0BCB284814FF47A74C5
:109ED00002E0BCB2B4420CD0058915F0010504F1D2
:109EE000FF37F6D08589ADB209B10D700131013B64
:109EF000DCE7104B98420BD0A3F57843984217D07B
:109F000003F58063984202D00120F0BC704702251F
:109F1000094B03EB05156B8901339BB26B81688993
:109F200080B2003018BF0120F0BC7047FF27C5E7A2
:109F30000125EDE7003001403CB9002070B5044632
:109F400040681E4610B103688088588341F0800144
:109F5000206840F2E93300E0F3B10589013B15F0D8
:109F6000020F9BB2F8D08BB2838140F2E93300E05C
:109F700093B10589013B15F0010F9BB2F8D083899D
:109F8000134631460022FFF78BFF636813B11A684E
:109F90009B881383012070BD0A49884207D00A4B71
:109FA00098420DD003F580639842E9D10223074916
:109FB00001EB03135989013189B259815B89DFE7CC
:109FC0000123F4E700300140003800403CB9002094
:109FD00038B50B4C2378054653B90A4B627818689C
:109FE00049212B4600252570FFF7A8FF012038BD29
:109FF000FFF7A6F90028F0D004F07CFDEDE700BFE4
:10A00000787F0020747F0020F0B54A4CE57C012D5C
:10A0100083B013D028D3022D0DD1474B1B780646B1
:10A02000002B77D16846FFF7D3FF20B19DF80630AB
:10A0300013F0030022D0002003B0F0BD3E4E337871
:10A04000002B62D16846FFF7C3FF9DF8003008B1CE
:10A05000DB0764D40023E37433784BB1002301336E
:10A060000020E37403B0F0BD334E3378002BF5D1FC
:10A07000012102202AF080F9E37CF0E79DF801E05D
:10A080009DF800109DF803709DF802209DF8055082
:10A090009DF80430E07441EA0E2142EA072243EAC7
:10A0A000052309B212B21BB2494252425B42234815
:10A0B00006EE901A07EE102A07EE903A90ED035A3A
:10A0C000D0ED045A90ED056AF8EEE66AB8EEC77A6C
:10A0D000F8EEE77A66EE856A27EE257A67EE867AED
:10A0E000FDEEE66ABDEEC77AFDEEE77A16EE901A4F
:10A0F00017EE102A17EE903A31807280B38001215A
:10A100000A202AF0E3F803B0F0BDFFF719F90028A0
:10A1100098D090E7FFF714F900288CD182E73378C4
:10A1200023B9072103202AF027F9E57C0135E574DE
:10A1300081E700BF6C1E0020787F00200000002017
:10A14000F8B50501684C694B625961199A4204EBF4
:10A15000050704BF01230B730646387A31F028FC4B
:10A160003B7A03F01F015B090122032B02FA01F283
:10A170006DD0042B66D0022B5CD0631901361879A0
:10A18000FFF72EFAF6B2074610B11223C67183719B
:10A1900063195879FFF724FA10B11323C67183713C
:10A1A00063199879FFF71CFA10B11423C6718371F3
:10A1B00066190A21F2793846FFF7D8FA7079FFF765
:10A1C0000FFAF2790A21FFF7D1FAB079FFF708FA0E
:10A1D000F2790A21FFF7CAFA6359454A934247D0F8
:10A1E000424A934250D0434A934259D0424A934202
:10A1F00062D0424A93426BD0414A93422CD02C44C5
:10A20000227BE2B901200222198801F4415141F474
:10A2100045710A4302431A809A8B22F400621204A9
:10A22000120C07219A8319821A8892B242F04002D6
:10A230001A80F8BD334B596A0A435A629DE70020E1
:10A240000246E1E72F4B19690A431A6195E72D4B46
:10A25000196A0A431A6290E702F564424FF400104B
:10A26000536A43F4001353622DF0EEF96359C6E7C5
:10A2700002F584324FF48050536A43F480535362A2
:10A280002DF0E2F96359BAE702F500324FF480404D
:10A29000136A43F4804313622DF0DEF96359AEE78D
:10A2A00002F5FE324FF40040136A43F40043136298
:10A2B0002DF0D2F96359A2E702F582324FF4005033
:10A2C000536A43F4005353622DF0BEF9635996E785
:10A2D00002F568424FF48010536A43F480135362CE
:10A2E0002DF0B2F963598AE73CB9002000380040EC
:10A2F00000300140003C004000340140005001406B
:10A300000054014000380240427A02B9704710B54B
:10A3100004460368406804F10A0198470023637209
:10A3200010BD00BF437A5A1C0344D2B242729972E4
:10A33000037A934200D802B9704710B50446036807
:10A34000406804F10A0198470023637210BD00BF02
:10A35000302828D0312828D0322828D0332828D0B7
:10A36000342828D0352828D0202828D0212828D0C3
:10A37000102828D0112828D0122828D0132828D017
:10A38000142828D0152828D0162805D0172808BF4B
:10A390000F2202D0002070470E22114B03EB420324
:10A3A00093F8210070470022F7E70122F5E7022227
:10A3B000F3E70322F1E70422EFE70522EDE70622A7
:10A3C000EBE70722E9E70822E7E70922E5E70A22A7
:10A3D000E3E70B22E1E70C22DFE70D22DDE700BF18
:10A3E0003404040870B5448806460D46C4F30B04D3
:10A3F00022460021284635F068FF3369094A934216
:10A4000009D3094A934206D2224628461946BDE896
:10A41000704033F0DBBC23B121462846BDE87040D4
:10A42000184770BDF0050008A9060008064B07494B
:10A430008B4202D30023184670471A88C2F30B02DE
:10A440009042F8D01433F3E790010008F0050008BB
:10A45000024A136823EA000010607047FC8700205E
:10A46000F8B51A4D2B789F2B2ED16B78BE2B2BD1A4
:10A4700005221749A81C35F073FF28BB072229467F
:10A480004FF6FF70FEF706F8124FEC1D22884AB116
:10A49000A618BE4218D2052A16D92146FDF7FAFFA2
:10A4A0003446F3E721460222FDF7F4FF0222A11809
:10A4B000FDF7F0FF0634084B641B1C8041F60F5378
:10A4C000C31A58425841F8BD0020F8BD00400008AA
:10A4D000EC33040800800008602500202DE9F04FCF
:10A4E000DFF85891504F8DB00326A7EB09071822CB
:10A4F0000DEB0200002135F0E8FE4C4BCDF8189032
:10A5000007971A69002A04DA494A5A6002F1883228
:10A510005A6001228DF82C20F322DA60454B464C1C
:10A5200018689A8804909B79ADF8142004A9072232
:10A5300006A88DF81630FEF74BFE072204A94FF649
:10A54000FF70FDF7A7FFDFF8F8B080464FF0000A74
:10A550005C4539D30CAC002524F82C5D0222214641
:10A5600006A8FEF735FE022221464046FDF792FF7F
:10A5700040BAC043ADF80800022202A906A8FEF7BF
:10A5800027FE099878B108ABC0F1040229461844A7
:10A5900035F09BFE0A9818B9089906A8FEF77AFDCF
:10A5A00000230A9009939DF82C300A9A23B11F4981
:10A5B0000B6943F000430B61013E2DD0002A96D178
:10A5C000FFF74EFF50B32CE065888DF80DA0C5F362
:10A5D0000B05AA1DADF808202288C2F30B01120B4F
:10A5E000ADF80A108DF80C2002A9062206A8FEF785
:10A5F000EFFD062202A94046FDF74CFF6168804648
:10A600002A4606A8FEF7E4FD616840462A46FDF7A3
:10A6100041FF143480469BE7002AD1D0052002F088
:10A620003DFF0DB0BDE8F08F00800008003C024007
:10A6300023016745740404089001000800400008E5
:10A64000F00500080378202B024600F10100F9D044
:10A65000092BF7D02D2B2CD02B2B03BF5378B7EE23
:10A66000000A0246B7EE000AA3F13001C8B2092879
:10A670009FED467A10D8F2EE046A07EE901AF8EED3
:10A68000E77A12F8013FE7EE267AA3F13001C8B26B
:10A690000928B0EE677AF0D92E2B4CD003F0DF03F7
:10A6A000452B0BD0F7EE007A67EE276A20EE260ADC
:10A6B00070475378BFEE000A0246D5E710B45178D0
:10A6C0002D2959D02B290ABF9178501C901C0024A9
:10A6D000A1F13003092B53D8002303EB830301EBD3
:10A6E000430310F8011FA1F13002092AA3F130033E
:10A6F000F3D9B3F59A7F28BF4FF49A73072B42D949
:10A70000DFED236A1A46F7EE007A083A072A67EE69
:10A71000A67AFAD803F007032BB1F2EE046A013BE4
:10A7200067EEA67AFBD124B3C7EE276A5DF8044B27
:10A7300020EE260A70475378A3F13001C8B20928E9
:10A7400002F10102AAD8F2EE046AF0EE665A07EEB0
:10A75000901AF8EEE77A12F8013F87EEA66AA3F1A5
:10A760003001C8B2092866EEA56A37EE067AEED93E
:10A7700094E767EE276AD9E7901C91780124A7E750
:10A78000F7EE007ACFE7F7EE007AC5E700000000A9
:10A7900020BCBE4CB5EEC00ADFED317AF1EE10FA06
:10A7A000CCBF30EE270A30EE670ADFED2E7A20EEBE
:10A7B000270A30B5FDEEC07A87B017EE904A0546FD
:10A7C00084EAE470002303A9A0EBE47001930093F2
:10A7D00002931FF0E5FA002CACBF20232D2303A821
:10A7E0008DF8003032F052FA012803A924D0022853
:10A7F0002DD0032805BF3023684668468DF8013008
:10A8000035F089FD684632F041FA0338C4B2224679
:10A810006946284635F0DDFD00232B55284632F0E9
:10A8200035FA2E22431C2A540DEB0401E81835F0AA
:10A830008FFD284607B030BD302368468DF80130C3
:10A840008DF802308DF8033035F065FDDAE73023FE
:10A8500068468DF801308DF8023035F05CFDD1E7A7
:10A860006F12033A00007A442DE9F041064615467E
:10A870000846B6FBF2F43CB905FB1464124B1B5DB1
:10A8800000F8013BBDE8F081B4FBF2F767B90E4B6D
:10A8900005FB174705FB1464DA5D00F8012B1B5D0F
:10A8A00000F8013BBDE8F081B7FBF2F8B8F1000F0A
:10A8B00002D04046FFF7D8FF05FB1878024B13F88B
:10A8C000082000F8012BE3E7F433040830B40268F1
:10A8D0001146531C036011F8024B0160D31C5178E0
:10A8E00003609378151D05601B0443EA0123D078AB
:10A8F000234343EA006030BC704700BF0368591C23
:10A900001A46016012F8021B0260587841EA0020E2
:10A91000704700BF38B504460068154633F056FA54
:10A9200022682A44226038BD036810B40A0E5C1CF9
:10A9300004601A7003680A0C5C1C04601A700368D7
:10A940000A0A5C1C04601A7003685A1C02601970C1
:10A950005DF8044B704700BF036810B40A0A5C1C22
:10A9600004601A7003685A1C026019705DF8044B89
:10A97000704700BF03685A1C026010B41970036866
:10A980000A0A5C1C04601A7003680A0C5C1C0460F0
:10A990001A700368090E5A1C026019705DF8044BA6
:10A9A000704700BF03685A1C026019700368090AE7
:10A9B0005A1C0260197070472DE9F047002488B0D6
:10A9C00080460F461E46A14605AD531C03931178E1
:10A9D00039B3252933D1931CCDF8109003935078C7
:10A9E00030284ED04FF0000AA0F13003DBB2092B23
:10A9F00042D96C2819D0642800F0938024D82528E7
:10AA00001CD063D9582876D063281BD131784046B2
:10AA1000B847039A531C0393117804360134002974
:10AA2000D7D1204608B0BDE8F087039B5A1C03929B
:10AA30001B78642B7CD02AD8252B54D12521404665
:10AA40000134B847039AC0E7732833D044D9752836
:10AA50004FD106F1040E30682B4600220A217646BB
:10AA6000FDF79CFC049A0095534639464046FDF795
:10AA7000D3FC039A0444A8E704AA03A91FF06CF9C5
:10AA8000B7E7D31C039390784FF0010AACE7732B20
:10AA900010D05BD9752B3AD0782B96D1A3F1580200
:10AAA000B2FA82F2306852092B4610210436FDF7C3
:10AAB00075FCD7E73368049A009339460023404673
:10AAC000FDF7AAFC04360444039A7EE70028B9D1B6
:10AAD000204608B0BDE8F0876E28B3D1039A3368EA
:10AAE00004361C6071E72AD9582BD7D0632B8DD040
:10AAF0006BE77828A6D1A0F15802B2FA82F230684A
:10AB000052092B461021FDF749FC0436AAE706F14D
:10AB1000040E30682B4600220A217646FDF73EFCE3
:10AB2000A0E7331D306829461E46FDF709FC99E76A
:10AB3000331D306829461E46FDF702FC92E7002BC4
:10AB40007FF443AF204608B0BDE8F0876E2BC6D037
:10AB50003BE700BF0EB400B584B005AB019053F8DD
:10AB6000042B0649039301A8FFF726FF019B00224F
:10AB70001A7004B05DF804EB03B070470D84000850
:10AB80000FB430B583B006AB0A490B4853F8042B19
:10AB9000096800680193FFF70FFF084C054620681D
:10ABA000FEF7E0FC0028FAD0284603B0BDE83040AC
:10ABB00004B070479C640020A0640020941F002013
:10ABC000DFED2B7AB4EEE70AF1EE10FA4ADDDFEDA5
:10ABD000296A9FED297A01E0B0EE670AB4EEC70A50
:10ABE000F1EE10FA70EE667AF6DC9FED247AF4EE60
:10ABF000C77AF1EE10FA38D5DFED1E6A9FED207AA4
:10AC000001E0F0EE407AF4EEC77AF1EE10FA37EE9A
:10AC1000A60AF6D4DFED1B7AB4EEE70AF1EE10FADD
:10AC200014DDDFED137A37EEC00A60EE006A9FEDA7
:10AC3000166A9FED167ADFED167AA6EE867A20EE7A
:10AC4000266AE6EE877AA6EE270A7047DFED117ACC
:10AC5000B4EEE70AF1EE10FA44BFDFED087A37EE02
:10AC6000C00AE2E7F0EE407ABFE7B0EE670AD1E74C
:10AC7000DB0F4940DB0FC940E4CB1641DB0F49C075
:10AC8000E4CB16C1DB0FC93F92E741B99730083CCE
:10AC900015A82ABEDB0FC9BF41404A0011F0800F42
:10ACA00082F0D503D2B2DBB208BF1346590013F0CD
:10ACB000800F81F0D502C9B2D2B208BF0A46510056
:10ACC00012F0800F81F0D503C9B2DBB208BF0B468A
:10ACD000590013F0800F81F0D502C9B2D2B208BF7B
:10ACE0000A46510012F0800F81F0D503C9B2DBB2E1
:10ACF00008BF0B46590013F0800F81F0D502C9B28E
:10AD0000D2B208BF0A46510012F0800F81F0D5037D
:10AD1000C9B2DBB208BF0B465A0082F0D50013F06F
:10AD2000800FD2B2C0B208BF1046704780EAE0730D
:10AD3000A3EBE0738B4205DB002801DD401A70476E
:10AD400002D17047002070470844704709B909E0F4
:10AD5000194690FBF1F301FB13030846002BF7D1D2
:10AD6000084670470146FBE7F0EEC07AB0EEE07AA5
:10AD7000B4EEE77AF1EE10FAB4BFB0EE676AB0EE67
:10AD8000476AB5EE406AF1EE10FA46D0B4EEE77AC3
:10AD9000F1EE10FA8CBFF0EE675AF0EE475AC5EEAE
:10ADA000866A9FED1F3A9FED1F6A9FED1F4A9FED38
:10ADB0001F5ADFED1F3ADFED1F4ADFED1F5AA6EEE7
:10ADC000C36AE6EEA34AA6EE864AB7EE006AA6EE8E
:10ADD000845AA6EEA46AE6EE855AC5EE866AB4EEFB
:10ADE000E77AF1EE10FA48BFDFED147AF5EEC00A0B
:10ADF00048BF77EEE66AF1EE10FA48BFDFED107A51
:10AE0000B5EEC00A48BF77EEE66AF1EE10FA48BF29
:10AE1000F1EE666AB0EE660A7047DFED076ADEE7BC
:10AE200039094E3DE3B59E3E88FA163E45FE7F3F0A
:10AE300099FB243F69A2163EA7DFA834DB0FC93F68
:10AE4000DB0F4940DFED317A30EE277AFDEEC76A3D
:10AE500016EE903A2033402B02D99FED2D0A704711
:10AE6000B4EEE70AF1EE10FA4DDD9FED2A6ADFED50
:10AE70002A6A01E0B0EE677AB4EEE67AF1EE10FAF3
:10AE800077EE467AF6DC9FED257AF4EEC77AF1EE9E
:10AE900010FA35D5DFED1F6A9FED217A01E0F0EE63
:10AEA000407AF4EEC77AF1EE10FA37EEA60AF6D43D
:10AEB000DFED167AB4EEE70AF1EE10FA1BDCDFEDF7
:10AEC000197AB4EEE70AF1EE10FA44BFDFED137A17
:10AED00037EEC00A60EE006A9FED136A9FED137AA9
:10AEE000DFED137AA6EE867A20EE266AE6EE877A02
:10AEF000A6EE270A7047DFED0F7A37EEC00AE9E7C2
:10AF0000B0EE670AD4E7F0EE477ABCE7DB0FC93F43
:10AF100000000000DB0FC940E4CB1641DB0F49C045
:10AF2000E4CB16C1DB0FC9BF92E741B99730083CAB
:10AF300015A82ABEDB0F4940FDEEC07A17EE903A05
:10AF40002033402B51D8DFED2D7AB4EEE70AF1EE35
:10AF500010FA50DDDFED2A6A9FED2A7A01E0B0EEAB
:10AF6000670AB4EEC70AF1EE10FA70EE667AF6DC04
:10AF70009FED257AF4EEC77AF1EE10FA38D5DFEDC1
:10AF8000206A9FED227A01E0F0EE407AF4EEC77A73
:10AF9000F1EE10FA37EEA60AF6D4DFED1D7AB4EE24
:10AFA000E70AF1EE10FA1BDCDFED1A7AB4EEE70ADD
:10AFB000F1EE10FA44BFDFED147A37EEC00A60EE0E
:10AFC000006A9FED156A9FED157ADFED157AA6EE02
:10AFD000867A20EE266AE6EE877AA6EE270A704782
:10AFE000DFED067A37EEC00AE9E79FED0E0A7047FB
:10AFF000B0EE670AD1E7F0EE407AB9E7DB0F4940DF
:10B00000DB0FC940E4CB1641DB0F49C0E4CB16C1CE
:10B01000DB0FC93FDB0FC9BF92E741B99730083C4E
:10B0200015A82ABE0000000010B507EE901A2DEDFD
:10B03000028BB8EE678ADFED227A28EE008A04469A
:10B0400028EE278AB0EE480A33F080F8F0EE408A06
:10B05000B0EE480A32F0DCFFF7EE007A9FED197A85
:10B06000F0EE675AE8EE875A0023A361B0EE676AF4
:10B07000C7EEA56A63612362E361A3626362A8EE1F
:10B08000C76ABDEC028B77EEC07AB6EE007AF8EEB6
:10B09000005A27EE877A20EE250A27EE267A26EE3A
:10B0A000266A67EEA67A20EE260A84ED046AC4EDCD
:10B0B000017A84ED007A84ED027A84ED030A10BDF2
:10B0C00027D4D236F304353F10B44C09012250F88E
:10B0D000243001F01F0102FA01F10B4340F8243043
:10B0E0005DF8044B704700BF4B0901F01F0150F899
:10B0F0002320012303FA01F1114214BF1846002056
:10B10000704700BFF0B4394B1B78012B66D0384B29
:10B110001B78012B5CD0374C37482368374A384EB0
:10B12000384D43F480630021236002270123442427
:10B130000772417271712C8213715371324D334C0D
:10B14000334E95E80F0005F1100784E80F0097E8EB
:10B150000F0004F1100787E80F0005F120030FCB63
:10B1600004F1200787E80F00402235202D21B2711D
:10B1700005F130033422122737723070F07071708D
:10B180003171B27072710FCB04F1300705F14006D6
:10B1900087E80F0096E80F0004F1400705F150061C
:10B1A00087E80F0096E80F0004F1500705F16006EC
:10B1B00087E80F0096E80F00703504F1600686E816
:10B1C0000F0095E80F00703484E80F00F0BC704762
:10B1D000094A052113721375D174AFE70D490E4A60
:10B1E0004FF4FA400880137091E700BFE47000202C
:10B1F0000C200020FC870020E8350020586D00203E
:10B2000030A80020408600207C04040868530020F9
:10B21000E88600200C310020C07D002010B53D20C4
:10B22000FEF7DEF90A4C606118B111220023827129
:10B23000C3712021FEF766FB30F0D8FB6069FEF792
:10B2400059FC044B002814BF012202221A7010BDC1
:10B250006C1E00200C200020074A084B10781B7839
:10B26000074A834296BFC31AC3F1800300201268C5
:10B2700018441044704700BF149700209096002097
:10B280008C960020064A074B10781B7883428ABFB1
:10B29000C3F18003C01AC018C0F17F00704700BF1F
:10B2A000149700209096002010B582B000249F23B0
:10B2B00032208DF804308DF805408DF806408DF869
:10B2C000074003F071FC8DF8014000BF334C20684B
:10B2D000FEF7D0FB01A90422684630F023FC206869
:10B2E000FEF7CEFB00BF9DF802309DF801009DF8EF
:10B2F00003102B4A1B0243EA00430B43934246D000
:10B300001ADD284A93423AD02FDD274A93422FD0A4
:10B310000132934222D1254B4FF480721A805A8019
:10B320009A881988224C120202FB01F101209A60CE
:10B33000D960207602B010BD1E4A934218D0013267
:10B340009342E8D0A2F51A42033A934206D1174B32
:10B3500020214FF4807219805A80E1E7134B0020BE
:10B36000188058809860D860E4E7023A9342F5D19B
:10B370000E4B80214FF4807219805A80D0E70B4B1E
:10B380004FF400714FF4807219805A80C8E7074B60
:10B3900040214FF4807219805A80C1E71465002063
:10B3A0001620C2001920C2001740EF00C00700207D
:10B3B0006C1E002017BA200030B5124C237E83B0DB
:10B3C0001BB90120237603B030BD052200238DF880
:10B3D00000208DF8013000BF0B4D2868FEF74AFBB6
:10B3E0006946022201A830F09DFB2868FEF748FB61
:10B3F00000BF9DF8053003F0010383F001002376C0
:10B4000003B030BD6C1E00201465002070B5064CE2
:10B410000646256803E023685B1BB34203D8FFF7A9
:10B42000CBFF0028F7D070BDC4B800202DE9F04F45
:10B4300089B0B2F1000801900391029340F39F801C
:10B440000B46002201EB880153F8040B8B420244A7
:10B45000FAD1029B0592002B00F08980059B002BFE
:10B460005ED04B4BDDF814B01B685FFA83FA0AEB31
:10B470000B02B2F5807F474AD2688CBFCAF5807A4A
:10B48000DA469A425ED9190C1A0A4FF002040620D5
:10B490008DF81F308DF81E208DF81D108DF81C4082
:10B4A000FFF7B4FF0620FEF7F1FA3B4A01231376BB
:10B4B00000BF3A4B1868FEF7DDFA07A90422002006
:10B4C00030F030FB0024039D019E5746A1462968B9
:10B4D000A30000200A46013459B1B94224D2316890
:10B4E00030F020FB2A68336813443360BF1AC5F874
:10B4F0000090A04505F1040506F10406E7D1274BAD
:10B500001868FEF7BDFA00BF214B214A1B6853445F
:10B510001360029AABEB0A0B0AB3BBF1000FA4D184
:10B52000059809B0BDE8F08F019C04933A46E158B4
:10B5300030F0F8FA049B2A68E1583944D71BE150EF
:10B540002F60DCE705981649164AA0EB0B00059022
:10B55000059800230B70137009B0BDE8F08F059BB0
:10B56000A3EB0B030593059809B0BDE8F08FFFF737
:10B5700023FF00287FF472AF029B0593D0E7029C63
:10B580001CB9FFF719FF0594CAE700230593C7E725
:10B590008C960020C00700206C1E0020146500203F
:10B5A000149700209096002070B5104D104E2B7807
:10B5B00031788B4284B016D00E4A03921A4402921C
:10B5C0008CBF0C46CA1A04A98CBFC3F180020024A8
:10B5D000012341F8102D02A802220194FFF726FF53
:10B5E000002333702B7004B070BD00BF9096002014
:10B5F000149700209496002070B5194C194D2378AB
:10B600002978994284B027D0174A03921A440292AB
:10B6100034BF0E46CA1A04A934BFC3F18002002603
:10B62000002341F8102D02A802220196FFF7FEFE2A
:10B6300023781844C0B203062B7848BF80F08000FE
:10B640008342207002D0002004B070BD002301208E
:10B650002B70237004B070BD012004B070BD00BF1A
:10B6600090960020149700209496002008B545F28B
:10B670000820FFF7CBFE0620FEF708FA064B012252
:10B68000C7201A76FEF702FA04480549054A002346
:10B6900003700B70136008BD6C1E0020149700200F
:10B6A000909600208C9600202DE9F04182B0034650
:10B6B000060C050A032406208DF807308846174635
:10B6C0008DF805608DF806508DF80440FFF79EFE5A
:10B6D00098B100BF0A4C2068FEF7CCF901A90422FA
:10B6E000002030F01FFA3A460021404630F01AFAA6
:10B6F0002068FEF7C5F900BF384602B0BDE8F0810A
:10B7000014650020F0B5124BDD6885B00DB905B0A9
:10B71000F0BDED0A14D0002704AE7C196410E002DD
:10B7200010226946FFF7C0FF0F2809DD6B4653F86A
:10B73000042B01320AD1B342F9D12546AF42ECDBEA
:10B74000FFF732FF034BED021D60E0E7671CF5E7F2
:10B75000C00700208C9600200C4B984213D0A3F514
:10B76000806398420FD003F5804398420BD003F5D5
:10B770008063984207D003F58063984203D0044B5E
:10B78000186840087047024B186870470004014071
:10B79000E0A60020F0B5774B774A87B01968914250
:10B7A00000AF00F0DB800023744A3B607B601368CD
:10B7B00043F48033136003E03B68B3F5A04F09D036
:10B7C000136803F400337B603B6801333B607B68A4
:10B7D000002BF1D0694B1B6813F4003318BF012311
:10B7E0007B607B68012B7BD0654D644B654AEA60CA
:10B7F0006549586F654A0860AA605E6B644C654A8B
:10B80000654826F080065E635E6F46F080765E6770
:10B81000196B0C431C63596B5963996B9963196CD1
:10B8200041F05B5141F47B1141F41F6141F00F0184
:10B830001964596C07F118040A4348F2FF715A64FD
:10B8400044F8101D002621460123FB733E737E73CE
:10B85000BE732BF0ADFE21464FF6FF734F48BB6021
:10B860002BF0A6FE4FF6FF7321464D48BB602BF030
:10B870009FFE21464B482BF09BFE21464A482BF069
:10B8800097FE214649482BF093FE214648482BF06D
:10B890008FFE214647482BF08BFE214646482BF071
:10B8A00087FE20462BF08EFF444B454C1B68BA6840
:10B8B00044484549A4FB03439B09A0FB0202013B0A
:10B8C000920CB3F1807F0A6007D2404AF020072132
:10B8D000536085F82300966011601C37BD46F0BDAB
:10B8E000264B3B4C1A6C3B4942F080521A6420684C
:10B8F000CA698D69096A40F4404020609868986080
:10B900009868120640F40040986042EA85129868F0
:10B9100042F48002490842F00802013942EA014239
:10B9200040F4A05098605A601A6842F080721A6021
:10B930001A689201FCD52849104A40F20570086047
:10B94000996821F003019960996841F002019960BA
:10B95000936803F00C03082BFAD145E700221A6024
:10B9600062B61E4B1B6883F308881D4B1B68984703
:10B97000FEE700BFFCFF0120EFBEADDE0038024055
:10B9800000ED00E00005FA05143600200000000874
:10B99000FF916700335F070000000240000402408F
:10B9A00000080240000C0240001002400014024057
:10B9B00000180240001C024000200240E0A60020C7
:10B9C000D34D621083DE1B43C8B8002010E000E0B6
:10B9D0000070004000000020003C02400000FF1FFB
:10B9E0000400FF1F08B5054B1B6803B19847044BC3
:10B9F000044A1A6072B6FDF761F800BF60A000202B
:10BA0000FCFF0120EFBEADDE08B5034B1B6803B1A0
:10BA1000984772B6FDF752F860A00020084B10B5A9
:10BA200007281B68C8BF143818440C46007EFDF771
:10BA3000D7FD20B12146BDE81040FEF739B810BD52
:10BA40004C7F002030B50446806D61718389A26807
:10BA500023F400531B041B0C838185B0A37900924F
:10BA600013F0040230D04FF4805213F00203ADF80B
:10BA7000042056D1ADF806304FF480630022ADF8B3
:10BA8000083011F00103ADF80C2028D1ADF80A30D0
:10BA900008238D07694648BFADF80A302BF0E0FE59
:10BAA000A279A36DD10724D412F0080F9A8A1BD172
:10BAB00022F008021204120C9A829A8992B242F47D
:10BAC00000529A8105B030BD13F00203ADF8042096
:10BAD00024D04FF400551346ADF80650CEE70423AA
:10BAE000ADF80A300C23D4E792B242F008029A82F1
:10BAF000E3E70D498B420FD0A1F54C418B4209D0B1
:10BB00000A498B42D0D103200121FFF787FFA27998
:10BB1000A36DC9E70120F7E70020F5E7ADF806308F
:10BB2000ACE74FF40053A5E700100140004C004083
:10BB300010B50446806DA160838923F400531B0473
:10BB40001B0C8381A37984B013F00402009135D0DB
:10BB50004FF4805213F00203ADF8042056D1ADF833
:10BB600006304FF480636279ADF80830D1074FF0AA
:10BB70000003ADF80A30ADF80C3045BF0423ADF832
:10BB80000A3008230C236946920748BFADF80A30F3
:10BB90002BF066FEA279A36DD1071FD412F0080F17
:10BBA0009A8A16D122F008021204120C9A829A89FB
:10BBB00092B242F400529A8104B010BD13F0020315
:10BBC000ADF804201FD04FF400511346ADF8061015
:10BBD000C9E792B242F008029A82E8E70D498B4227
:10BBE0000FD0A1F54C418B4209D00B498B42D5D1E6
:10BBF00003200121FFF712FFA279A36DCEE70120F8
:10BC0000F7E70020F5E7ADF80630ACE74FF4005356
:10BC1000A5E700BF00100140004C004038B50D4BB7
:10BC200007281B68CCBFA0F1140404462344054632
:10BC3000187EFDF7D5FC58B101342722C4718271FA
:10BC40000121FDF75FFE28460021BDE83840E5E60A
:10BC500038BD00BF4C7F0020064A00235168814256
:10BC600002F11C0204D00133102BF7D100207047E1
:10BC7000D8B270474000002070B50F4C0F4DC0EB9C
:10BC8000C00004EB8004286B26693043286382B02F
:10BC90009209667BA1600025012101A863618DF8EE
:10BCA00004608DF805208DF806508DF807102FF0F0
:10BCB0005DFE02B070BD00BF4000002000380240B1
:10BCC000074BC0EBC00030B403EB8000054C0569A6
:10BCD000236B2B4323630176427630BC704700BF51
:10BCE00040000020003802402DE9F04F534C54F83A
:10BCF000204083B0002C00F09C80E56D002D00F00A
:10BD00009A8017464E4A9846064604F1620328690F
:10BD1000226004F262226361A2614FF400736A68D8
:10BD2000A160E3602361A265A24668B1FFF794FFBA
:10BD3000721CD2B20C21FFF7C3FFA36DA9682A6958
:10BD400022630433A1636365E868A0B1FFF784FF51
:10BD5000721C8146D2B20B21FFF7B2FF2346EA7F65
:10BD600038494846FFF788FFA36DA968EA6862630F
:10BD70000433E163236594F86100FDF731FC8146EB
:10BD800094F86000FDF72CFC8346287F00284DD1F5
:10BD900018F0080F36D1BA070DD5B9F1000F0AD047
:10BDA0000B22731C89F8062089F8073048466A7F01
:10BDB0002221FDF7DBFCFB0715D4A36B7BB995F8BB
:10BDC0002020A97F8DF8063001A8930901228DF863
:10BDD00005308DF804108DF807202FF0C7FD504670
:10BDE00003B0BDE8F08FBBF1000FE6D001360C23A5
:10BDF0008BF807608BF8063058466A7F2221FDF7E2
:10BE0000B5FCDAE70136F6B2B9F1000F04D00B2326
:10BE100089F8076089F8063018F0100F484614BFFB
:10BE2000022112216A7FFDF7A1FCC6E72FF0C0FDB9
:10BE3000AEE7A246D3E7AA46D1E700BFA864002038
:10BE4000FC040408E18A00080348D0F8AC3113B1BF
:10BE500000F5D27018477047400000200348D0F822
:10BE6000903113B100F5C4701847704740000020AE
:10BE70000348D0F8743113B100F5B6701847704715
:10BE8000400000200348D0F8583113B100F5A870E5
:10BE900018477047400000200348D0F83C3113B1E8
:10BEA00000F59A7018477047400000200348D0F80A
:10BEB000203113B100F58C70184770474000002006
:10BEC0000348D0F804310BB1FC301847704700BF6D
:10BED000400000200348D0F8E8300BB1E0301847AC
:10BEE000704700BF400000200348D0F8CC300BB1B1
:10BEF000C4301847704700BF400000200348D0F806
:10BF0000B0300BB1A8301847704700BF4000002088
:10BF10000348D0F894300BB18C301847704700BFFD
:10BF2000400000200248836F0BB170301847704703
:10BF3000400000200248C36D0BB1543018477047D1
:10BF4000400000200248036C0BB13830184770479E
:10BF5000400000200248436A0BB11C30184770476C
:10BF6000400000200248836803B11847704700BFB3
:10BF700040000020431C00F013812DE9F04F4FEAF0
:10BF8000C00B0BEB00039B00DFF8848258F803A082
:10BF900087B008EB0304BAF1000F00F0FE80143301
:10BFA00008EB03010022DAF8047048F803204A6025
:10BFB0008A60CA60A568D4F80C90431CDBB215B146
:10BFC0001522EB71AA71B9F1000F04D0162289F87D
:10BFD000073089F8062001909AF80E002FF0E8FC4F
:10BFE000BB8823F440731B041B0CBB802846FDF761
:10BFF00047FD4846FDF744FD11212846FDF782FC28
:10C0000011214846FDF77EFC0826642403E03CB17C
:10C010002FF0ECFC013C2846FDF76CFD0028F6D023
:10C020002846FDF727FD2FF0E1FC2846FDF728FD07
:10C030002FF0DCFC013EEED14846FDF71BFD2FF052
:10C04000D5FC2846FDF716FD2FF0D0FC2846FDF75D
:10C0500017FD2FF0CBFC4846FDF712FD019B0BEBC3
:10C06000030408EB84042846637C002B0CBF1221D8
:10C0700032210422FDF77AFB637C002B0CBF1221D6
:10C08000322148460422FDF771FB584B9F4200F0D5
:10C090009880574B9F4200F09E80564B9F4200F085
:10C0A0008680BB880199544A544C23F440731B0486
:10C0B0001B0CBB803B888B4408EB8B089BB243F086
:10C0C000010398F810103B80BD8802A8002918BF12
:10C0D00014462BF077FB049A4948B2FBF4F325F0A1
:10C0E0003F05A0FB02122D04900C2D0C0543BD80D2
:10C0F000444C39884FF4967202FB00F284FB0240F4
:10C100009BB2D217002BC2EBA01221F0010108BF95
:10C1100001230904013243F40043090C92B239802F
:10C120003A84BB833B889BB243F001033B803B884E
:10C1300023F4816323F002031B041B0C4FF48042A1
:10C1400043F480633B803A813B8823F080031B04E7
:10C150001B0C3B809AF810308DF80830002402A8A0
:10C1600001258DF809408DF80A408DF80B502FF00D
:10C17000FDFB9DF80B209AF80F308DF808308DF8F4
:10C1800009408DF80A4062B95A09203203F01F03B2
:10C190001D4905FA03F341F8223007B0BDE8F08FDE
:10C1A000704702A82FF0E2FB07B0BDE8F08F174AF6
:10C1B000136A43F4000313624FF400002BF04CFAAF
:10C1C0006FE7124A136A43F4001313624FF400102E
:10C1D0002BF042FA65E70D4A136A43F480031362B9
:10C1E0004FF480002BF038FA5BE700BF00540040AA
:10C1F00000580040005C0040009F2400804F120067
:10C2000083DE1B43D34D621000E100E000380240A2
:10C21000CCB80020F0B5C60033189B00254DEA5875
:10C220005468A28A83B092B20192019A2B4412F40C
:10C23000706F1CBF01221A75019B13F4E06F074653
:10C240000CD1A38A3E4423F4706305EB86051B04DE
:10C250001B0C0022A3826A7503B0F0BD238BA38858
:10C2600023F480631B041B0CA380019B9B05E8D473
:10C2700023889805E5D42388D9050ED52388DA05C7
:10C28000FCD423889BB243F40073238023889B054E
:10C29000FCD43846FFF76EFED3E723889BB243F405
:10C2A00000732380A38823F440731B041B0CA3801A
:10C2B000C7E700BFCCB80020F0B583B0441C8DF8B0
:10C2C000073001D0032802DD002003B0F0BDC70015
:10C2D000244E3B1806EB83035D68002DF4D0490023
:10C2E000C9B2997501240021DA755C7699761C76BD
:10C2F0005C751975A9880DF107028905DA611A6262
:10C3000014D42B88DA050CD44FF4805401E0013C9E
:10C310001ED02B889B05FAD42B889BB243F48073E4
:10C320002B80AB889BB243F44073AB80074406EB91
:10C3300087024FF4805401E0013C09D0537D002B6B
:10C34000FAD106EB87073C7D84F0010003B0F0BD15
:10C35000054A138801339BB21380FFF70BFE20467A
:10C36000B3E700BFCCB8002038B900202DE9F04376
:10C37000322083B002F018FC0022104611231E2147
:10C38000FFF79AFF602301221E210020FFF794FF90
:10C39000642002F009FC6846FCF736FF0024DFF851
:10C3A0005481254626460A27012302221E21002009
:10C3B000FFF782FF322002F0F7FB6846FCF724FF0C
:10C3C000BDF900E0BDF90210BDF904208E457346A9
:10C3D000A8BF0B469342A8BF134643454FF0010048
:10C3E00076440D44144479DBFDF7EAF8013FDBD1D4
:10C3F0004FF001090022104612231E21FFF75CFFB7
:10C40000DFF8F0800A27012302221E210020FFF717
:10C4100053FF322002F0C8FB6846FCF7F5FEBDF979
:10C4200000E0BDF90210BDF904208E457346A8BF97
:10C430000B469342A8BF134643454FF00100A6EBBD
:10C440000E06A5EB0105A4EB02044ADBFDF7B8F8E4
:10C45000013FD8D107EE906AF8EEE76A07EE905AEE
:10C46000B8EEE77A07EE904ADFED1F5A9FED1F5AAC
:10C470001F4EF8EEE77A85EEA66A0022104670237A
:10C480001E21C5EE876A85EE277AB0EEC66AF0EE09
:10C49000E66AF0EEC77A86ED006AC6ED016AC6ED7F
:10C4A000027AFFF709FF202301221E210020FFF757
:10C4B00003FF0023184602221E21FFF7FDFE642021
:10C4C00002F072FBB9F1000F04D14FF07E533360DC
:10C4D0007360B360012003B0BDE8F0834FF0000942
:10C4E00088E74FF00009B5E700406F4601C05E469F
:10C4F0000000002001F0FFFF0123482277210020E7
:10C50000DAE600BF0123582277210020D4E600BFDD
:10C510003123F42276210020CEE600BF134600200E
:10C520000A466821C8E600BF0220FCF7C7BB00BF6F
:10C5300002206FE60120FCF7C1BB00BF012069E6C5
:10C540000020FCF7BBBB00BF002063E61549164B7B
:10C5500016488A6910B40C6A1549B2FBF4F203FB61
:10C5600002F30360D1F88820124B134C42F470029E
:10C57000C1F888201A68002042F001021A60986011
:10C580001A6822F0847222F480321A605C601A68A1
:10C590004FF0006422F480221A60D8608C605DF84D
:10C5A000044B70470000002040420F00E0A600202E
:10C5B00000ED00E00038024010300024044B4FF43E
:10C5C000F07002210A2298611962DA61FFF7BEBF9A
:10C5D0000000002003680A7A591C01601A70704735
:10C5E00038B50B4C23688BB15A68821A002A05466D
:10C5F00004DA0CE05A68AA1A002A07DB9A6822605B
:10C6000018461A6890472368002BF3D138BD38BD0F
:10C61000D02B00200B4B002210B4027203F5907453
:10C62000032102E0072A09DC9979890702D51979E3
:10C63000815401329C4203F11803F3D15DF8044B9D
:10C64000704700BF702D040818230370704700BFA7
:10C65000012310B431213024342244704171C2705E
:10C660000370037183705DF8044B704770B54E68BA
:10C670000546304630F00AFB31460446024628683B
:10C6800031F0A4FB2A68131901333B212B601155AB
:10C6900070BD00BF08B524F00FFFFFF7B5F900BF6C
:10C6A000024A034B1278197816F0A6BB1820002016
:10C6B0001920002038B5384B5A899989914224BFF6
:10C6C00000225A81198ADA89914224BF0022DA8134
:10C6D000DA788AB1072A0FD0304C3148A27801218C
:10C6E0000025062A01709970DD714CD92379DFEDA0
:10C6F0002D6A002B36D138BDDA799B78284807EEB1
:10C70000103A002A44D0DFED276A0178234CB8EEB6
:10C71000C77A07EE901AA278F8EEE77A27EE267A23
:10C72000062A67EE877A2BD81F4B03EB8203D3EDE3
:10C73000006AF4EEE76AF1EE10FA10DDC6EE877AD1
:10C74000FDEEE77A17EE903A102BA8BF1023012BCD
:10C75000B8BF0123DBB28B4228BF0B46037023799D
:10C76000002BC8D0013A032AC5D8B7EE000A80EEE4
:10C77000260A31F09FFC2388984238BF208038BDBC
:10C78000DFED086AD5E7DFED097AB0EE677ACBE72F
:10C79000DFED076AB9E700BF149800200C310020D4
:10C7A000C07D00206F120338240504086F12833AFD
:10C7B0006F120339038A2DE9F0478589ADB21D4018
:10C7C00029D00F4606464FF000484FF00009B5FA51
:10C7D00085F328FA03F2D24391B21B3B1540318214
:10C7E000042B16D8DFE803F03129211903007B6AF6
:10C7F000002B32D003F1FF3A1FFA8AFAC7F82490CF
:10C800003C6A34B123682046514698476468002C3E
:10C81000F8D1002DDBD1BDE8F0873868716B036873
:10C8200089B29847002DD2D1F5E77868B16B0368DB
:10C8300089B29847002DCAD1EDE7B868F16B03685B
:10C8400089B29847002DC2D1E5E7F868316C0368DA
:10C8500089B29847002DBAD1DDE7F36A1FFA83FA4F
:10C86000CEE700BFF0B54B4B4B491A68096883B05F
:10C870000123570200935CBF03F180530093D6005D
:10C880005CBF43F0100300938C0744BF43F0C60322
:10C890000093480744BF43F0080300930F0748BFC5
:10C8A00043F020033D4948BF0093160648BF43F4B8
:10C8B0004063097848BF0093D40548BF43F0006344
:10C8C00001F0EF0048BF009308286D4655D00E29AF
:10C8D00053D0D0033248009B00784CBF43F4204330
:10C8E00043F40053D7044CBF43F0644343F0444344
:10C8F00000280CBF07200F20960648BF43F4807322
:10C90000540748BF43F4003343F400245205009415
:10C9100002D5244A1279A2BB182936D001900027EB
:10C92000012639462846FCB2FEF7DEFB60B11E4BFD
:10C93000002203F5D87103E08B420FD013F80C2CC2
:10C94000944203F10C03F7D10137242FE9D195E884
:10C950000300164B83E8030003B0F0BD7A0904F02E
:10C960001F0455F8223006FA04F4013723EA0404C0
:10C97000242F45F82240D4D1E9E743F480530093B3
:10C98000A7E743F4C0130093C6E7009B43F060732E
:10C990000093C3E71836002064A00020FC7D00202F
:10C9A0003431002030A80020700604081020002038
:10C9B0002DE9F84F4E014FF0000B174D8146904680
:10C9C00006F120075C46594628465FFA8BFAFEF7C7
:10C9D0008BFBC0B1A64215D8A74213D900200F4A3D
:10C9E000014604E00131242914D012F80C0C504502
:10C9F00002F10C02F6D10A4B01EB410103EB81017C
:10CA00004846C04701340BF1010BBBF1240FDAD1CA
:10CA1000BDE8F88F0021F3E710200020700604081D
:10CA20006406040800210A4A0B4604E00133242B63
:10CA30000BD012F80C1C884202F10C02F6D105480A
:10CA400003EB430300EB830070470020704700BFF7
:10CA5000780604086406040800210A4A0B4604E02C
:10CA60000133242B0BD012F80C1C884202F10C026B
:10CA7000F6D1054803EB430300EB83007047002029
:10CA8000704700BF700604086406040808B5012159
:10CA90000220FDF715F8094B1B7803F00503052B61
:10CAA00008D000210120FDF70BF800210846FDF712
:10CAB00007F8FEE724F0B0FDF3E700BFA464002010
:10CAC000022828BF022010B4084C094B207000EB4C
:10CAD000C00200EB820207495DF8044B013003EB12
:10CAE0004203C0B20B6021F0D7BE00BFFC2700207C
:10CAF000E8860020C06D002008B518F045F9FDF764
:10CB0000EDFCBDE8084018F027B900BF38B50E4C61
:10CB10000E4DAC4206D2616820461434FDF762FC2B
:10CB2000AC42F8D3FEF7EEFA094C0A4B0A481860FB
:10CB30000025257024F042FB084B094A65701A60F5
:10CB4000BDE838401AF036BF90010008F005000833
:10CB5000FC270020C06D0020E8860020C46D002066
:10CB60001228002008B5FFF7D1FF18F00DF9FDF7E6
:10CB7000B5FCBDE8084018F0EFB800BFF0B50C29CF
:10CB800034D8DFE801F0893333335E333333343361
:10CB900033330700048C9689B2F802E01788734D8E
:10CBA00024F480542404240C0484038C8488818B12
:10CBB00023F4005321F4E6411B0409041B0C46EA4C
:10CBC0000E06090C43EA063341EA0721A8429BB24C
:10CBD000A4B289B200F09E8005F58065A84200F0FD
:10CBE000998092688480818302640384F0BD048C00
:10CBF0009589B2F802C0B2F800E05C4F24F480746A
:10CC00002404240C0484038C8688818B23F4007311
:10CC10001B0421F073011B0C45EA0C04090443EAD0
:10CC20000423090CB8429BB2B6B241EA0E015CD0B3
:10CC30004F4CA04259D0926886808183C26303849E
:10CC4000F0BD048C9589B2F802C0B2F800E0474EFE
:10CC500024F010042404240C0484038C8788018BA2
:10CC600023F0200321F4E6411B0409041B0C45EAD0
:10CC70000C04090C43EA041341EA0E21B0429BB2B2
:10CC8000BFB289B25DD03A4CA0425AD09268878038
:10CC9000018382630384F0BD048C9789B2F802E0BB
:10CCA0001688324D24F001042404240C0484038CDF
:10CCB0008488018B23F002031B0421F073011B0CF9
:10CCC00047EA0E0709043B43090CA8429BB2A4B2F1
:10CCD00041EA060125D005F58065A84221D0926879
:10CCE0008480018342630384F0BDD589148A578A06
:10CCF00023F4006343EA05254FF6FF332B40958864
:10CD000026F440563C4343EA052346EA04169BB208
:10CD1000B6B290E7158A24F4804444EA8514A4B29C
:10CD20005FE7D689158A578A23F00803334324F432
:10CD3000407496883D4323F004032C433343A4B24C
:10CD4000CDE7D489158A568A23F0800343EA041379
:10CD50004FF6BF741C40938827F44067354344EA7C
:10CD6000031347EA85079BB2BFB28FE7000001407B
:10CD7000000401402DE9F84FC82200219348944C4B
:10CD8000DFF87492934D944E944FDFF8708233F035
:10CD90009CFA93489349DFF868E2DFF868C2002202
:10CDA0001359834200F0F980B3F1804F00F0F7800F
:10CDB000AB4200F0F680B34200F0F580BB4200F0D9
:10CDC000F480734500F0F380634500F0F280434542
:10CDD00000F0F180DFF830A2534500F0EE800AF554
:10CDE000806A534500F0EB800AF5806A534500F0F5
:10CDF000E880AAF5983A534500F0E5800AF5806A84
:10CE0000534500F09C800AF5806A534508BF0D2306
:10CE100000F096801832B2F59C7FC1D1DFF8B08166
:10CE2000714E08F59C774FF0030A4FF0020998F80D
:10CE300004301C09013C032C03F00F0378D86B4A23
:10CE400032F8140040FA03F2D20771D5012505FA31
:10CE500003F3013B184030F013FC654B1B5D184495
:10CE600016EBC00264D056F83030624C98F80810C7
:10CE700003F13F4000F57E00800A205C00F01F04B3
:10CE80004009032805FA04F500F08180042878D0D1
:10CE9000022804D15348406C054352484564B2F817
:10CEA00004E0BEFA8EF2C2F11F0292B2D00803EB88
:10CEB000800002F00702046A92000F25954024EAE0
:10CEC00005040462046A01FA02F2224300250262A8
:10CED0004FF0010C2A4603E0102A05F1020527D085
:10CEE0000CFA02F030EA0E0102F10102F4D11C68E2
:10CEF0000AFA05F1C9430C401C60D3F800B009FAE6
:10CF000005F444EA0B041C609C680C409C609C681F
:10CF10009C605C6824EA0000586058685860D868D3
:10CF20000140D960D968D960102A05F10205D7D12E
:10CF300008F1180847457FF47AAFBDE8F88F0C2355
:10CF400009EBC3034FF0010A93F8203003F01F0BE5
:10CF50005B09032B0AFA0BFA09D0042B0CD0022B25
:10CF60007FF458AF4B6C4AEA03034B6452E70B6CF7
:10CF70004AEA03030B644DE70B6B4AEA03030B63B6
:10CF800048E71848006B05431648056387E71548CE
:10CF9000006C05431348056481E70023D0E70123B3
:10CFA000CEE70223CCE70323CAE70423C8E705231F
:10CFB000C6E70623C4E70723C2E70823C0E709231F
:10CFC000BEE70A23BCE70B23BAE700BF807F00203F
:10CFD000702D04080004004000080040000C0040D0
:10CFE00000000140003802406CB90020E43304081E
:10CFF000E0330408B03304082405040800040140A9
:10D000000010004000140040004001400149024867
:10D01000FFF7D0BB208000200004014001490248F6
:10D02000FFF7C8BB208000200004014001490248EE
:10D03000FFF7C0BBF87F0020000C00400149024808
:10D04000FFF7B8BBD07F002000080040014902482C
:10D05000FFF7B0BBA87F0020000400400149024850
:10D06000FFF7A8BB807F0020000001400149024873
:10D07000FFF7A0BB807F002000000140F0B50468EE
:10D08000474DA30AAB426ED009D8023DAB4266D0F1
:10D090000135AB4258D14FF0700E022608E0414DE9
:10D0A000AB4264D00135AB424FD14FF0C00E0426E5
:10D0B0004779B0004FEA970C00295CD063460227FD
:10D0C000A5899F4083190CEB43032F4303F1040C04
:10D0D000354DBFB245F8231045F82C20A781EFF35A
:10D0E0001181502282F31288821905EBC202136962
:10D0F00063B313620433821905EBC202576917B197
:10D100001F6053690433821905EBC202976917B196
:10D110001F6093690433821905EBC202D76917B106
:10D120001F60D36904330027CAB21F6082F31188DD
:10D13000304405EBC000036A5BB9A38923F0010307
:10D140001B041B0CA381F0BDF0BDF0BD05EB0E036D
:10D15000D1E7A3899BB243F00103A381F0BD4FF057
:10D16000480E0126A4E74FF0980E0326A0E74FF0E3
:10D17000200E00269CE70223BF0803FA07F7A389C5
:10D18000094D9BB223EA070387190CEB470CA381D7
:10D190000CF1040345F82C1045F823209FE700BF4D
:10D1A0000300100040001000807F002010B50368CD
:10D1B00083480139834282B089B200F0CB80A0F568
:10D1C0008060834200F0C68000F58040834200F01A
:10D1D000B88000F58060834200F0B38000F5806085
:10D1E000834200F0AE80774C188824686408B4FB52
:10D1F000F2F4013CA4B282B2B3F1804F0AD072487B
:10D20000834207D000F58060834203D000F5806040
:10D21000834202D122F0700292B26C48834200F045
:10D22000A28000F58060834200F0A78022F4407263
:10D2300000F56C4092B283421A80D9621C854FD0AF
:10D240005F4A93424CD001229A821A8892B242F0ED
:10D2500001021A80B3F1804F00F099805A4A93423C
:10D2600000F0978002F58062934200F0948002F50E
:10D270008062934200F0918002F58062934200F058
:10D280008E8002F58062934200F08B8002F570423E
:10D29000934200F0888002F57052934200F085803E
:10D2A00002F58062934200F0828002F58062934230
:10D2B0007FD0A2F5983293427DD002F580629342EE
:10D2C0007BD002F58062934208BF0D2215D002A8E0
:10D2D0004FF0012340F8043D2EF048FB02B010BD92
:10D2E0000122002119869A821A88394892B242F0A6
:10D2F000010283421A80ADD10A46364B03EBC203CA
:10D3000001A893F821408DF80440012300228DF8F4
:10D3100005308DF807308DF806202EF027FB1B2CEA
:10D3200008D02E2CDAD12C4B019301A82EF01EFB35
:10D3300002B010BD294B019301A82EF017FB02B0DB
:10D3400010BD204C18882468B4FBF2F4013CA4B250
:10D3500082B251E71B4C18882468B4FBF2F4013CFC
:10D36000A4B282B256E701201A80D9621C85988245
:10D370001A8892B202431A8070E701201A80D9629B
:10D380001C8598821A8892B202431A8062E70122B1
:10D39000B3E70222B1E70322AFE70422ADE705229B
:10D3A000ABE70622A9E70722A7E70822A5E709229B
:10D3B000A3E70A22A1E70B229FE70C229DE700BF0B
:10D3C00000040140E0A600200004004000100040DE
:10D3D00000000140240504082C010001190100018E
:10D3E0002C4B98423DD0B0F1804F3CD0A3F57C430C
:10D3F00098423AD003F58063984238D003F58063B1
:10D40000984236D003F58063984234D003F58063A8
:10D41000984232D003F57043984230D003F57053F0
:10D4200098422ED003F5806398422CD003F5806398
:10D4300098422AD0A3F59833984228D003F5806308
:10D44000984207D003F58063984208BF0D2202D0AE
:10D45000002070470C22104B03EBC20393F820000E
:10D4600070470022F7E70122F5E70222F3E70322E3
:10D47000F1E70422EFE70522EDE70622EBE70722BA
:10D48000E9E70822E7E70922E5E70A22E3E70B22BA
:10D49000E1E700BF00000140240504082DE98048B1
:10D4A000013085B0C3B203938A4D8B4F8B4C8C4EA9
:10D4B0000A230293DFF82C9226F088FA4FF4FA7AC6
:10D4C0004FF0100C4FF47A70D9F80430C3F308030E
:10D4D000002B40F0C180EFF31183002B40F0BC80A3
:10D4E0002968A26800BF2B689942F9D1D7F800E0FB
:10D4F00000FB0EF39B1AB3FBFEF300FB01314FF070
:10D50000010E0191D9F80430C3F30803002B40F059
:10D510008780EFF31183002B40F082802B68A16895
:10D5200000BF2A689342F9D1D7F800B000FB0BF294
:10D53000521AB2FBFBF200FB0323019A9B1AB3F5CC
:10D540007A7FDFD3BAF1010ABED1039B002B40F0F2
:10D55000BD804FF47A7ADFF88C9150464FF0100C72
:10D56000D9F80430C3F30803002B40F09280EFF3A6
:10D570001183002B40F08D802968A26800BF2B68C2
:10D580009942F9D1D7F800E000FB0EF39B1AB3FBE8
:10D59000FEF300FB01314FF0010E0191D9F8043088
:10D5A000C3F3080303BBEFF31183EBB92B68A16846
:10D5B00000BF2A689342F9D1D7F800B000FB0BF204
:10D5C000521AB2FBFBF200FB0323019A9B1AB3F53C
:10D5D0007A7FE3D3BAF1010AC2D1029B013B0293E5
:10D5E0007FF468AFFEF710FAEFF311888CF312881E
:10D5F000A1682368DB0344BFC6F800E0A1682B687C
:10D6000032685FFA88F888F31188D7F800801A44E6
:10D6100000FB08F35B1AB3FBF8F300FB0233D4E71B
:10D62000EFF311888CF31288A1682368DB0344BFF1
:10D63000C6F800E0A1682B6832685FFA88F888F3C2
:10D640001188D7F800801A4400FB08F35B1AB3FB7B
:10D65000F8F300FB023370E7EFF311828CF31288CA
:10D66000D4F808E02368D90303D501233360D4F844
:10D6700008E02B683168D2B282F311883A68194405
:10D6800000FB02F3A3EB0E03B3FBF2F300FB01314B
:10D6900035E7EFF311828CF31288D4F808E02368A1
:10D6A000D90303D501233360D4F808E02B6831682F
:10D6B000D2B282F311883A68194400FB02F3A3EB5B
:10D6C0000E03B3FBF2F300FB013164E718462EF0C2
:10D6D000F5FA3EE7C4B80020C8B8002010E000E02A
:10D6E000C0B8002000ED00E02DE9F047AD4FAE4E90
:10D6F00017F04AFBBE421ED2DFF83883DFF83893BA
:10D700004446258862197DB14A450DD2052D0BD9B5
:10D7100033886188C3F30B03994200F0D880144624
:10D7200025886219002DEFD1716830461436FCF758
:10D7300059FEBE42E4D39D4B5A78022A40F2EC8057
:10D7400000225A701A789A489A490160022A00F217
:10D75000DD8002EBC201984B02EB810203EB420237
:10D76000964C1046226023F029FD954A1378A3F1C8
:10D77000170102290FD9934911F83300002840F00E
:10D780000381D8000144497829B18F4911F8333019
:10D790000BB9182313708D4B9A78042A00F0EB8094
:10D7A00032B91A88B2F5F07F84BF4FF4F0721A8054
:10D7B000874D884A2B681A40002A00F0EE80DE0769
:10D7C00000F1B580580400F1B980190700F1BD805F
:10D7D0009A0100F1C1809B0400F1C68023689A8CF5
:10D7E000D98C914224BF00229A84FEF763FF1BF07C
:10D7F00045FE10B978481FF015FE2EF073FF00218A
:10D800003022764832F061FD754B256803F15001F6
:10D8100002E0043399427DD01A78002AF9D19C782D
:10D82000D8788442F5D26F496F4B0A7028461D6044
:10D8300015F01AFA6D4B6E4A1E786E496E486F4BA2
:10D840001160C825642212FB06526D4C006B31F842
:10D85000041C5A60002221809A60DA601A615A61C1
:10D860009A61DA6183F8202083F8212008B117F04B
:10D87000C7F9644B9FED645A1B88644A9FED646A44
:10D880005579644C64496548086006EE903AF8EEB4
:10D89000E66A1388C5EE265A07EE103A53881279C5
:10D8A000C4ED005A07EE903AB8EEC77A5C4BF8EE3A
:10D8B000E77A1D725A7227EE067A67EE867ABDE81D
:10D8C000F04783ED017AC3ED007A17F045BA63792A
:10D8D0009B077FF424AF716894F804A03046FCF7EE
:10D8E00081FD3388BAEB133F0BD173887068AA1F90
:10D8F000C3F30B039A4204F10601A8BF1A4630F0A5
:10D9000065FA1436BE42FFF4FBAE14E700221A702B
:10D91000294A25E7012286E72649254802EB4202EB
:10D9200001EB82011A780160022AEFD811E73D4825
:10D93000FCF78EFD2B6858047FF547AF3A48FCF79B
:10D9400087FD2B6819077FF543AF3848FCF780FD4A
:10D950002B689A017FF53FAF46F20900FCF778FD8E
:10D960002B689B047FF53AAF3148FCF771FD4020EE
:10D97000FCF76EFD32E71A8BB2F57A7FBFF418AF71
:10D980004FF47A721A8313E7D8000D186D68002DD2
:10D990007FF4F8AE17251570F4E643F008032B600A
:10D9A0000DE700BFF005000890010008FC270020EB
:10D9B000C46D002012280020E8860020C06D0020E1
:10D9C000FC7D0020C01104087C1D04080C310020DF
:10D9D000FC8700200960000240860020501F0020C4
:10D9E000007E002004020020841F00200C7A00200A
:10D9F000E41F0020D07D0020746D0020682D0020E1
:10DA0000302B0020F8220020C0C9FB48901E0020C7
:10DA100017B7D138FC220020407100203661023D4A
:10DA20001C71002008600002092000020160000251
:10DA30000940000207400008008000082DE9F0437B
:10DA40000B684A680B388BB00C46D51AEF2800F2E9
:10DA50007881DFE810F07C017601760176017601AD
:10DA600076017601760176017601760176017601FE
:10DA700076017601760176017601760176017601EE
:10DA8000760176017601A902760186027601770297
:10DA900076017601760170027601C4017601AC014F
:10DAA00076019B0176019401760112027601520102
:10DAB00076017601760176014D0176017F047601CB
:10DAC000760173047601760176017601760176019E
:10DAD0006F0476017601760151047601A004760187
:10DAE00076018B0476017601760176017601760166
:10DAF0007601F00076011B047601C80376019A03D3
:10DB00007601E603760176017601760176017601EB
:10DB1000760176017601760176017601760176014D
:10DB2000760176017601760176017601760176013D
:10DB3000760176017601760176017601760176012D
:10DB4000760176017601760176017601760176011D
:10DB5000760176017601760176017601760176010D
:10DB600076017601760176017601760176017601FD
:10DB700076017601760176017601760176017601ED
:10DB800076017601760176017601760176017601DD
:10DB900076017601760176017601760176017601CD
:10DBA00076017601760176017601760176017601BD
:10DBB00076017601760176017601760176017601AD
:10DBC000760176017601760176017601760176019D
:10DBD0006E0347032E037601F102E6026605760125
:10DBE0005A052B0519051205E8047601D5047601BE
:10DBF0007601C604CB05C205AF057305F605E10540
:10DC000006067601760176017601760176017601C7
:10DC10007601760176017601760176017601DB02E6
:10DC2000760176014502760176017601760176016C
:10DC3000760176013A020846FCF760FE054615F0CB
:10DC4000BFF8FF2854D0B5F57A7F80F03A850AAF47
:10DC5000002307F8243DEE0839460DF103008DF846
:10DC60000330013615F08CF89DF80330F6B205F05C
:10DC70000705B34205F1010503D19DF80430AB421D
:10DC800003D02946304615F087F894E80C009B1A1B
:10DC9000012B2DDD531C0AA823600023157800F802
:10DCA000253D15F061F89DF80330AB420AD0B24B28
:10DCB0001B683BB19A79AA4204D31B681B690BB15C
:10DCC0002846984723685A1C2260384600221C7850
:10DCD0008DF8042015F03CF89DF80430A34207D0DD
:10DCE000A54B1B6823B11B685B690BB120469847A5
:10DCF000012318460BB0BDE8F083A049A1FB052124
:10DD00006A1A01EB52018908C1EBC102B5EB0208A6
:10DD100017D1C9B24E1EF6B20029E9D0DFF86092E1
:10DD200001365A1C226093F90010954B002593F997
:10DD300002208A4203F1080300F09E840135062D7B
:10DD4000F5D14FF0FF3318460BB0BDE8F0838D4995
:10DD5000102D4FF0000328BF10250B604B608B6027
:10DD6000CB600B74002DC3D023685A190133236094
:10DD700013F8010C01F8010B9A42F7D1B8E75A1CCD
:10DD80000A60814A1B7853750123B2E75A1C0A6066
:10DD90001E781F2ED5D8052DD3D10846FCF796FD49
:10DDA0007A4B43F8260019F005FE0123A1E7774DD1
:10DDB00005F140062046FCF7A1FD2368A5F8800088
:10DDC000591C1A46216012F8021B85F88210226045
:10DDD0005B7885F883300435AE42EBD188E75A1C76
:10DDE0000A60694E1B7833720846FCF787FDB083E2
:10DDF0002046FCF783FD30832046FCF77FFD236837
:10DE000070835A1C22601B78F374082D7FF670AF64
:10DE10002046FCF773FDF0842046FCF76FFD0C2DC7
:10DE200030857FF665AF23681A46591C216012F8C9
:10DE3000021BB17722605B7886F820302046FCF721
:10DE40005DFD102DB0847FF653AF23685A1C22600D
:10DE50001B78F3722046FCF739FD2368F0605A1CEA
:10DE600022601A783274162D7FF642AF9A1C226017
:10DE70005B7886F8213001233BE75A1C0A601A7848
:10DE80000E2A3FF65EAF991C2160587803283FF6B2
:10DE900058AF3F4D02EB42025200A918DE1C4871F8
:10DEA00026609878A8541A1D2260DA784A705A1DA4
:10DEB00022601A798A709A1D22605A79CA70DA1D16
:10DEC00022609B790B71012313E7324B1B78DB0730
:10DED0003FF537AFFEF710FEFFF706FC012308E71A
:10DEE0005A1C0A601A780F2A3FF62BAF991C216042
:10DEF000C2EBC202284958788854D81C20600A44D2
:10DF000099785170191D2160D9789170591D21603F
:10DF10001979D170991D216059791171D91D21602C
:10DF20009979517103F108012160DB79937122F035
:10DF3000D9FD0123DDE65A1C0A60184A1B781370CC
:10DF40000123D6E60846FCF7D9FC154D286020468B
:10DF5000FCF7D4FC68602046FCF7D0FC0123A860E5
:10DF6000C7E6104D00232B600846FCF7AFFC2B687A
:10DF7000184328600123BCE6682800202549922424
:10DF80004086002001280020E8350020EC6E0020AB
:10DF9000A826002071970020B8720020FC7D002088
:10DFA000D8640020FC8700205A1C0A601E78132EBB
:10DFB0003FF6C7AE9A1C0A6000205D78A24902466F
:10DFC00005E00132242A3FF4BCAE11F80C0C854266
:10DFD00001F10C01F5D19D489D4902EB420210F878
:10DFE000222001F82620D81C206001EB86029978B7
:10DFF0005170191D2160D8789070581D2060954986
:10E000001B790868D37013F0B9FD71E60846FCF778
:10E0100075FC914DA8812046FCF770FC01236881B6
:10E0200067E68E4B1B78D9073FF562AE8C4B4FF4F9
:10E03000C8721A8001235CE6092D7FF682AE894FF3
:10E040001A46591C3E68216012F8021B317022608A
:10E050005A78B270DA1C22609A78642A03F10401BB
:10E06000A8BF642272712160DA78642A03F1050185
:10E07000A8BF6422B27121601A79F2719A1D2260E0
:10E080005A79642A28BF6422D91D327221609A7994
:10E09000F27003F108022260DB7933712046FCF74D
:10E0A0002DFC0A2D708140F079832EF01BFB01239B
:10E0B0001FE6684A1068DA1C01462133951E256068
:10E0C00012F8035C0D70551E256012F8025C4D704D
:10E0D000226012F8015C8D7003329A4201F1030153
:10E0E000ECD17CE05A1C0A601A785F49002A00F0E3
:10E0F000E4820A7842F00202981C0A705B4D2060AC
:10E100005B782B702046FCF7E1FB68602046FCF74B
:10E11000DDFBA8602046FCF7F1FBA8812046FCF758
:10E12000EDFB534A6882137843F002031370012316
:10E13000DFE5C5F34705122D3FF603AEBDB10AABCF
:10E140000DF1020703EB45083E46A8F126082046DC
:10E15000FCF7D4FB26F8020FB045F8D1454B37F851
:10E16000022F23F8022FBE42F9D1112D09D8424ABD
:10E170006B00023B13440021223223F8021F93421A
:10E18000FBD13E4A01231370B3E50846FCF7B6FB0A
:10E190002046FCF7B3FB2046FCF7B0FB23682D4F6D
:10E1A0009A1C3E6822605A7886F82F20DA1C22607A
:10E1B0009A7886F83A201A1D2260DA7886F83B2091
:10E1C000073323602046FCF799FBF08720463E6822
:10E1D000FCF794FB112DB08700F28A82386822F098
:10E1E00015FD012385E55A1C0A601A4FDFF8988057
:10E1F0001B783E6888F805300846FCF77FFB3084C2
:10E2000020463E68FCF77AFB052D708400F27E8282
:10E21000FEF750FA2AF050FC386822F00BFE01237A
:10E2200067E51A46591C21600B4912F8020BC870A9
:10E23000226013495A780A70DA1C2260114A9B78CE
:10E24000D370012355E500BF78060408640604086E
:10E25000007E0020C06D0020CC7D00207197002042
:10E260005ABC0020C46D00203D6D0020406D002090
:10E27000E42D0020526500205465002050650020E8
:10E28000DC7D0020E47D0020149800201A46591CF3
:10E290002160B34E12F8021BB1702260B1495A7866
:10E2A0000A70DA1C2260B04D9A782A711A1D226019
:10E2B000DB78092BA8BF09232046AB70FCF71EFBB7
:10E2C000236862682880D11A012905DD2046FCF701
:10E2D00015FB626823686882934240F04D82FEF726
:10E2E000E9F9236862689A423FF402AD5A1C226041
:10E2F0001B78EB700123FCE41A46591C21609B4DEE
:10E3000012F8021B297022605B786B702046FCF7C4
:10E31000F5FA236868805A1C22601B782B7120460E
:10E32000FCF7ECFA2368E8805A1C22601B782B72F9
:10E330000123DEE4FDF79AF90123DAE48C4A03F1C4
:10E3400008000133236013F8011C02F8011F9842F2
:10E35000F7D1CDE4591C1A462160864912F8020B08
:10E36000887022605B784B700123C2E4824A127885
:10E37000012A3FF6BDAC19465A1C22607F4A11F8AB
:10E38000020B9070216059781170D91C21609B7824
:10E3900053700123ADE45A1C0A601E78112E3FF61B
:10E3A000D0AC9A1C0A60764D5B7805F816300846AA
:10E3B000FCF7A4FA40F6CA039842A8BF184640F2F8
:10E3C000EE239842B8BF18466E4BA0F2EE2083FBB6
:10E3D000002305EB4605C017C0EBE3036B70012378
:10E3E00087E40846FCF78AFA674D28802046FCF748
:10E3F00085FA68802046FCF781FA0123A88078E43A
:10E40000624F3B78002B3FF473AC614E00252046F1
:10E41000FCF774FA23F01AF83B78A6EC010A0135F0
:10E42000AB42F4DC64E40F2D7FF48BAC5A1C0A6021
:10E430001D78072D3FF685AC0846564F05EB450580
:10E44000FCF75CFAAD007E19B0802046FCF756FA66
:10E45000F0802046FCF752FA236830811A46591C96
:10E46000216012F8021BB17222605B78F3722046C1
:10E47000FCF72CFA012378513BE40846FCF73EFAFE
:10E48000454A0123108034E45A1C0A6018780506B6
:10E4900000F17A81414B1B78DC073FF529AC03285A
:10E4A00028BF0020FEF70CFB012322E45A1C0A605F
:10E4B00008461D78FCF70AFA80462046FCF706FA63
:10E4C00007462046FCF702FA06462046FCF716FAF5
:10E4D0002046FCF713FA236801332360002D00F077
:10E4E0003781102D7FF404AC2D4BC3F800805F60A2
:10E4F0000EB12C4B1E602C492C4B0222081F1A70A7
:10E5000014F050FB0123FFF7F4BB244B1B78D80712
:10E510003FF5EEABFEF726FBFFF7E6F80123FFF72A
:10E52000E8BB1E4B1B78DA073FF5E2AB204A1378B5
:10E5300043F0040313700123FFF7DBBB1A46591C99
:10E54000216012F8020B2260DA1C597822609A7856
:10E5500021F0DAFC00287FF4CBABFFF7F2BB00BF61
:10E5600014980020C07D00200C3100200C7A00207F
:10E57000E7350020F07D0020008800200188002081
:10E580001C2D00201F85EB51F479002045A70020A9
:10E59000FC7800208C7A0020FC2E0020719700204F
:10E5A000881F0020EC2200208C1F0020E62D002078
:10E5B0003D6D00201A46591C21607F4912F8020B5C
:10E5C000087022607D495A788A70DA1C22607C4A81
:10E5D0009B7893700123FFF78CBB7A4B7A491868BC
:10E5E0004A222FF0F3FB0123FFF783BB19465A1C85
:10E5F0002260764A11F8020B107021605978517030
:10E60000D91C21609B7893702046FCF777F9704AFB
:10E610000123D080FFF76DBB19465A1C22606D4A5A
:10E6200011F8020B1070216059785170D91C2160CB
:10E6300099789170191D2160DB78D3700123FFF761
:10E6400058BB0846FCF75AF9634DA8822046FCF7F0
:10E6500055F9E8822046FCF751F901232883FFF79A
:10E6600048BB0846FCF74AF9554B00EB80004000D8
:10E6700018800123FFF73DBB09EBC5072046B970A1
:10E68000FCF73CF9216829F835000B464A1C22604A
:10E6900013F8022BFA7023604B783B71CB1C23607C
:10E6A0008B78BB710B1D236008F10108CA787A7161
:10E6B00046457FF436ABFFF71BBB0A7802F0FD023C
:10E6C0001AE501AF384614F037FBBDF80430AB4211
:10E6D0003FF4DBAA414B1B68002B3FF4D6AA1B6812
:10E6E0009B69002B3FF4D1AA28469847FFF7CDBA83
:10E6F00023683868591C1A46216012F8021B80F8FA
:10E70000311022605B7880F8323068E52046FCF7F3
:10E71000F5F8A8F80A002046FCF7F0F8A8F80C0075
:10E7200020463E68FCF7EAF8B08420463E68FCF7D5
:10E73000E5F80D2DF0847FF66BAD2046FCF7DEF892
:10E74000A8F80E002046FCF7D9F8A8F810005FE5FD
:10E75000234B1020C3F800805F6020F0B5F8214AF9
:10E76000137843F001031370002E3FF4C1AA1E4A30
:10E7700001231660FFF7BDBA5A1C22601B780033D4
:10E7800018BF0123F371AAE500F07F00032828BF1A
:10E7900000200BF03FF90123FFF7ABBA23683A687A
:10E7A000591C2160197851720B2D3FF47EAC991CD5
:10E7B00021605B78537078E414980020CC7D0020B1
:10E7C000E47D0020C06D0020A01A0408C47D002054
:10E7D000F4790020142F00200C310020682800203C
:10E7E000282E00203D6D0020EC22002008B516F0F8
:10E7F000CBFAFBF773FE16F0AFFAFEF775FF0120B8
:10E80000BDE8084020F048B82DE9F04F013085B050
:10E81000C3B203930B4602918B4C8C4E002B00F03D
:10E8200099808B4D8B4FDFF8309225F0CFF84FF465
:10E83000FA7A4FF0100C4FF47A70D9F80430C3F321
:10E840000803002B40F0DE80EFF31183002B40F033
:10E85000D9802968A26800BF2B689942F9D1D7F8FE
:10E8600000E000FB0EF39B1AB3FBFEF300FB01314B
:10E870004FF0010E0191D9F80430C3F30803002BC7
:10E8800040F08780EFF31183002B40F082802B68EB
:10E89000A16800BF2A689342F9D1D7F800B000FB05
:10E8A0000BF2521AB2FBFBF200FB0323019A9B1AF4
:10E8B000B3F57A7FDFD3BAF1010ABED1039B002BF7
:10E8C00040F0BD804FF47A7ADFF88C9150464FF0DB
:10E8D000100CD9F80430C3F30803002B75D1EFF303
:10E8E0001183002B71D12968A26800BF2B6899425F
:10E8F000F9D1D7F800E000FB0EF39B1AB3FBFEF34F
:10E9000000FB01314FF0010E0191D9F80430C3F33F
:10E91000080313BBEFF31183FBB92B68A16800BF99
:10E920002A689342F9D1D7F800B000FB0BF2521AD3
:10E93000B2FBFBF200FB0323019A9B1AB3F57A7F2B
:10E94000E3D3BAF1010AC4D1029B013B0293002B2D
:10E950007FF467AF05B0BDE8F08FEFF311888CF35B
:10E960001288A1682368DB0344BFC6F800E0A168F1
:10E970002B6832685FFA88F888F31188D7F800802E
:10E980001A4400FB08F35B1AB3FBF8F300FB0233F5
:10E99000D2E7EFF311888CF31288A1682368DB03B8
:10E9A00044BFC6F800E0A1682B6832685FFA88F8B7
:10E9B00088F31188D7F800801A4400FB08F35B1A2B
:10E9C000B3FBF8F300FB023370E7EFF311828CF333
:10E9D0001288D4F808E02368D90303D501233360F3
:10E9E000D4F808E02B683168D2B282F311883A6813
:10E9F000194400FB02F3A3EB0E03B3FBF2F300FB9D
:10EA000001317FE7EFF311828CF31288D4F808E02C
:10EA10002368D90303D501233360D4F808E02B68B9
:10EA20003168D2B282F311883A68194400FB02F3CC
:10EA3000A3EB0E03B3FBF2F300FB013118E718461A
:10EA40002DF03CF93EE700BF10E000E0C0B8002028
:10EA5000C4B80020C8B8002000ED00E0204B5B687F
:10EA6000C3F3080330B4BBB9EFF31183A3B91D4B53
:10EA70001D4C1868A16800BF1A689042F9D11B4B61
:10EA80001C684FF47A7202FB04F3591AB1FBF4F1DB
:10EA900030BC02FB00107047EFF31182102383F3A8
:10EAA000128811498C680B6813F4803F104B02D018
:10EAB000012018608C680B49D2B20D68186882F387
:10EAC00011880A4B19684FF47A72284402FB01F34B
:10EAD0001B1B30BCB3FBF1F302FB0030704700BFDF
:10EAE00000ED00E0C4B8002010E000E0C8B800204D
:10EAF000C0B800202DE9F84F8046FFF7AFFF254E44
:10EB00002549DFF8A0E0254A254D844610274FF41B
:10EB10007A740120DEF80430C3F30803D3B9EFF3AD
:10EB20001183BBB90B68D2F808A000BFD1F80090E0
:10EB30004B45F7D1D6F800B004FB0BF9A9EB0A0955
:10EB4000B9FBFBF904FB0393A3EB0C034345E1D3AF
:10EB5000BDE8F88FEFF3118A87F31288D2F808B076
:10EB60001368DB0344BF2860D2F808B00B68D5F8FF
:10EB700000905FFA8AFA8AF31188D6F800A09944C7
:10EB800004FB0AF3A3EB0B03B3FBFAF304FB093317
:10EB9000DAE700BFC8B80020C4B8002010E000E0E9
:10EBA000C0B8002000ED00E02DE9F04FDFF830C1E3
:10EBB000474A4849484E494D8046102718F1FF38CA
:10EBC000C0F08480DCF80430C3F30803002B5CD170
:10EBD000EFF31183002B58D10B68946800BF0868CD
:10EBE0008342F9D1D6F800904FF47A7000FB09FE09
:10EBF000AEEB040EBEFBF9FE00FB03EEDCF80430C6
:10EC0000C3F308034FF47A740120FBB9EFF31183C7
:10EC1000E3B90B68D2F808A000BFD1F800904B45CB
:10EC2000F7D1D6F800B004FB0BF9A9EB0A09B9FB40
:10EC3000FBF904FB0393A3EB0E03B3F57A7FBDD27C
:10EC4000DCF80430C3F30803002BDFD0EFF3118AA4
:10EC500087F31288D2F808B01368DB0344BF28603A
:10EC6000D2F808B00B68D5F800905FFA8AFA8AF3F8
:10EC70001188D6F800A0994404FB0AF3A3EB0B0318
:10EC8000B3FBFAF304FB0933D5E7EFF3118487F301
:10EC90001288D2F808901368D80303D501232B609B
:10ECA000D2F808900B682868E4B284F31188D6F88B
:10ECB00000A04FF47A7400EB030E04FB0AF3A3EBFD
:10ECC0000903B3FBFAF304FB0E3E97E7BDE8F08FB0
:10ECD00010E000E0C4B80020C8B80020C0B8002090
:10ECE00000ED00E030B4EFF31183102282F31288BC
:10ECF0000649074C0A680748013200250A6025606A
:10ED0000DBB2026883F3118830BC7047C4B80020BE
:10ED1000C0B8002010E000E00F4B1B88014643B94B
:10ED20000E4B0F4A1B7810680BB981F00101FAF7FE
:10ED3000BFBE0C4B5A691AB118B91A6810605874E2
:10ED40007047094A18681188084A92FBF1F20121BC
:10ED500002605974704700BF04BB002006BB00204E
:10ED600008BB00200CBB002024BB002020A1070012
:10ED700038B5254BDC68236B73B1A36D626BCAB1E8
:10ED8000998A1A88C90592B201D5D20700D438BD34
:10ED90004FF6F7721A8038BDA36D99891A888906D3
:10EDA00092B2EBD59206E9D5E26ACAB1988880B2F0
:10EDB0009047E2E799891A880D0692B2E0D51006CD
:10EDC000DED5A26A616A8A4219D0A1692569885C88
:10EDD00098800132B2FBF5F105FB1122A262CFE768
:10EDE0009B88E2696169DBB28B54E269E068A36DDC
:10EDF0000132B2FBF0F100FB1122E261BEE7DA68FA
:10EE000022F08002DA60BBE7A864002038B5254B09
:10EE10005C68236B73B1A36D626BCAB1998A1A885F
:10EE2000C90592B201D5D20700D438BD4FF6F772AA
:10EE30001A8038BDA36D99891A88890692B2EBD5DC
:10EE40009206E9D5E26ACAB1988880B29047E2E7B3
:10EE500099891A880D0692B2E0D51006DED5A26A0D
:10EE6000616A8A4219D0A1692569885C988001325B
:10EE7000B2FBF5F105FB1122A262CFE79B88E269A4
:10EE80006169DBB28B54E269E068A36D0132B2FBC9
:10EE9000F0F100FB1122E261BEE7DA6822F08002A5
:10EEA000DA60BBE7A86400202DE9F04F9A4A9B493D
:10EEB000137895B00446099000F59C4020300C90E2
:10EEC0000860002B00F03284954909688C4240F2BA
:10EED00096809449059109689348944DDFF888B26B
:10EEE0000391013B137001F4805302900893002BAF
:10EEF00040F09480029B5B7D002B40F06083039B7D
:10EF0000180400F16386039BD9050BD5099A884B39
:10EF1000DFF858A29A429AF8022001F21D80002AD6
:10EF200041F01E80834B0493834C039B13F4805762
:10EF300040F0A483029BBBF906605B8B9E42B4BF8A
:10EF4000002601267D4B1B6813F0805373D0049A72
:10EF5000127812F0010275D002987949808C91EDF7
:10EF6000037A07EE900AF8EEE77AB4EEE77AF1EE6C
:10EF700010FA80F20487002E69D195F8A4100029B8
:10EF800065D170487049006890F830004FF0000E6D
:10EF9000C1F800E0C1F804E0C1F808E06B490028BE
:10EFA00056D10870002A57D0039AD00654D5684A23
:10EFB0001278D10650D4002F4ED1002B4CD1039B98
:10EFC0005A0249D494F800C0BCF1000F01F05286F7
:10EFD000604B9B78002E41F076863BB15E4A5F4BDA
:10EFE00012681B689B1A002BC1F29B8610201FF031
:10EFF0003FFB012385F8A53094F800C02EE0494B73
:10F0000005931B680393484A484D029203F48053CA
:10F01000DFF854B10893002B3FF46CAF0021474850
:10F02000FCF762F800287FF465AF0AF011F8059B41
:10F030001B6803935EE7039A520288D4049A1278FD
:10F0400002F00102002185F8A410002E99D03F495A
:10F0500001200870002AA7D194F800C0029ABBF9D9
:10F0600000E0508B918BBBF902208645CCBF8027F6
:10F07000002747F040038E45A8BF3B469B0843F05E
:10F0800080078242C8BF3B4643F040078A42B4BF74
:10F090003A461A469208BBF904E0BBF9067042F002
:10F0A00080038645C8BF1A4642F040038E45A8BF7C
:10F0B00013469B0843F080028742D4BF184610468F
:10F0C00040F0400295F8A6308F42ACBF0146114691
:10F0D0008B4200F08F84002385F8A61085F8A730B6
:10F0E000BCF1000F00F0F885059B1D4A1B680392D8
:10F0F00003F00403002B40F02C840DF14808194C58
:10F100000023C8F8043004F15009129340F6330A82
:10F11000192740F283362EE0802C00202C2B002073
:10F120007C2C002018360020E8350020A01E00208E
:10F13000404B4C007197002004020020107C0020FE
:10F1400040A80020C06D0020747B0020F424002023
:10F150003D6D0020F07D0020C4B800207423002005
:10F1600064A00020007E0020CC540020682D0020E8
:10F1700004344C4520D0A278E3789A4217FB026110
:10F18000F6D26278043217FB03633BF91220524532
:10F19000A8BF5246B2F5617FB8BF4FF461728A4290
:10F1A000E6DD9A42E4DC21782329E1D840460434A4
:10F1B000FBF78AFF4C45DED1AD4B98E803001E7883
:10F1C000AC4B83E80300002E00F053830121A948D3
:10F1D000FBF78AFF002840F00D81059B1B68D905CD
:10F1E00000F10381A44C23881EB226F001061FFA09
:10F1F00086F84345A4F8008000F070849F4E0227F3
:10F200000F204FF0140A4FF0FF09377086F801A065
:10F2100086F802901FF02CFA39469648B4F8008020
:10F22000FBF762FF002840F0DE8728F002039BB264
:10F23000434523800BD0914B1421FF2202260F203F
:10F240001E7059709A701FF013FAB4F800808C4B3E
:10F25000DFF848A21978DAF80400029318F0030FD7
:10F2600008BF81F00201C1F34001FAF721FC039BC2
:10F270001B6813F00A0F1DD005217E48FBF734FFF1
:10F28000002800F014852688730740F151877948DB
:10F290000621FBF729FF002800F0F684770640F1ED
:10F2A000648707217348FBF71FFF002840F0A78100
:10F2B000039B1B68980600F1B28126886D480C21DB
:10F2C000FBF712FF002800F0B48046F48073B342CD
:10F2D000238009D0694B02251421FF220F201D70C5
:10F2E00059709A701FF0C4F9664B1B78082B00F018
:10F2F000AC800E2B00F0A980059B1B685E0542D5F3
:10F30000614B1B79002B58D014215A48FBF7ECFEB7
:10F31000002856D120F0C8FA01201FF0FBF890B366
:10F32000DFF87C8100254FF0CC0902E0DDB2022D30
:10F3300029D809FB05F76B1C58F80760002EF5D19A
:10F34000C378524A90F9020052F823300196032202
:10F350000092012132461EF0B7F8034605EB450046
:10F3600000EB0010059353B1314608EB8000CC222E
:10F3700030F0ABFF059B48F807300135EDB225F0C2
:10F3800059FC0028D3D1049B1B78DD0740F18A800B
:10F390003F49404A01230B701370029BDAF80000CA
:10F3A000197801F00101FAF783FB039B1B685A07E8
:10F3B00000F1E88015B0BDE8F08F049B1B78D807FA
:10F3C000A8D53C201AF0EAFE0028DCD01CF0F8FC9E
:10F3D0003C201AF085FE0028D5D01CF0F1FC3C2022
:10F3E0001AF07EFE0028F1D1CDE72B4BDB78002B05
:10F3F0003FF4F8AE039B1B689A077FF5F3AE1E4CF3
:10F40000B4F8008018F0010F7FF40FAF48F001034B
:10F41000984523803FF409AF184B1421FF220226A0
:10F420000F201E7059709A701FF022F9B4F80080F6
:10F43000FBE626F480739BB2B34223807FF44AAF8D
:10F44000104B1B78082B7FF454AF228822F0400326
:10F450009BB29A4223803FF44FAF084B0225142100
:10F46000FF220F201D7059709A701FF001F943E7B9
:10F47000F6270020107C0020BC6D00209027002083
:10F48000F4BA0020FC7D002030A80020441A0408B3
:10F490007297002000230020682D0020F8BA002079
:10F4A000B4500020814B93F80090B9F1000F5FD168
:10F4B000DFF874827E4F18F8030C3E784146A8F1BD
:10F4C000030512F02BFB002800F02883002E40F0EB
:10F4D0007A8305F10801687912F020FB002841F0D9
:10F4E00052827449A87A12F019FB002800F029838F
:10F4F000022E41F04C827049E87B12F00FFB00288D
:10F5000041F031826D49287D12F008FB002800F09F
:10F510002983042E41F02B826949687E12F0FEFA9D
:10F52000002841F028826749A87F12F0F7FA0028E6
:10F5300000F02983062E41F02282634995F82300CA
:10F5400012F0ECFA002840F06D87604995F8280029
:10F5500012F0E4FA002800F02983082E40F07887A2
:10F560005B4995F82D0012F0D9FA002840F0298364
:10F57000584B01221A702DF099FA039B1B685A0709
:10F580007FF518AF032012F0F3FA002800F0408650
:10F59000238813F008047FF40DAF08201FF0ACF9A6
:10F5A0004D484E4D4E494F4A4F4BBBF806600068E0
:10F5B0002E80086014601C6015B0BDE8F08F029AC0
:10F5C000013BD27D3BF91330002A40F09E83A3F526
:10F5D0007A73B3F57A7FA8BF4FF47A7323EAE373A3
:10F5E00007EE903A9FED417AF8EEE77A67EE877A78
:10F5F0003F4AFCEEE77A17EE903A138083E43D4BE6
:10F600003D4AB3F904303D4982FB0302DB17C3EBEB
:10F61000A202039B0A801B6898067FF54EAE384B0A
:10F620001B78990704D5374F3B78042B00F28B8663
:10F63000268816F0300F3FF441AE10201FF044F939
:10F6400020201FF041F9304B268800221A702F49E4
:10F650002F48304F304D00220A6030493A60002375
:10F660002A6042608261036083604361C3610B6012
:10F670004A608B604B618A61CB611FE61D2128487F
:10F68000FBF732FD00287FF455AC264A029BD28856
:10F690001B8BBBF90660991A8E4240F33F861344D8
:10F6A0009E42B4BF002601264CE400BF72970020A2
:10F6B00034000020792600207E26002083260020AA
:10F6C000882600208D2600209226002097260020E4
:10F6D0009C26002000230020646D0020E0220020F2
:10F6E000EC220020E4220020DC220020AAF1823F4C
:10F6F000622D00206C6D002067666666D4220020B3
:10F700003D6D0020406D0020E62D0020DC2E002005
:10F710008C2E0020C82400205C230020B42E002062
:10F72000107C0020F47900206F2600209A4D9B4B1E
:10F730002E7802939A4F002E00F0F082B6B1DFF8D7
:10F74000A092DFF8A0B2DFF85882CA460024072C46
:10F750004046E1B27B6841F35082984700B20134E1
:10F76000A6422BF8020F0AF1040AF0D18D4B059343
:10F770001A4609998C4B12680392A3FB013E42F290
:10F78000010313404FEA9E1E079300F0C38287488F
:10F79000874A884B00788849069012781A70069B31
:10F7A00008702BB1834B93F800B08BF001030693E4
:10F7B000824A0299127838781090B1F82680088D24
:10F7C00091F822C00B92098B0B9A119195F8291090
:10F7D0007B4B0E9008461146A3FB01135B0803EB1D
:10F7E0004303D31ADBB20D93039B2C78754EDFF8DD
:10F7F000F8B1DFF8F891CDF810800F220CF1040C6D
:10F8000003F4805385F828200A955FFA8CFC109D3C
:10F810000F92A24608930021804610972CB9AC4560
:10F8200099BFE2466446AA462C46A14280F225834F
:10F83000069B002B00F0D682634B049833F911200D
:10F8400097B287424FEA410303D30E98874240F2B2
:10F850000F8359F82120964580F0CE823BF9032092
:10F86000079F002F40F0E2822BF80320013106367B
:10F87000D4E7DFF87C91554F09F15A044FF00108A5
:10F88000494619F8010C12F049F9F8B199F8040049
:10F8900099F8023099F803E000EB400105EB810193
:10F8A000013BD1F8B42003EB43033B4493420DD01A
:10F8B00095F8E02081F8B0E008FA00F022EA0000B4
:10F8C000C1F8B430C1F8B86085F8E00009F1060964
:10F8D0004C45D5D13E493F4A374B0968D2F8009094
:10F8E00093F800A03C4C0691002663685BB31F7838
:10F8F0004FB3A268A9EB0202002A0ADB95F8E020C8
:10F900000121B14022EA010209F5FA7185F8E020EF
:10F91000A160BAF1000F16D0227859780432D2B221
:10F92000002940F0318202993BF91220098B01F144
:10F93000C800824240F3C68495F8E0209B783241AB
:10F94000D20740F146850136042E04F10C04CCD1D7
:10F950003CE495F8AB3053B1049B1B78D90706D52E
:10F96000029BBBF906205B8B9A4200F32485112190
:10F970001A48FBF7B9FB002800F0E88195F8AE3093
:10F980002BB995F8A93013B93223A5F8AC3001236F
:10F9900085F8AE30FFF7B1BBA01E0020E83500208F
:10F9A0005C28002018360020D34D6210082B002060
:10F9B0000802002009020020592D0020812C00207F
:10F9C000ABAAAAAACC1E0020A41E0020B0050408E1
:10F9D000C46D0020C4B80020501F0020107C0020FF
:10F9E000E82C0020A21E0020CC540020842C0020F3
:10F9F000A926002095F8A790B9F1F90F00F2B88177
:10FA000009F101095FFA89F985F8A79085F8A61030
:10FA1000BCF1000F00F06181B9F1140F7FF464AB09
:10FA20005F2940F06D81049E337813F0010300F0EC
:10FA3000558709F00DFB337803F00103002B7FF4A9
:10FA400053AB95F8A620572A00F0B886059B1B6893
:10FA500013F0040302D05A2A00F0FE845D2A00F05D
:10FA60001E875B2A00F036875E2A00F0B884562A8B
:10FA700000F0B78723782BB16F2A00F0A287CB4B19
:10FA800000211960972A00F0A087A72A00F0868439
:10FA90000021BB2A129101F06180B72A01F03E805B
:10FAA000BE2A01F05E80BD2A01F06480792A01F04F
:10FAB0009D807A2A01F093809E2A01F089809D2AF8
:10FAC00001F07E80AE2A01F06780AD2A7FF40CAB96
:10FAD000FF21002027F026FFFFF706BB0221B448D4
:10FAE000FBF702FB00283FF4A0AB268018F0020FC2
:10FAF0007FF4ADAB48F00203434523803FF4A7AB4E
:10FB0000AC4B022214211A700F20FF2259709A70F8
:10FB10001EF0AEFDB4F80080FFF799BB08F10501B7
:10FB2000687911F0FBFF00283FF4DBAC012E40F0B8
:10FB30002A8705F10D01A87A11F0F0FF002840F0A6
:10FB400026879D49E87B11F0E9FF00283FF4DAACF5
:10FB5000032E40F008879949287D11F0DFFF002827
:10FB600040F005879649687E11F0D8FF00283FF4E1
:10FB7000DAAC052E40F0FF869249A87F11F0CEFF47
:10FB8000002840F0FC86904995F8230011F0C6FF4C
:10FB900000283FF4DAAC072E40F044848B4995F8F6
:10FBA000280011F0BBFF002840F05284884995F8E6
:10FBB0002D0011F0B3FF00283FF4DAAC092E3FF41A
:10FBC000D7AC4FF009094B4600F02FBCD5F88C306C
:10FBD000099AD31A002BFFF696A97E4A95F8903021
:10FBE000517C7D4A029C32F811200C98A17DC5F809
:10FBF0008C00013303F00F0385F890302B4492B250
:10FC000092FBF1F283F8942095F8940095F8951002
:10FC100095F8962095F8973001440A4495F8980095
:10FC200095F899101344184495F89A2095F89B304C
:10FC300001440A4495F89C0095F89D10134418441B
:10FC400095F89E2095F89F3001440A4495F8A0004D
:10FC500095F8A1101344184495F8A23095F8A32004
:10FC600001440B441A4442F30B12642AE17DA8BFFD
:10FC7000642213B209B1C2F1640307EE903A9FED1A
:10FC8000577AF8EEE77AB1E426F040039BB2B3422C
:10FC900023803FF406AB474B02261421FF220F209E
:10FCA0001E7059709A701EF0E3FCFFF7FABA2388B1
:10FCB00023F00406B6B2B34226803FF4E8AA3D4BD7
:10FCC00002261421FF220F201E7059709A701EF018
:10FCD000CFFC2688FFF7DBBAE14600213448FBF76A
:10FCE00003FA30B3002385F8A83008F04FFC95F8EC
:10FCF000A730142B7FF4F8A92378002B40F0DF877E
:10FD0000049B1B7803F0010398E6C3F53B630833BB
:10FD10001BB25CE4324B1B78069342E593F8223029
:10FD20003E780433DBB2B3428EBF2E702B701E467A
:10FD300004E5049B1D4A1B781060DB0700F1218558
:10FD4000B9F1140F3FF47DAEFFF7CEB995F8A930A5
:10FD5000002B3FF4D2A9049B1B7813F001037FF41E
:10FD6000CCA9012285F8A93085F8AA20FFF7C5B9EA
:10FD700085F8A630BCF1000FAFD0FFF7B5B901216F
:10FD800085F8A410FFF763B9012900F0368595F8CE
:10FD9000E0200123B34001361343042E85F8E03000
:10FDA00004F10C047FF4A1ADFFF710BA7823002012
:10FDB000107C0020902700207E2600208326002033
:10FDC000882600208D2600209226002097260020DD
:10FDD0009C260020287F0020447F002014AE234171
:10FDE000592D0020049B002B40D059F82120964526
:10FDF0004FEA4103FFF432ADB84AB848D25CC718A5
:10FE0000002A00F0BA81022A40F065817A7802EB7C
:10FE1000820202EB820202F2EE2292B2032940F346
:10FE20009280079F12B2002F3FF41EAD0D985F180D
:10FE300007440A9800EB4707BA85B8F1000F03D1D1
:10FE40000B9802287FF610ADB6F802803288B7888A
:10FE500042441744A24A3FB282FB0702A148A2EBE8
:10FE6000E772C75212B24FF00108FDE41A464B0088
:10FE70000EF5967749F82170F2E40F990A9D9A4B96
:10FE8000109F85F800A00F2942460CBF01220022D6
:10FE900085F8298085F828101A7006D11B2193480F
:10FEA000FBF722F9002800F0E5849148914B826825
:10FEB0001968914BC1608A1A0121197043688F4EED
:10FEC0009A42029A317088BF002392F8226088BF5C
:10FED00080F82130089B3878B2F826C0B2F818E0D4
:10FEE0000436F6B2002B00F0558186427B4A40F280
:10FEF000C781834E174600210CB982460446A142B1
:10FF000018DA12F8113083B1022B0CD17B7803EB95
:10FF1000830303EB830303F2EE239BB226F8023B39
:10FF200001310237E8E73388F8E7CBB2032BFAD880
:10FF30007346F3E785F800A00B9B724A01331370F8
:10FF4000089BFEF7D4BF012000FA01F70F9820EAC2
:10FF5000070012B20F9083E412B901228AF802203E
:10FF6000694B04931C789AF8218004F001031B204C
:10FF7000039311F0FDFDB8F1010F079000F0D1815E
:10FF800004F0020306939AF82020604CDFF8849175
:10FF90005F4E584F052A00F29580DFE802F0857920
:10FFA000032F3E51B8F1010F04BF05238AF820301A
:10FFB000039B002B00F0BA80029B3868B3F918103D
:10FFC000B9F80230002261F30F0263F31F420023ED
:10FFD00061F30F0361F31F43DAF81410CBF8042028
:10FFE0008142CBF8003080F01E810323069347F254
:10FFF00030520323CAF81C208AF82030338843F09B
:020000040801F1
:100000000203338009F024F83A68DAF81C3013440C
:100010000422CAF818308AF82020B8F1010F40F005
:1000200037843B68DAF818209A424BD2207818B906
:1000300011F09EFD002845D1338823F00203338060
:100040003A68B9F80630642101FB03234FF480605D
:1000500000228AF820208AF80320CAF810301EF007
:1000600033FC9AF8202095E711F0AEFD012800F04E
:100070007084079B002B40F05781B8F1010F21D00D
:100080003B68DAF810209A4246D301238AF82030E0
:10009000B8F1010FD4D099F80830012B3CD021F0F1
:1000A0003FFF9AF8202075E7039B002BDCD1079BCC
:1000B0004FF48060002B00F0A8801EF01DFC002291
:1000C000CAF81020069B002B40F0A980059B1B68F6
:1000D0000393FEF72BBF3BF803209FE61C2D002067
:1000E00056555555141F00205A280020107C00201A
:1000F000682D0020C4B8002008020020090200205A
:10010000CC540020812C0020719700200402002094
:10011000BA6D00200C7A002021F002FF032240F685
:10012000B8338AF82020CAF81C3067E73B685EE7DE
:1001300046F004039E4223800AD0AE4B02261421CF
:10014000FF220F201E7059709A701EF091FA2688B7
:10015000A94BAA4AB3F90430A94982FB0302DB1771
:10016000C3EBA2030B80FFF792B846F04003B34203
:1001700023807FF490ADFFF794B8CAB2022A40F210
:10018000FD82032AA7D1119A0898049F002808BF6E
:100190003A4643E6864219469A4A4CD89A48174648
:1001A0000CB9B24634468C427FF7C4AE12F8113017
:1001B00083B1022B0CD17B7803EB830303EB830326
:1001C00003F2EE239BB220F8023B01310237E7E74E
:1001D0000388F8E7CBB2022B03D9032BF8D163468F
:1001E000F1E77346EFE728F001039BB24345238014
:1001F0003FF47CAC0F20377086F801A086F802909F
:100200001EF036FAB4F8008070E41EF05DFB56E78D
:1002100008201EF059FBFFF7CDB80323069306987C
:100220001EF026FA52E7B8F1010FF6D103239AF82F
:1002300020200693AEE6744E17460CB9824604465B
:10024000A142BFF677AE12F8113083B1022B0CD168
:100250007B7803EB830303EB830303F2EE239BB270
:1002600026F8023B01310237E7E73388F8E7CBB2E3
:10027000022B03D9032BF8D16346F1E77346EFE76E
:100280006148174600210CB9B24634468C427FF7CC
:1002900051AE12F8113083B1022B0CD17B7803EBF5
:1002A000830303EB830303F2EE239BB220F8023BAC
:1002B00001310237E7E70388F8E7CBB2032BFAD81E
:1002C0007346F3E7C8398A425BDA95F8E0209B78F9
:1002D0003241D0073FF537ABC3F1000801201EF0D3
:1002E000DBFA7A1E162A00F25F81DFE812F0F101D4
:1002F0000502DA013F0123023402B2019F018A01A3
:10030000750160015D013F014F013402B2019F019F
:100310002B0117010301C501ED00D9000126FEF7ED
:1003200011BE002306932EE699F80430002B3FF40B
:10033000A4AE21F0F5FD03224FF47A738AF8202051
:10034000CAF81C305AE60A2011F012FC26888046B2
:10035000002800F0A882F20640F1CF8395F8F080E3
:10036000B8F1000F7EF4AAAF0E201EF081F9012330
:1003700085F8F0302688B8F1000F7FF468A9FEF701
:100380009DBF95F8E0300122B24023EA020309F54F
:10039000FA7285F8E030A260FFF7D5BA1B49059BD9
:1003A0000A781B6842F004020A7003F00403184A3A
:1003B0000392FEF79FBE00211648FAF795FE00282B
:1003C0007FF4D5AA322385F8AB00A5F8AC30FFF74F
:1003D000CEBA9846002B0CBF012002207FE70E4BBF
:1003E000022203200D4C0E4922700B601EF054FABD
:1003F000FEF77ABE902700206C6D00206766666667
:10040000FC2E00201C2D0020CC5400203D6D00202F
:1004100064A00020107C00207C870020FC270020A6
:10042000C06D00204FF007094B4603EB83031D44CA
:1004300087F80090A978687812F0AEFC049BB84A5F
:100440001B7801211170D9077FF595A8FEF7A5BF8C
:100450004FF008094B46E8E795F8A920002A40F03C
:10046000918395F8AB2082F0010285F8AB20002A39
:1004700040F08383AB49096811F4003104D0AA49E4
:100480000979002940F047840A46A848845C0D2C6D
:1004900002F10C0200F0D58301311529F6D186E76F
:1004A000D5F8E400A24B90F83A109A7841446429B8
:1004B000A8BF642121EAE17180F83A10002A40F0D7
:1004C000198420F0A3FB62E4D5F8E400984B90F87F
:1004D0003B109A784144FE29A8BFFE2121EAE17130
:1004E00080F83B10002AECD016202CF0E1F8D5F86B
:1004F000E400E6E7D5F8E40081788D4B4144C82953
:10050000A8BFC82121EAE17181709B78002BD8D067
:1005100014202CF0CDF8D5F8E400D2E7D5F8E400AB
:100520004178834B4144C829A8BFC82121EAE17121
:1005300041709B78002BC4D013202CF0B9F8D5F86B
:10054000E400BEE7D5F8E4000178794B4144C829BE
:10055000A8BFC82121EAE17101709B78002BB0D0BF
:1005600012202CF0A5F8D5F8E400AAE70698704B05
:1005700081799A7841446429A8BF642121EAE17114
:100580008171002A40F097830D2F0DD00698684B9B
:1005900041799A7841446429A8BF642121EAE17134
:1005A0004171002A40F0B083D5F8E40089E7D5F81E
:1005B000E4005F4B017A9A784144C829A8BFC8215A
:1005C00021EAE1710172002A3FF47BAF0B202CF08D
:1005D0006FF8D5F8E40074E7D5F8E400544BC1791E
:1005E0009A784144C829A8BFC82121EAE171C171A4
:1005F000002A3FF466AF0A202CF05AF8D5F8E40040
:100600005FE7D5F8E4004A4B81799A784144C829DC
:10061000A8BFC82121EAE1718171002A3FF451AFDE
:1006200009202CF045F8D5F8E4004AE7D5F8E400B5
:100630003F4B41799A784144C829A8BFC82121EA93
:10064000E1714171002A40F03083112F7FF454AFE3
:1006500037E7D5F8E400364B01799A784144C82948
:10066000A8BFC82121EAE1710171002A40F0468348
:10067000102F7FF455AF24E7069A2D4B5178414453
:10068000B1F5967FA8BF4FF4967121EAE1715170E0
:100690009B78002B88D015202CF00AF8D5F8E400C0
:1006A0000FE7069A17794744642FA8BF642727EA03
:1006B000E77717712CF016F81D4B9B78002B3FF451
:1006C00073AF032039462BF0F3FFD5F8E400F8E6CA
:1006D000069A174B11784144FA29A8BFFA2121EA5A
:1006E000E17111709B78002B3FF45EAF01202BF07D
:1006F000DFFFD5F8E400E4E6069A0D4B917841441B
:100700006429A8BF642121EAE17191709B78002BD4
:100710003FF44AAF02202BF0CBFFD5F8E400D0E63F
:100720000023002044250020586D0020D00C040830
:10073000018800200698B24BC1799A78414481F330
:100740000801C171002A3FF42FAF05202BF0B0FF44
:10075000D5F8E400B5E6D5F8E400A94BC1789A785D
:100760004144C829A8BFC82121EAE171C170002A0B
:1007700040F095820F2F7FF4E7AEA2E6119AFFF7C3
:100780004DBBA04B1B78002B3EF4AEAC9E4BDB78F0
:10079000002B7EF4A9AC95F8A8300133DBB2032B13
:1007A00085F8A8307EF6A0AC984B5B7813B9002E84
:1007B0007EF49AAC08F04CFCFFF799BA944B95493B
:1007C0001A684FF47A73B3FBF2F3C3EB431203EBF3
:1007D0008203059A1268DB001606A1F8A83000F122
:1007E000E3808D4B03931B68580700F1D480059B71
:1007F0001B6803F00403FEF77DBC3BF912209978D7
:10080000B2F5617F4FF4966393FBF1F3C0F29880E9
:1008100040F633019142A8BF11460C2FA1F561713A
:1008200091FBF3F800F07781182F7FF4B0AA5FFAFC
:1008300088F1C8290B46A8BFC823D5F8E400C27DBB
:10084000DFB297423FF4A3AA9B1A6D4AC77548BF0F
:100850000733DB1092785F1CFFB23AB9002F3FF4E8
:1008600096AA38461EF018F8FFF791BA18202BF018
:100870001FFFF3E76449694BCA681B688B609B1ACA
:10088000C82B7FF659AB012381F82130FFF754BB09
:100890003968DAF81C200A44CAF8182012E4604BC0
:1008A000002201209EE5F30600F108810B2011F0E3
:1008B0005FF9002840F0CC80B70600F1548195F82C
:1008C000F030002B3FF450ADB8F1000F7EF4BFAE16
:1008D000FEF7F4BC534B0122022083E5524A126812
:1008E000970304D5514A1279002A40F05D8150489F
:1008F00019461A46465C0B2E01F10C0107D0013255
:10090000152AF7D1002285F8A720FFF797B8494E9E
:10091000D6F800E05100BEF1000F07D08F1800EBB1
:1009200087079EF801E07F787745EBD20A44424F73
:10093000424900EB82020020326038800860E1E723
:100940000C2F00F0C580182F7FF421AA00210B4640
:1009500073E73A68B9F80630642101FB0323CAF84B
:100960001030FFF786BB4FF003094B465DE54FF0B3
:1009700004094B4659E54FF005094B4655E54FF044
:1009800006094B4651E54FF001094B464DE54FF046
:1009900002094B4649E5059B294A1B680A2111803B
:1009A00003F00403FEF7A6BB264B1B789C077FF5DC
:1009B00018AF254B1B78042B7FF613AF12F07CF891
:1009C0000FE707F0E3FDFEF78FBB059B1F4A1B688F
:1009D0004FF4C8711180104A039203F00403FEF72C
:1009E00089BB14F0D1F9F9F779FD14F0B5F9FCF7EA
:1009F0007BFE01201DF050FF95F8A620FFF73AB8C6
:100A000001880020592D0020682D0020F07D002055
:100A10004CA000202898002064A00020C4B800202A
:100A2000E88600203287002044250020586D0020F1
:100A3000D00C0408A02400203A2500203C250020EA
:100A400058BC00203D6D0020406D00205ABC0020A5
:100A5000B94ABA4B528993ED007A07EE902AF8EE24
:100A6000E77AB0EEC77AB4EEE77AF1EE10FA7FF5E6
:100A700023AF93ED017AB0EEC77AF4EEC77AF1EEC8
:100A800010FA7FF719AFB3063FF519AF20201DF01C
:100A900033FFAB497A68BB68C5F8E820081FC5F882
:100AA000EC3012F07FF8A74B01221A7095F8F03065
:100AB000002B00F0F0802688FEF7C9BD10201DF045
:100AC00003FFA04B268883F800804FF00108EDE675
:100AD0000027B8469C4B5B78BB423FF458A9384688
:100AE00008F098FF994B9B7823B15FFA88F10C20AE
:100AF0002BF0DEFD0137FFB2B0E610201DF0FCFE4A
:100B000020201DF0E1FE9249081F12F04BF88D4B9A
:100B100002221A70CAE75FFA88F7DBE70B464FF646
:100B2000FE718C4A8C485489039090892344014477
:100B30005381918114F028F9F9F7D0FC14F00CF9E5
:100B4000FCF7D2FD01201DF0A7FE059B1B680022CB
:100B500003F0040385F8A720FEF7CCBA0B46022168
:100B6000DFE70223DDE720201DF0AEFE754B0022FB
:100B70001A709BE74FF6FE73D3E70C201DF078FD4B
:100B8000FEF7B2BA0122002185F8AA20724A85F840
:100B9000A9100392FEF7AEBA0121002026F0C2FE92
:100BA00095F8A620FEF791BF6C4A1278002A7FF4D0
:100BB0009EAE1DF041FD049B1B7803F00103A1E6EE
:100BC0000021FF2026F0AEFE95F8A620FEF77ABFA2
:100BD000012026F0A7FE95F8A620FEF770BF604A18
:100BE000137A43F001031372FEF77EBA5C4A137A5C
:100BF00023F001031372FEF777BA029A115D98474A
:100C0000032C1BDC40F2EE2240F6CA0C00283EF416
:100C1000A6AD39F824E0BAF802104FF47A73A0EBCD
:100C20000E0003FB00F0A1EB0E0190FBF1F0184465
:100C30009042B8BF10466045A8BF604600B2FEF7BC
:100C40008EBD484E37684A003FB1541800EB84040B
:100C50007F786478BC42BFF4AAAB0A4400EB8202FE
:100C6000414F424C326000213B4A3980216003925F
:100C7000FEF740BA002E3EF4B9A995F8A5C0BCF124
:100C8000000F3EF4EBA91DF0D7FC94F800C085F8E6
:100C9000A570FEF7E3B94FF00108FFF765BB0F2021
:100CA0002BF006FDD5F8E40064E511202BF000FDE3
:100CB000D5F8E400C9E40D202BF0FAFC64E495F8C3
:100CC000A610FEF7ADBE3BB129492A4A09684FF488
:100CD0007A7000FB0313136095F8A530002B3EF4E7
:100CE000BDA91DF0A9FC002385F8A53094F800C02B
:100CF000FEF7B4B917202BF0DBFC55E410202BF0E5
:100D0000D7FCD5F8E400B3E40E202BF0D1FCD5F8E5
:100D1000E400FFF7D6BB1149097849B11146FFF746
:100D2000B4BB08F095F9002385F8A530FEF794B917
:100D30001DF082FCFEF7D8B9802E002040A80020CC
:100D40008C1F0020E62D0020FC27002001880020B9
:100D50002C2E0020CC7D002064A000203EA8002086
:100D6000042F0020A02400203A2500203C2500204C
:100D7000C4B8002074230020F8B55D4B1B78DB0756
:100D80002DD55C4B5C4D1C785C4E012C49D079D341
:100D9000022C1BD06B7A7BB1EB886BB1584B1B7864
:100DA00053B119F0CBFF00287CD0AB7A83422CBF23
:100DB00001230023337000E0337852492A7A9C42A1
:100DC00038BF1C460C70002A53D1F8BD4E494F4A1B
:100DD000098812889142DDD901241C70DAE74A4B58
:100DE0004B48454D1988EC78B0F8F230A142A1EBA0
:100DF000030303F1020223D32B788B4220D33D4B14
:100E00001C78032C51D03D4E424A1278022A04D15C
:100E10003B4F414A3F78D7809480012CA0F8F210D4
:100E2000B5D13A4A38491288E87A0988121A9142AB
:100E300035DD3A4A12888A42ACD200241C70A9E7F8
:100E4000B1EB440FDBDC2B4B1C78032CDBD0042AEA
:100E5000D9D82A4EDFF8A8C0DFF8C0E02B4F002217
:100E6000032434701C708CF80020AEF800203A8007
:100E7000CAE7012C36D0022C10D10720BDE8F8407B
:100E80001DF0F6BB254A20491288E87A0988121A13
:100E900091423FF77FAF01241C707BE7F8BD02242D
:100EA0001C7077E70223337087E7042AABD82A78CF
:100EB00091FBF2F20132082ADFF844E06C78AE7858
:100EC000164FA8BF08228EF8002092B216FB02F639
:100ED00014FB02F20D4C3E80084E22800024347038
:100EE0001C7091E70820BDE8F8401DF0C1BB00BFB1
:100EF00071970020F4560020586D0020FA5600200B
:100F00003EA80020652D00202CA80020F8560020C7
:100F1000A01E002055A7002058A70020F65600204C
:100F20002DE9F04FB74B1E788BB0002E40F081803A
:100F3000B54BB64C1D78B64FDFF8FCB205F0010595
:100F4000A4F10A0954F80A0CB8B14FF0CC0808FB18
:100F50000698F8F717FB80B154F80A0CF8F70AFB6B
:100F600014F8023C024683B924283BD075B354F8E8
:100F70000A0CF8F707FB0028EED10136032E04F126
:100F8000CC04DFD10BB0BDE8F08F012B2ED0022BAB
:100F900033D0032B40D0042B00F06681052B00F0EA
:100FA0005481062BE3D114F801ECBEF1000F00F0E0
:100FB000D581BEF1010F00F01A8201360023032E05
:100FC00004F8023C04F1CC04BCD1DBE7232A54F83A
:100FD0000A0C00F07F818F4B93F832309342B8D1E6
:100FE000FAF700FD012304F8023CC0E74D2800F0A9
:100FF0006481002304F8023CB9E700233C2804F88C
:10100000023C00F054813E28B1D10122032304F8B0
:10101000012C04F8023CAAE7C028EAD800210423E6
:1010200004F8050C04F8040C04F8061C04F8023C4F
:101030009DE7794B18680028A4D0F9F765F9774B3C
:10104000774D03F5247A774B1868F8F79BFA002858
:1010500098D0744B1868F8F78DFA09281BD03F28F0
:1010600019D02B68002B67D1042800F0B8810C2818
:1010700000F0E4807F28E6D0A0F12002D2B25E2A00
:10108000E1D80BB92028DED067495A1CC8542A6021
:101090000FF042F9D7E72C68002C5AD12646DFF82A
:1010A0007C8100E0984608F11003002E08BF4646F8
:1010B0005345F7D3002E6CD03068D8F80020075D78
:1010C000135D9F42204402EB040140F04581564FDE
:1010D00004F1FF3EBE4422460BB9FD2A5DD90EF84D
:1010E000013F01322A6010F8013F11F801CF9C4501
:1010F000F2D00AB1B04512D04C480FF015F9B04506
:1011000008D356F8100B0FF00FF909200FF004F96F
:101110004645F6D946480FF007F92A68002494425C
:1011200091D2444E264416F8010F0FF0F5F82B68C3
:1011300001349C42F7D386E70C287FD00A2833D0AD
:101140000D2831D07F2800F0BC80FF2B3FF67BAF0D
:1011500092E7324FDFF8D0B04FF0000807F524795E
:10116000464602E010374F450DD2224639685846B0
:101170002FF0F6F80028F5D1B846002EF2D13E4601
:1011800010374F45F1D3002E96D1B8F1000F3FF440
:101190005AAF26480FF0C8F8B3E7511C2020B854C6
:1011A00029607B540A46A5E71F4F0FF02AF93846FD
:1011B00023212FF0BFF8002800F00F81C01B28600A
:1011C00080B1431EF95C202940F00F81FA1843B129
:1011D00012F8011D202903F1FF3050D10346002BE6
:1011E000F6D12B604FF4807200210F482FF06DF87C
:1011F000044B1B78002B3FF4C5AE0D480FF094F85C
:1012000021E700BFF627002071970020BE50002084
:10121000A01E00204086002050250020EC1A040863
:101220006826002064250020682500201C3404085E
:101230002434040867250020F80504087A480FF0D4
:1012400073F87A480FF070F8FDE614F8063C14F8CD
:10125000051C994274D814F8043C83427FF4C9AE4B
:10126000062304F8023C9EE614F8043C04F8030C40
:101270005A40052304F8042C04F8023C77E62B605E
:101280006B4C6C4E002204F52479FA5402E01034C1
:101290004C4551D2216830460EF0F8FB0028F6D0BC
:1012A0004C4549D2E368984700232B609AE7032214
:1012B00004F8013C04F8022C59E6022304F8023C2D
:1012C00055E6013B5B4A5C482B600021D1540FF08E
:1012D0002BF8B8E6594B5A49DB785A4ADFF888E1CF
:1012E0001060003318BF01230B70574B574ACEF8DC
:1012F0000030574BC7F8F8204FF0400E0121C7F8D7
:10130000F400C7F8FC0087F800E1524887F8015163
:1013100019700FF0E5FD45480FF006F84E4A4F49A9
:10132000138891F8321043F08003232913803FF48F
:1013300057AE14F8023C34E649480EF0F5FFB3E727
:1013400014F8041C08EB03005140013304F8041C9A
:1013500004F8063C82720AE62246CAE69BE80F00C1
:101360000DF1280C0DF1080888E80F004CF824ED69
:1013700014F8053C14F803AC0694624623444FF07D
:10138000010C414606A8ADF822E00793ADF820A075
:101390008DF824C000F082FA40B1029A314B0392DA
:1013A0004146A4F10A00029319F004FFDDF804801D
:1013B000002304F8023CB8F1000F3FF4DEAD54F80E
:1013C0000A0C1AF035FC013654F80A0CC047032EFB
:1013D00004F1CC047FF4B6ADD4E52868F0E61548F6
:1013E0000EF072F90BB0BDE8F08F034648E714F831
:1013F000053C14F8032C0694234407936E2A4FF0FF
:10140000000308930993ADF820207FF4D6AD631C48
:1014100006A80693F9F772FA06A8F9F76FFA06A874
:10142000F9F76CFAC9E500BF2C3404082434040829
:10143000EC1A04086825002054340408FC27002016
:101440006857002064250020981F0020898100082B
:10145000F627002058340408BA6D0020408600208A
:101460003834040864BC0020502500202DE9F047E2
:10147000B74C636820469847002800F09F80B54B22
:101480001B780122042B84F8402000F09980B4F9E5
:101490001210B4F91420B4F916306163A263E36347
:1014A000AD4B1B88002B69D0AC4DD4ED0D7AD5ED3A
:1014B000004A95ED090A95ED015A95ED0A7AD5EDA8
:1014C000035A95ED026AF8EEE76AD5ED047AA4EEC8
:1014D000A60AA5EE267A67EEC07AA5EEC07AE6EEF9
:1014E000267A85ED097AC5ED0A7A2CF0E3FDD4ED74
:1014F0000E6AD5ED0B4A95ED140A95ED0C5A95ED53
:10150000157AD5ED0F7AD5ED0E5A95ED0D6A60631B
:10151000F8EEE66AA4EEA60AA5EE267A67EEC07A91
:10152000A5EEC07AE6EE267A85ED147AC5ED157A39
:101530002CF0C0FDD4ED0F6AD5ED164A95ED1F0ACB
:1015400095ED175A95ED207AD5ED1A7AD5ED195A01
:1015500095ED186AA063F8EEE66AA6EEA40AA6EE78
:10156000857A67EEC07AA0EE657AE6EE867A85ED3A
:101570001F7AC5ED207A2CF09DFDE063784EA17EA8
:10158000784813F0BFFA3288002A61D1764DD5F839
:101590004431764A1268520720D404F1340007C857
:1015A000B3F90050401B6063B3F90200091AA1634C
:1015B000B3F90430D21AE263BDE8F087BDE8F087E2
:1015C0006B4BB4F91200B4F91410B4F9162018805A
:1015D00060635980A1639A80E26361E7B5F8AC105B
:1015E000322900F08980002967D195F8AA20002AC5
:1015F000D3D0D5F860115F4E5F4886FB0172C917E2
:10160000C1EB22111980D5F8641186FB0172C9174C
:10161000C1EB22115980D5F86821278A86FB026127
:10162000D217C2EB2112D21B9A800023C0F80A30D5
:1016300085F8AA3013F0A8FBF8F750FF13F08CFBE5
:10164000FCF752F801201DF027F9D5F84431A4E742
:10165000454D616BD5F84431B2F5C87F4FF00002BB
:1016600062631A80308814BFD5F848710027B0F53E
:10167000C87F18BFD5F84C21A06B39443788C5F80E
:1016800048114FF0000E0244B7F5C87FC4F838E0A7
:10169000C5F84C21A3F802E052D0D4F83CC0D5F8EC
:1016A0005001C4F83CE06044012FA3F804E0C5F801
:1016B000500165D0013F37806BE7D5F86061626B00
:1016C00000203244C5F8602160631880D5F8646159
:1016D000A26BA0633244C5F864215880E26BD5F850
:1016E0006861E06332440129C5F86821988073D0AD
:1016F0000139A5F8AC1078E71A8820481E4E676BB0
:10170000A5F854210022B3F802E0B3F804C0D6F8DB
:101710000A60426082606263C5F860711A80A06BE3
:10172000C5F86401A2635A80E06BC5F86801E26302
:10173000A5F856E1A5F858C1C5F85C619A80D7E7CD
:10174000E26BC5F85021C4F83CE0A3F804E0B1E72F
:10175000746D002055A70020302B0020342B002072
:101760005ABC0020A86D0020A01E002018360020C2
:1017700058A700201F85EB51CC7D002000200020C1
:10178000DFF81081DFF8FCC0C83188FB01A9C8323E
:10179000C917C1EBE91188FB02A9D217C2EBE91204
:1017A0005A801980C83088FB0028218AC217C2EBF2
:1017B000E812521A9A80CCF80AE013F0E5FAF8F72A
:1017C0008DFE13F0C9FAFBF78FFF38461DF064F861
:1017D0003788D5F844316DE7274A85F8AE0012689E
:1017E00085F8A91012F4003203D0244A1279002A95
:1017F00035D11046224E375C0C2F00F10C0011D071
:101800000132152AF7D1B5F854011E4A1880B5F8EF
:101810005671B5F85861D5F85C015F809E80C2F8BA
:101820000A0065E7184FD7F800C05000BCF1000F60
:1018300009D000EB020E06EB8E0E9CF801C09EF85C
:1018400001E0E645DFD20244DFF84CE00F4806EB4A
:10185000820600223E60AEF800200260D3E70C4A08
:1018600012780AB10246C5E71CF0E6FED5F844310D
:10187000B5F8AC10C7E700BF44250020586D002024
:10188000D00C0408CC7D0020A02400203C250020A2
:101890003EA800201F85EB513A2500202DE9F04F8E
:1018A000B0F908502DED048B0D81EDB2382D87B0C5
:1018B0000C4600F0B4828046914634D9802D00F069
:1018C0000A8179D8522D00F0BA8040F28882542DD6
:1018D00000F0F1826E2D40F04781944B0A681B881E
:1018E000934DFF2BA8BFFF23511C21601370A968E3
:1018F00081F3100189B22046F9F754F88D4B204648
:101900001988F9F74FF8296801F30F0189B22046C9
:10191000F9F748F801252B462846638107B0BDEC4E
:10192000048BBDE8F08F042D00F09F8240F22282EC
:10193000202D00F0B48040F25D82242D00F0C7829B
:10194000282D40F011810B68DFF810827A4E591C67
:10195000022221601A70236806275A1C22601F7019
:1019600023680A22591C21601A70236801255A191C
:1019700022601D70B8F800102046F9F713F8B8F887
:1019800002102046F9F70EF823685A1922601F70DA
:1019900023685022591921601A70236800225919AE
:1019A00021601A7031882046F8F7FCFF71882046C4
:1019B000F8F7F8FF2B46AFE7822D48D0C0F09982A8
:1019C000A02D00F08A82FE2D40F0CE805B4D05F107
:1019D000080635F8021B2046F8F7E4FFB542F8D1B7
:1019E00098E7F52D01F05E82762D40F0EA82D8F876
:1019F00000305A1CC8F800201B78002B01F04D83E2
:101A0000102B07BF4E4A92E8220000252946226883
:101A1000501C206013702046F8F7ACFF2946204682
:101A2000F8F7A8FF474B20461968F8F7A3FF0021F5
:101A30002046F8F7B7FF00212046F8F7B3FF2268E9
:101A40000021531C012523602B46117064E70B68AD
:101A50003D4A374D11783D4A581C20601970D18895
:101A60002046F8F79FFF314B22681B88FF2B02F1BD
:101A70000101A8BFFF2321601370A96881F3100141
:101A800089B22046F8F78EFF296801F30F0189B269
:101A90002046F8F787FF2E4B22681978D1E70B68AC
:101AA0002A4D591C6A7821601A7023682A78591CBB
:101AB00021601A702368AA78591C21601A70E9887D
:101AC0002046F8F76FFF23682A79591C21601A70A5
:101AD00022686979B5E71F4E1F4FDFF884A0DFF851
:101AE000849006F10D080A2517E0322D00F05A8186
:101AF000A5F13C00C0B2132840F25B8100232268AC
:101B0000511C216015702268B04502F1010121606D
:101B100013703FF4FFAE16F8015B0A2DE5D1B9F85A
:101B20000030FF2BA8BFFF23DBB2E8E72CA8002082
:101B3000AC6B0020622D00207C56002058A70020AE
:101B4000881F0020EC2200203EA80020586D0020B5
:101B5000652D00204906040867666666BC7D002086
:101B600094560020C4560020A5F10A03E72B00F28A
:101B7000EA80DFE813F04F06E800E800E800E8003C
:101B8000E800E800E800E800E800E800E800E80015
:101B9000E800E800E800E800E800E800E800E80005
:101BA000E800E800E8001E06E800E800E8000D068E
:101BB000E800E800E8000806E800C705E800760548
:101BC000E8006A05E8006505E8003F05E8002C0527
:101BD000E800E800E80024051B05E8001105E8001E
:101BE000E8000805E800E800E800E800E800EA048A
:101BF000E800E800E800E800CE04E8000D08E8008E
:101C0000A807F507E800E800E800E800E800E800B9
:101C1000E8003107E800EB06E800BC06E8007206C1
:101C2000E8006106E800E800E800E800CF07750773
:101C3000C5049D048B0465044F043604B203E80018
:101C400078035B03E800E800E800E8004F03E800E1
:101C5000E800D103E800E800E800C0031D043F03EA
:101C60000103E800E800E800F002DD02D202E8002B
:101C7000E800E800E800E800E800E800E800E80024
:101C8000E800E800E800E800E800E800E800CF0726
:101C9000E800E800E800E800E800E800E800E80004
:101CA000E800E800E800E800E8009902E800E80041
:101CB000E800E800E800E800E800E800E800E800E4
:101CC000E800E800E800E800E800E800E800E800D4
:101CD000E800E800E800E800E800E800E800E800C4
:101CE000E800E800E800E800E800E800E800E800B4
:101CF000E800E800E800E800E800E800E800E800A4
:101D0000E800E800E800E800E800E800E800E80093
:101D1000E800E800E800E800E800E800E800E80083
:101D2000E800E800E800E800E800E800E800E80073
:101D3000E800E800E800E800E800E800E800E80063
:101D4000E8008D023D02742D00F02A81772D7FF48A
:101D500048AED8F80030D8F804209A421EBF5A1C6A
:101D6000C8F800201978B74A08BF00212046FAF7C2
:101D70001FFECFE5022D00F0968000F28380012D3A
:101D80007FF4F2AE0B680022591C21601A702368A0
:101D90005A1C22601D7022682421531C23602B468C
:101DA0001170B9E5BAF80030FF2BA8BFFF23DBB2F2
:101DB000A5E628F0F3FD00283FF4A0AE03780A2B37
:101DC00000F21481B0F9023087FB0312DB17C3EB7A
:101DD000A2039BB2FF2BA8BFFF23DBB28FE6442DEB
:101DE0007FF4C2AE002A3FF495AD974B13600125F6
:101DF0002B4691E5052D7FF4B7AE0B229349204683
:101E0000F8F788FD082292492046F8F783FD01255E
:101E1000072290492046F8F77DFD2B467CE50A68AD
:101E20008D4B0125511C2160157022680521501928
:101E30002060117022680A215019206011702268F8
:101E40000021501920601170226819785019206003
:101E500011702268597850192060117022689978A1
:101E6000531923602B46117056E52A467B492046BC
:101E7000F8F750FD7A4B20461978F8F793FD226861
:101E80000021DEE50B680222591C21601A702368CC
:101E900001255A1922601D70226800215319236000
:101EA0002B46117038E504226E4920460125F8F7CB
:101EB00031FD2B4630E50B6800215A1C2260197059
:101EC00022680125531923602B46117024E5664BC7
:101ED00019682046F8F74EFD1CE5644B0846196862
:101EE000F8F748FD624B20461968F8F743FD614B4F
:101EF000EEE7DFF89891604F09F10E064FF00A08FF
:101F00001DE0B8F1500F32D0B8F1320F31D0A8F146
:101F10003C00C0B213282FD90025294623685A1C3B
:101F20002260204683F80080F8F73CFD29462046D1
:101F3000F8F738FD4E453FF4EDAC19F8018BB8F1D8
:101F40000A0FDED14D4B9D68196805EB85054FF6EC
:101F5000FF736D009D42A8BF1D469942A8BF194658
:101F600025EAE57521EAE171ADB289B2D6E7444BC5
:101F7000E9E797E82200E8E728F010FD0028CBD039
:101F800003780A2BC8D8B0F90430B0F9061003EB77
:101F9000830383F3500521EAE171ADB289B2BDE755
:101FA000D8F80030D8F804209A421EBF5A1CC8F84E
:101FB00000201978334A08BF00212046FAF7F8FCC0
:101FC000A8E4472D00F06C86292DD8F8003000F0E9
:101FD0005086392D00F01E86212D00F027862846D8
:101FE0004146FBF72BFD054603B295E40023F4E6DA
:101FF000254B03F1700522681978501C2060117080
:1020000022685978501C2060117022689978501C01
:10201000206011702268D978501C206011702268ED
:102020001979501C2060117022685979501C206069
:102030001170226899790733501CAB4220601170EF
:10204000D9D167E4D5C5000895C60008A0340408B6
:10205000AC340408B8340408D78600209834040847
:102060000C20002090340408FC870020107AFF1F09
:10207000147AFF1F187AFF1F8C560020405600204C
:10208000805600206DC60008B8720020390604088A
:10209000B24D2046A989F8F785FC698920460125BB
:1020A000F8F780FC2B4637E42368DFF8FCC2591CA4
:1020B0009CF8002021601A709CF80030002B3FF43F
:1020C00029ACA74EA74DA848A8490023226816F8B6
:1020D000017F02F1010EC4F800E01770226815F8C4
:1020E000017F02F1010EC4F800E01770226810F8B9
:1020F000017F02F1010EC4F800E01770226811F8A8
:10210000017F02F1010EC4F800E017709CF8002076
:1021100001339342DADBFFF7FDBB954B9549B3F9E9
:10212000003081FB0321DB17C3EBA101FFF7EEBBFE
:102130002268914B501C19782060117022685978E0
:10214000501C2060117022689978501C206011701A
:102150002268D97875E4894D2046A98AF8F722FCCF
:10216000E98A2046F8F71EFC298B20460125F8F75E
:1021700019FC2B46FFF7D0BBDFF830E20027FEB298
:10218000714600232268501C206016702268501C83
:1021900020601370226811F8010F0133551C062BC3
:1021A00025601070EED10137062F0EF1060EE6D134
:1021B000734900232268501C206017702268501C4D
:1021C00020601370226811F8010F0133551C0B2B8E
:1021D00025601070EED123686A49581C07222060E0
:1021E0001A7023680022581C20601A70226891F827
:1021F000F01026E42368644A5D491078574A5D1C54
:102200002560187023689278581C20601A70226824
:10221000897816E45D4952232268501C20601370AF
:1022200011F8013F002BF7D1FFF774BB584800238A
:102230002268056803EB4301561C6D5C266015702F
:10224000026825680A446E1C527826602A7002686B
:1022500025680A4401339278691C0A2B21602A7090
:10226000E6D1FFF757BB4B4D23682A68591C1278FB
:1022700021601A702B6822689978531C2360002310
:1022800011702A6821681A4401335279481C032BC3
:1022900020600A70F5D123682A68591C127A2160DF
:1022A0001A7023682A68591CD27821601A70236832
:1022B0002A68591C127921601A702B6820465989A6
:1022C000F8F770FB23682A68591C527A21601A704B
:1022D0002B6822685978FFF7B4BB2F4B204619684A
:1022E000F8F748FB2D4B204619880125F8F75AFBD3
:1022F0002B46FFF711BB2A4D20462988F8F752FBE1
:1023000069882046F8F74EFBA98820460125F8F792
:1023100049FB2B46FFF700BB224D05F16006A9885B
:102320002046F8F73FFBE9882046F8F73BFB298970
:102330002046F8F737FB2368AA7A591C21601A70E7
:102340002368EA7A591C21601A7055F80C1B204644
:10235000F8F710FBB542E2D1FFF7DCBACC7D0020E4
:102360002F2F00203F2F00205F2F00204F2F002015
:10237000E47D002067666666142F00200C31002083
:10238000CF6F0020EC6E002014980020080604088F
:10239000C06D0020C46D0020646D0020686D0020B9
:1023A000F47900208C7A00202D2F0020AB6F0020C4
:1023B0002268B84BB8491878551C256010702268FF
:1023C0005878551C2560107022689B78501C20603E
:1023D0001370C98820460125F8F7E4FA2B46FFF769
:1023E0009BBAAE4D20462988F8F7DCFA698820466A
:1023F000F8F7D8FAB5F90430A949DA1781FB0313C5
:10240000C2EBA30399B220460125F8F7CBFA2B467D
:10241000FFF782BAA34B20461988F8F7C3FAA24BFC
:1024200020461988F8F7BEFAA04B21681A780125D2
:102430004B1C02F0010223602B460A70FFF76CBAB6
:102440009B4B22681B789B4D511C03F002032160BB
:10245000137023682A78591C21601A706968204615
:10246000F8F788FAA9682046F8F784FAA98920467F
:10247000F8F798FA698A2046F8F794FAA98A20466C
:102480000125F8F78FFA2B46FFF746BA8A4E3378C4
:10249000002B3FF43FAA894F002537F8021F204642
:1024A000F8F780FA337801359D42F6DBFFF732BA50
:1024B000834D844EDFF84482DFF84492DFED828A58
:1024C000DFED829A9FED829A05F1200708E0204611
:1024D0000435F8F767FAAF4206F118063FF41AAA76
:1024E000717C0029F3D095ED008AB0EE480A2BF0FC
:1024F000E1FD98F80030002B40F0468581B2E6E718
:102500001022744920460125F8F704FA2B46FFF7FC
:1025100003BA2368704D591C2A7821601A70236809
:102520006A78591C21601A7069882046F8F73AFACF
:1025300023682A79591C21601A70E9882046F8F727
:1025400031FA2268297AFFF77CBAF8F735FF236859
:10255000624D002803F101010CBF02220322216019
:102560001A7029882046F8F705FAE9682046F8F736
:1025700001FAF8F771FE012501462046F8F7FAF94D
:102580002B46FFF7C9B90822554920460125F8F71F
:10259000C1F92B46FFF7C0B92268524B501C9978FD
:1025A0002060117022685978FFF74BBA2268012128
:1025B000531823600D460B461170FFF7ADB900218B
:1025C00020460125F8F7D6F92B46FFF7A5B9464D69
:1025D000464E05F1300795F902100023F2568A4263
:1025E00000F0FB820C33482BF8D10835AF42F2D112
:1025F000FFF790B93E4B03F15A0522685979501CF8
:102600002060117022681978501C206011702268B7
:102610005978501C2060117022689978501C2060F5
:1026200011702268D978501C2060117022681979C5
:102630000633501C9D4220601170DED1FFF76AB94D
:10264000274B2268597DFFF7FCB92A4D05F180061A
:1026500055F8041F2046F8F78DF9AE42F8D1FFF780
:1026600059B9254D05F14006B5F880102046F8F718
:1026700099F9236895F88220591C21601A70236803
:1026800095F883200435591CAE4221601A70EBD1B5
:10269000FFF740B9C47D0020F47900206C6D002064
:1026A00067666666302E0020322E0020E42D002062
:1026B0003D6D0020406D00205C280020CA540020A1
:1026C000BC7B0020F0A40020000040420040744485
:1026D00000E08244AC7B00200C7A0020C007002080
:1026E000E8350020F07D002040860020A035002045
:1026F000A8260020E86E0020EC6E00203431002077
:1027000018360020A74D23682A7A591C21601A70B8
:10271000A98B2046F8F746F9298B2046F8F742F9AD
:10272000698B2046F8F73EF92368EA7C591C216042
:102730001A70E98C2046F8F735F9298D2046F8F70C
:1027400031F92368AA7F591C21601A70236895F813
:102750002020591C21601A70A98C2046F8F722F914
:102760002368EA7A591C21601A70E9682046F8F754
:1027700001F923682A7C591C21601A70226895F897
:102780002110FFF75EB9884B22681978FFF759B915
:10279000864D20462988F8F705F9A9882046F8F7DC
:1027A00001F9298920460125F8F7FCF82B46FFF7A7
:1027B000B3B87F4D7F4F05F15006002128787E4A3F
:1027C0000B4607E00133242B02F10C0200F00282D9
:1027D00012F80C1C8842F5D103EB4303226807EB87
:1027E0008303511C93F864302160137023686A7866
:1027F000591C21601A702368AA78591C21601A702C
:102800002368EA780435591CAE4221601A70D4D18D
:10281000FFF780B869482AF039FA00287FF77AA8CC
:10282000664B1D18226813F8011B501C9D42206046
:102830001170F7D1FFF76EB82368614A6149D0780B
:10284000614A5D1C2560187023681278581C20604E
:102850001A702268C978FFF7F4B800212046F8F70B
:10286000A1F800212046F8F79DF800212046F8F74E
:1028700099F82268554D0023511C2160137022687D
:102880002968501C91F82F10206011702268296867
:10289000501C91F83A102060117022682968501C71
:1028A00091F83B10206011702268511C2160137058
:1028B0002268511C216013702268511C2160137022
:1028C0002B682046D98FF8F76DF82B682046998F32
:1028D000F8F768F823682A68591C92F831202160BB
:1028E0001A702B68226893F83210FFF7AAB8384D97
:1028F00023686A79354E591C21601A703368204666
:10290000198CF8F74FF833682046598CF8F74AF8D5
:1029100069892046F8F746F8A9892046F8F742F871
:1029200033682046998CF8F73DF833682046D98CF7
:10293000F8F738F8E9892046F8F734F8298A20466C
:102940000125F8F72FF82B46FEF7E6BF204EF37867
:10295000002B00F0058323680822591C21601A709F
:1029600023680122991821601A702368194D591C97
:102970002A7921601A702368AA78591C21601A707C
:1029800029882046F8F70EF8698A2046F8F70AF8F1
:102990002368F279591C21601A702268E978FFF7E0
:1029A00050B800BFE8350020FC7D0020D86400202E
:1029B000007E002008060408700604080128002094
:1029C000CC7D0020E47D0020DC7D0020C06D002057
:1029D000149800200C31002010F0F2F9FF28064670
:1029E00000F0088306A9002501F8125D0DF105002D
:1029F0008DF8055010F0C4F906A800F8115D10F02C
:102A0000B3F906A800F8105D10F0A2F906A820F8A6
:102A1000085D10F091F923685A1C22601E7023682B
:102A20009DF80520591C21601A7023689DF8062026
:102A3000591C21601A7023689DF80720591C2160D9
:102A40001A7023689DF80820591C21601A70BDF87F
:102A5000101020460125F7F7A5FF2B46FEF75CBFB7
:102A6000C74E338AB3F5007F06F1340594BF0127C2
:102A70000427403655F8041B91FBF7F1204689B234
:102A8000F7F790FFAE42F5D1BE4DBF4F05F10C06F2
:102A9000B5EC010AD7ED087A80EE270A2BF00AFB85
:102AA00081B22046F7F77EFFAE42F1D1B74D05F176
:102AB0000C0655F8041B204689B2F7F773FFAE42A7
:102AC000F7D1FEF727BF2368B14D01269A1922607E
:102AD0001E7025F095FB002840F07F82AD4B2268E8
:102AE000511C21601070226841F2B410511C185C16
:102AF000216041F27811107059582046890AF7F781
:102B000039FFE96B204649080125F7F733FF2B46CB
:102B1000FEF702BF0023DFF89492DFF894B203932C
:102B2000029304930593984601214FF6FF7A07E03C
:102B300008F10108B8F10B0F00F0FA8019F9011F34
:102B40004E1CF5D04AFA08F3D807F1D5BBF800308F
:102B500043FA08F3DA07EBD504A8F8F7B5FAE7E784
:102B600022688D4B0125511C2160157022689978CF
:102B70005019206011702268197850192060117066
:102B800022685978531923602B461170FEF7C4BE92
:102B9000824E3378002B3EF4BDAE814F0025B846FF
:102BA000236817F81520591C21601A7098F8011035
:102BB00001EB810101EB810101F2EE2189B2204696
:102BC000F7F7F0FE337801359D4208F10208E7DBA4
:102BD000FEF7A0BE00231B7AFFDE23685A1C22608A
:102BE000197029882046F7F7DDFE2368EA78591C1A
:102BF00021601A7023682A79591C21601A70236891
:102C0000AA79591C21601A7023686A79591C2160BD
:102C10001A70EAE45A1CC8F800201A780A2A00F050
:102C2000A0824FF0FF352B46FEF776BE1A46591CA0
:102C3000C8F800105B4D12F8021B6970C8F800203C
:102C40005A782A70DA1CC8F800209B78AB7040468E
:102C5000F7F754FED8F80030E880591C1A46C8F837
:102C6000001012F8021B2971C8F800205B786B7104
:102C7000D7E75A1CC8F800201B780A2B00F0B58152
:102C8000502BCED14046F7F739FE474E30804046B4
:102C9000F7F734FE4FF0FF3570802B46FEF73CBE51
:102CA000D8F80430D8F8005040465D1BF7F70EFE08
:102CB000052D064600F2608180252F464FF0010861
:102CC00094E80C009B1A103BDFF8E890AB42B8BFC9
:102CD0009FB2D9F80C309B1B9F423146204688BFDB
:102CE0009FB2F7F747FEB8F1000F00F08B81D9F8DB
:102CF0000C30D4F80080F2199A4200F24382F8F7BF
:102D000053FC41463A463046F8F7CEFC2368A842C9
:102D100003442360B8BF002102DBFEF7FBBD23683C
:102D200001305A1CA84222601970F8D1FEF7F2BD9A
:102D3000DFF884A04FF000084FF0080908F10108FF
:102D4000B8F1240F3AD0C8F1200209FA02F22AFAA7
:102D500008F6A8F12003164329FA03F31E4306F0F0
:102D6000010200231343E9D05FFA88F00EF000FF60
:102D70000028E3D0414604A8F8F7A6F9DEE700BF33
:102D8000746D002050A000202898002038280020D2
:102D900018530020903E0020018800205C2800206D
:102DA0001C2D0020586D00207C5600205806040879
:102DB000BC6D0020C007002090E33FF4C64B1B7899
:102DC000DB0700F148810026C44FB04602E001361F
:102DD000242E0ED031463846F8F786F90028F6D072
:102DE000314604A8F8F780F9002856D108F1010807
:102DF000EDE7BB4BBB4EB3F850102046F7F7D2FDC2
:102E0000B94B1988204689B2F7F7CCFDB74B1A6841
:102E1000530103F02001C2F340030B43C2F38001CE
:102E200043EA4103C2F3C00143EA8103C2F3401104
:102E300043EAC10102F0100211432046F7F7B2FD48
:102E400002A904222046F7F765FD23683178A84AD5
:102E5000581C2060197011886429A8BF642120467D
:102E6000F7F7A0FD962D00F0EB8000212046F7F744
:102E700099FD2168B8F1190348BFA8F11203A3F323
:102E8000C4034A1C226020460B701A4603A9012580
:102E9000F7F740FD2B46FEF73FBD414602A8F8F785
:102EA00013F9A3E7D8F80030D8F804209A4240F08C
:102EB0000081904BFF221A734FF000088E4D06F0F0
:102EC00037FD414630228D4885F800802DF0FDF910
:102ED0008DF810809DF810300B2B00F25A81884F2E
:102EE000864E42469DF8103003EB430307EBC303C5
:102EF0005B7CE3B19DF8103003EB430307EBC303A6
:102F00005B69A3B19DF8103003EB430307EBC303E8
:102F10002021586946F82200F6F7F4FC2B7856F881
:102F20002300F6F7ADFD2A780132D2B22A709DF85F
:102F300010300133DBB28DF810309DF810300B2BC0
:102F4000D0D92368591C21601A70B9F1000F3EF4E2
:102F5000E1AC6C4BC9F8003001252B46FEF7DCBC18
:102F60002368B178684A581C206019702368127869
:102F7000591C21601A70F8E44046F7F7BFFC4FF087
:102F80000008074605469BE6D9F8003013F4805345
:102F9000B4EEE88A00F08680F1EE10FA11DBB4EEB0
:102FA000C98AF1EE10FA5BD8DFED587A9FED587AB6
:102FB00077EEC87AB4EEC78AF1EE10FAB0EE678AFF
:102FC0004ED94FF47A71B5EE408AF1EE10FA40F224
:102FD000DC5308BF1946FFF77ABA95F824204D4B09
:102FE000002A40F0B680304679E54046F7F786FC87
:102FF000494E4BE622680125531923602B46107079
:10300000FEF78ABC39462046F7F7CCFC23685A1CE9
:10301000226083F80080D9F80C50D4F80080F219AF
:10302000954280F0B880AD1BF8F7BEFA2A464146BB
:103030003046F8F739FB236803442360FEF76ABC87
:1030400023680322591C21601A7023687278591C66
:1030500021601A700DE7049B43F001030493B2E66C
:10306000F7EE007A78EE677AB6EE007AF0EE696AEB
:10307000E7EE876A40F2E932FDEEE67A17EE901A43
:10308000B1F5FA6FA8BF4FF4FA619142B8BF11468B
:1030900089B2002B3FF41BAA95E7204A92E8220050
:1030A000FEF7B5BCF1EE10FADADA4FF47A71FFF7F9
:1030B0000EBA5A1C1946C8F800200E4811F8022B07
:1030C0000273C8F800105B784373042A28D9FF2ADA
:1030D0007EF4B5ACF0E600BF719700201020002010
:1030E0003C030020FC27002038B9002064A0002009
:1030F000622500200C2000209B6600204C660020EA
:10310000F0A4002059CD0208C07D002000C08844F2
:1031100000C08244903E0020BC7D0020282E00206C
:1031200024490978994205D8022A7EF488ACFF2BFD
:103130007EF485AC236801255A1922601D70B9F10F
:10314000000F3EF4E7AB1C4BC9F800302B46FEF7EE
:10315000E3BB5978022917D003290CBF042030465D
:10316000BDE49A1CC8F80020144A59781170D91C83
:10317000C8F8001099785170191DC8F80010DB7854
:1031800093704EE59F1BBAE5042A34BF022003204A
:10319000A5E44246D5E6F8F707FA3A4641463046F6
:1031A000F8F782FA23680125034423602B46FEF7D3
:1031B000B3BB00BF45A70020A1C60008D7860020EA
:1031C0002DE9F04F2DED028B91B005461CF06CFB04
:1031D000814B1F7827B111B0BDEC028BBDE8F08F99
:1031E0007E4B1A685205F6D57D4A1278002A40F0C7
:1031F00098817C4B1B78002B6DD07B4C7B4AD4F89C
:103200001C31EB1A934201F26C8494F82471A7BB31
:10321000DFF80C82D8F80000F6F7B4F9C0B2012844
:103220000ED9022841F09686714B1A78002A42F096
:103230007580D4F82821AA1AB2F57A6F82F02A8113
:10324000D4F82C31002B46D094F82431C3B9694B03
:103250001B689B7801211E3B00228B4284F82411BD
:1032600084F8382142F2BF80D8F8000002210430EF
:103270001CF0F6F994F8303110E0D4F82C3153B347
:10328000D4F8343140F6B732EB1A934223D994F88C
:103290003031002B01F08085DFF88481013BDBB207
:1032A00084F83031002B01F05485D4F82C7194F857
:1032B000382117F8011B94F83931D8F80000C4F808
:1032C0002C710A44013384F8382184F83931F6F737
:1032D0005DF9C4F834511BF0BFFD474B1B786BB14F
:1032E000DFF84091D9F8003043B1444B3E4C1B68A5
:1032F000D4F83C219A1A632A00F2F681404C2378D4
:10330000022B01F03685DFF8208198F80030032B7E
:1033100001F00B853B4B1B7873B13B4F3B685BB1B6
:10332000314CFBF79BFBD4F84431019044F61F620B
:10333000C31A934200F2BA82344B1B78002B75D12A
:10334000334B1B7843B1284CD4F8943203F5C33384
:10335000A0339D4281F086832E4B1B78002B3FF4D7
:103360003AAF214E2C4C2D4D06F2B5272068F6F7CA
:1033700009F900283FF42FAF2068F6F7FBF82B7807
:1033800080465A1E33B120682A70F6F7FBF80028F1
:10339000F2D120E703223946781E2CF07CFF96F804
:1033A000B43296F8B52286F8B78283F47F4383F06F
:1033B000FF039B1A1FFA88F89BB2B8EB132FD5D1E5
:1033C00096F8B622DBB29A42D0D1781E27F05EFB87
:1033D0002B7818442870C9E7F627002018360020FB
:1033E000246E00202E6E00201C2000203F0D0300C4
:1033F00035000020CC6D0020386E0020C4B80020BD
:1034000010660020406E0020446E0020D86E002020
:10341000E66E00204A6E0020506E0020546E0020A0
:10342000C86D002050A80020D10200209D4C2278B9
:10343000002A41F00E839C4CD4F88C3203F5C33340
:10344000A0339D42FFF47CAF984A94F89032C4F8C0
:103450008C52D75CFA0701F1E585BB0701F1A08525
:10346000780701F12C863A074FD5914BDFF86C8233
:10347000099310AA1146A3F1210241F8202D002042
:10348000A3F124020E4603F8240C02910223112119
:10349000517093703046D8F80410F7F745FA30466B
:1034A000D8F80810F7F740FAB8F81230814903EB62
:1034B000C3039B00053381FB0321DB17C3EBA10191
:1034C000304689B2F7F748FAB8F8143003EB8303B3
:1034D000590089B23046F7F73FFA774B029E1B78C6
:1034E0009B0743BFB8F80C1001F57A7189B24FF40D
:1034F0007A713046F7F730FA089B98F80020591C8B
:10350000089130461A701CF08DF96C4A94F890328C
:103510001178013393FBF1F201FB123384F89032FE
:103520000EE7614C664BD4F8102119688A1A7C2A80
:103530007FF65FAE94F81421DFF8A4919FED618AC5
:10354000C4F81011013284F81421A9F1340A4FF0A3
:10355000240840461CF0FCF8BAF81030F9EC016A77
:1035600007EE103AF8EEE66AB8EEC77A08F10108FD
:10357000C6EE877A5FFA88F867EE887AFDEEE77A1A
:10358000CDED017ABDF904B05FFA8BF01CF0B6F80E
:10359000CBF307201CF0B2F8B8F1270FD9D13020B7
:1035A0001CF0D6F8484ADFF83C91D2F800805FFA68
:1035B00088F01CF0A3F8C8F307201CF09FF8D9F896
:1035C00000005E21F5F7E2FF94F8142193072DD156
:1035D000D4F8101141F28832914201F22C87142064
:1035E0001CF0B6F8394A3349B2F9042081FB0231A4
:1035F0004FEAE278C8EBA1080FFA88F85FFA88F082
:103600001CF07CF8C8F307201CF078F81C201CF094
:103610009FF800201CF072F800201CF06FF85E216B
:10362000D9F80000F5F7B2FF94F8142112F007085A
:1036300001F0A685282A7FF4DCAD214B4FF000086D
:1036400017201F6884F814811CF082F840461CF093
:1036500055F81F4B1F4CA3FB07239B0BA4FB031226
:103660005209C2EB0212A3EB8203D8B21CF046F857
:1036700018201CF06DF8184BA3FB07239B09A4FB33
:1036800003125209C2EB0212A3EB8203D8B21CF060
:1036900035F840461CF032F8D9F800005E21F5F705
:1036A00075FFA6E51C6E00201C200020E06E0020A7
:1036B000F86D0020676666663D6D0020E56E0020AF
:1036C000C4B8002000007A44686D00206C6D0020B2
:1036D00073B2E74589888888D34D6210406D002019
:1036E000A86D0020D06D0020DFF8B081019341204B
:1036F00027F0A6FA644FB8F90220DFF8A4B187FBDF
:103700000230D217C2EBA00080B227F07DFAB8F9E0
:10371000002087FB0230D217C2EBA00080B227F056
:1037200073FAB8F9042087FB0230D217C2EBA0006D
:1037300080B227F069FA9BF80010D9F80000F5F77D
:1037400025FF94F84071019B17F0010801F07D837B
:10375000DFF844A1DAF80020910640F185804B4A59
:10376000DFF840811278920741F13A8698F80020FC
:10377000042A8CBF032702274720029327F060FA10
:10378000D8F8040027F00CFAD8F8080027F008FA57
:10379000B8F812203E49D9F80000A1FB0232C2F36A
:1037A000471211460192F5F7F1FE9BF80000DAF896
:1037B0000010019A029B424011F0140F8BF8002078
:1037C00041F0A885B8F80C20642000FB02F00193BA
:1037D00027F0E6F998F80020D9F8000047EA8207B8
:1037E000FFB23946F5F7D2FE9BF80020D9F8000069
:1037F000574039468BF80070F5F7C8FE94F84071D1
:10380000019B8FBBDFF8A08001934F2027F018FAAF
:10381000D8F8000027F0C4F9D8F8040027F0C0F960
:10382000384627F0BDF90121D9F80000F5F7AEFEC2
:1038300016499BF800200F78D9F8000007F001071F
:10384000394682F001028BF80020F5F79FFE9BF8C5
:103850000020D9F80000574039468BF80070F5F782
:1038600095FE94F84071019B0A4AC4F83C317B1CD8
:10387000DBB2A2FB0312D20802EB8202A3EB4203EB
:1038800084F840313AE500BF676666663D6D00200A
:103890001F85EB51CDCCCCCC64A000206C6D0020FA
:1038A00054A80020406D0020282E002094F84A31B2
:1038B000002B41F03383E84B1B6803F00802002A19
:1038C00048F603414AF60B404BF60F4249F60748CB
:1038D00004BF0246884613F0040F4FF0190118BFC9
:1038E00090469B0684F84A1103D548F4804848F076
:1038F0002008DA4B1A79C8F3090B002A41F0FE853B
:103900005B79002B41F08C87994664204FF0FF33A0
:103910004FF0000ACDF82080CDF82480CDF828B0F3
:10392000ADF82E90ADF830308DF83E00ADF82CA0FB
:10393000CDF832A0CDF836A0CDF83AA00DF1200E8A
:10394000BEE80F00DFF824C384F805A0ACE80F0040
:103950009EE80F00ACE807002CF8023B61464FF0F0
:1039600001081B0C4FF0FE0E1F20C82201F81E3963
:1039700084F802E0A27184F80780E07094F85A019C
:10398000207180F0F10383EA0313DAB2130983F0A4
:10399000E70343EA022383EAC2031BB283EA03126A
:1039A000D2B2C3F3072383EA121343EA022383EA62
:1039B000C2031BB283F0C80282EA0212D2B2C3F37E
:1039C000072383EA121343EA022383EAC2031BB2EA
:1039D00083EA080E8EEA0E1E5FFA8EFEC3F30722FC
:1039E00082EA1E1242EA0E2200EB080382EACE0EA1
:1039F0000CEB080084F85A31A4F800E011F8013B00
:103A000083EA0E0383EA0313DBB21A0982EA1E2259
:103A100042EA032282EAC3031BB21FFA83FE8142F9
:103A2000A4F800E0EAD183F07C0383EA0313DBB25D
:103A30004FEA131C8CEA1E2C8CEA032C8CEAC30C74
:103A40000FFA8CFC1FFA8CFADFF82492A4F800A07D
:103A50005FFA8CFC4FEA1A2A84F828A084F827C061
:103A600009F5C17B04F12208D9F80000D9F8041047
:103A7000D9F80820D9F80C30DE46AEE80F0009F17D
:103A80001009C145F346EFD1D9F80000CEF8000087
:103A9000DFF8E08199F804308EF8043008F1270946
:103AA00084F8A9C184F8AAA118F8011F3868F5F7AD
:103AB0006DFDC145F8D194F84B21002A41F0788181
:103AC0006749684B08781B680A2184F84B11002865
:103AD00001F05182DFF8A0C10128BCF80010039169
:103AE00041F296860228BCF8029001F04B85BCF8A2
:103AF00004100291032801F0A3860428BCF806B044
:103B000001F099860528BCF808E001F090860628A7
:103B1000BCF80A8001F066860728BCF80C1001D0BA
:103B2000BCF80E2094F85A010893064686F030033C
:103B300083EA0313DBB24FEA131C4B4804968CF064
:103B40007A0C4CEA032C008826718CEAC303DFF858
:103B50002CC1C0EB00208CFB00AC8444C0171BB20E
:103B6000C0EB6C200646C3F3072C83EA0310039BCB
:103B70008DF83560C0B24FF0000A63F30F0A8CEA8B
:103B8000101303934FF0000C029B69F31F4A6EF36E
:103B90000F0C4FF000094FF0000E63F30F0961F3B3
:103BA0000F0E039BCDF824A068F31F4C62F31F4E49
:103BB0004FF000086BF31F49CDF82890CDF82CC0CA
:103BC000CDF830E08DF8348043EA00230DF1200970
:103BD00083EAC00EB9E80F000FFA8EFE8EF0C80A15
:103BE0008AEA0A1ADFF884C084F805805FFA8AFA44
:103BF000CEF3072EACE80F008EEA1A1E4EEA0A2317
:103C000099E8030083EACA031BB283F0230E4CF841
:103C1000040B8EEA0E1E5FFA8EFEC3F3072282EAC1
:103C20001E12049B604642EA0E2203F1010882EA5A
:103C3000CE0E20F814194FF02309FE211622C823B6
:103C400084F85A81A4F800E084F807900CF1020C83
:103C5000A170E27014E000BF64A00020586D002045
:103C60005C280020C4B80020622D00202420002001
:103C70001E2000209F210020CC540020030820801B
:103C8000A37110F8013B83EA0E0383EA0313DBB24E
:103C90001A0982EA1E2242EA032282EAC3031BB205
:103CA0001FFA83FE6045A4F800E0EAD183F0F40334
:103CB00083EA0313DBB21A0982EA1E2282EA032294
:103CC00082EAC3031BB21FFA83FEDFF80C84A4F858
:103CD00000E05FFA83FC4FEA1E2A84F81EC084F8D5
:103CE0001FA0D8F80410D8F80820D8F80000D8F899
:103CF0000C3008F5C17EAEE80F00D8F81000D8F8F7
:103D00001410D8F8182004F2A119AEE8070004F244
:103D1000831884F8A1A184F8A0C118F8011F38689D
:103D2000F5F734FCC145F8D194F84E31002B41F041
:103D3000FA80DFF8B0A3DAF800301922980684F888
:103D40004E2140F12083E34BDFF89C831B789907D9
:103D500041F1D08398F80030042B8CBF4FF0030959
:103D60004FF00209FAF77AFEB8F81430B8F80C20D0
:103D7000089003EB83035B00ADF83A304FF47A70A0
:103D8000D8F804300A93B8F8121098F800E0D8F880
:103D900008308DF83C9000FB02F24FF0000C4FF021
:103DA000FF3008AE8DF83DE0CDF824C00C920B93A7
:103DB000ADF838100D90B146B9E80F00DFF82CE3EC
:103DC0000296AEE80F0099E80F00AEE807007246D1
:103DD000182122F81C39E17194F85A1184F805C0B1
:103DE00081F0780383EA0313D8B2030983F0F60362
:103DF00043EA002383EAC0031BB283EA0310C0B284
:103E0000C3F3072383EA101343EA002383EAC003C2
:103E10001BB283F0C80080EA001C5FFA8CFCC3F37D
:103E2000072080EA1C1040EA0C2080EACC0000B297
:103E300080F0180383EA0313DBB2C0F3072080EAA3
:103E4000131040EA032080EAC30301F101091E2098
:103E50004FF0FE0C4FF0C80BE0700EF1020E217116
:103E600084F85A91238084F802C084F806B018467A
:103E700012F8011B414081EA0111C9B20B0983EA22
:103E8000102343EA012383EAC10109B288B27245D3
:103E90002080EDD181F0180181EA0111C9B20A092F
:103EA00082EA102383EA012383EAC1031BB29AB298
:103EB00089492280DBB2120A039104921E4684F8DB
:103EC000272084F826308E4601F5C17B04F12209B3
:103ED000DEF80000DEF80410DEF80820DEF80C3012
:103EE000DC46ACE80F000EF1100ECE45E346EFD1F4
:103EF000DEF80000CCF80000DFF8F4919DF81030F7
:103F000084F8A86184F8A931CB461BF8011F3868F2
:103F1000F5F73CFB714B5B45F7D1FAF79FFDDAF8FB
:103F20000030B8F80C20D8F804A0D8F808804FF476
:103F30007A7113F0140F01FB02F141F05D828E469D
:103F400094F85AB108908BF06A00654BDFF8A4C171
:103F5000B3F90420CDF824A080EA0010C0B2030910
:103F600083F0D50343EA002383EAC0031BB283EA4C
:103F70000310C0B2C3F3072383EA101343EA0023FC
:103F800083EAC0031BB28CFB020CD2174FF0000A6D
:103F9000CDF82880C2EBAC02DDF80880CDF830E027
:103FA00083F0C80C0B91ADF83A20ADF834A0ADF811
:103FB00036A0ADF838A08CEA0C1C5FFA8CFCC3F379
:103FC000072EB8E80F008EEA1C1E4EEA0C2E8EEA71
:103FD000CC0CDFF818E184F804B00FFA8CFCAEE8E2
:103FE0000F008CF0210398E8070083EA0313DBB28B
:103FF000CCF3072C8CEA131C4CEA03280BF1010CC0
:104000008EE8070088EAC30384F85AC14FF0210BF9
:104010004FF0FE084FF01C0CC8220EF10C0E84F875
:1040200005A084F807B084F8028084F803C0AEF1DC
:104030001C01A2711846238011F8012B424082EA2C
:104040000212D2B2130983EA102343EA022383EA5D
:10405000C20212B290B271452080EDD182F06802A6
:1040600082EA0212D2B24FEA121B8BEA102B8BEAC1
:10407000022B8BEAC20B0FFA8BFB1FFA8BF3DFF8D4
:1040800058E023805FFA8BFB1B0A1E4684F825301C
:1040900084F824B00EF5C17A04F12208DEF800009D
:1040A000DEF80410DEF80820DEF80C30D446ACE868
:1040B0000F000EF1100EC645E246EFD1BEF80030FB
:1040C000DFF83480ACF80030CA4684F8A6B184F832
:1040D000A76113E03D6D00201E200020C5210020B7
:1040E0006C6D002064A00020406D00202420002082
:1040F0009F21002067666666C32100201AF8011F11
:104100003868F5F743FAD045F8D194F85AA1E14A56
:10411000E14E84F804A08AF0EB0383EA0313D9B2DA
:104120000B0983F0C50343EA012383EAC1031BB2F1
:1041300083EA0310C0B2C3F3072181EA101141EAF8
:10414000002181EAC0010CCA09B281F0C80E8EEAD2
:104150000E1E5FFA8EFE4FF0000C0892C1F307218D
:10416000029A0993CDF828C081EA1E1343EA0E2370
:1041700007CA83EACE031BB283F0310E86E807003C
:104180008EEA0E1E5FFA8EFEC3F3072383EA1E1328
:1041900043EA0E2383EACE0394F808E0607AA27A19
:1041A000E17A84F805C01BB28EEA030E8EEA0E1E79
:1041B0005FFA8EFEC3F3072383EA1E1343EA0E233E
:1041C00083EACE031BB2584080EA0010C0B2C3F3AA
:1041D000072383EA101343EA002383EAC0031BB2D8
:1041E0005A4082EA0210C0B2C3F3072282EA1012D8
:1041F00042EA002282EAC00212B2514081EA011171
:10420000C9B2C2F3072383EA111343EA012383EA05
:10421000C10394F80CC094F80DE0A07BE17B227CF4
:1042200094F811801BB28CEA030C8CEA0C1C5FFA28
:104230008CFCC3F3072383EA1C1343EA0C2383EAB1
:10424000CC031BB28EEA030E8EEA0E1E5FFA8EFEC0
:10425000C3F3072383EA1E1343EA0E2383EACE0344
:104260001BB2584080EA0010C0B2C3F3072383EAB0
:10427000101343EA002383EAC0031BB2594081EACA
:104280000111C9B2C3F3072383EA111343EA0123DF
:1042900083EAC1031BB25A4082EA0212D2B2C3F3CC
:1042A000072383EA121343EA022383EAC2031BB201
:1042B00088EA030888EA08185FFA88F8C3F3072336
:1042C00083EA181343EA082383EAC803A17CE27C4B
:1042D0001BB2594081EA0111C9B2C3F3072383EA33
:1042E000111343EA012383EAC1031BB25A4082EA55
:1042F0000212D2B2C3F3072383EA121343EA022362
:1043000083EAC2031BB283F0270E8EEA0E12D2B2EA
:10431000C3F3072E8EEA121E4EEA022E8EEAC20E5A
:104320000AF101030FFA8EFE1FFA8EF24FF0310AE6
:10433000FE200C2184F85A31C8234FEA122C06F5CE
:10434000BE785FFA8EFE228084F807A0A070E1702C
:10435000A371039E84F814E084F815C07168B268F4
:10436000F3683068B6F810A0A8E80F0028F803AB8F
:1043700084F897C184F896E119F8011F3868F5F7B9
:1043800005F9C845F8D194F852C1BCF1000F40F0CE
:104390005685424B94F85A91B3F90010B3F90220B4
:1043A000B3F904309FED3E6A84F805C007EE103A79
:1043B0003C4B1B68089389F06A0383EA031306EEFB
:1043C000901AD9B20B0983F0D50343EA012383EA9B
:1043D000C1031BB283EA03115242C9B207EE902A0D
:1043E000C3F3072383EA111343EA0123F8EEE77AC4
:1043F000F8EEE66AB8EEC77A83EAC1031BB267EE4D
:10440000867A66EE866A27EE067A002083F0C80870
:10441000CDED0A7ACDED096A8DED0B7A0C900D90F9
:104420000E9088EA081E0DF1200A5FFA8EFEC3F393
:104430000728BAE80F0088EA1E1848EA0E2888EA1A
:10444000CE08DFF854E00FFA88F8AEE80F0088F0E5
:104450001E0C9AE807008CEA0C1C5FFA8CFCC8F36F
:10446000072383EA1C1343EA0C238EE8070083EA40
:10447000CC0CC8214FF0050A4FF01E08FE231C206B
:1044800009F10102A17184F852A184F80780A37098
:10449000E07009E0282E0020242000206C6D002010
:1044A00088C3E43AC4B80020AEF1100184F8049047
:1044B0000EF10C0EA4F800C084F85A2111F8013B4B
:1044C00083EA0C0383EA0313DBB21A0982EA1C2293
:1044D00042EA032282EAC3031BB21FFA83FC71453E
:1044E000A4F800C0EAD183F0270383EA0313DBB208
:1044F0001A0982EA1C2C8CEA032C8CEAC30C0FFAF2
:104500008CFC1FFA8CFADFF81094A4F800A05FFA74
:104510008CFC4FEA1A2A84F825A084F824C009F5F7
:10452000C17B04F12208D9F80000D9F80410D9F8A9
:104530000820D9F80C30DE46AEE80F0009F110096A
:10454000C145F346EFD1DFF8E483B9F80030AEF8A7
:10455000003008F1240984F8A6C184F8A7A118F84E
:10456000011F3868F5F712F8C145F8D194F853A146
:10457000BAF1000F40F05E84E04B1B68052284F81E
:1045800053219A0640F10185DD4ADFEDDE7A518A3A
:1045900007EE101AB8EEC77A13F0140F27EE277A39
:1045A00001F0E380D84BDFEDD76AD3ED007AF8EE67
:1045B000E77A67EEA67A94F85A91D44BD44AB3F9C5
:1045C0000410B2F90620DFF868E3D2488DED097ACD
:1045D00089F0220383EA03135FFA83FC4FEA1C137A
:1045E00083F0590343EA0C2383EACC03B2F5FA6F54
:1045F0001BB2A8BF4FF4FA6283EA031C5FFA8CFC7B
:10460000B2F57A7FC3F3072383EA1C13B8BF4FF4D4
:104610007A724FF0640843EA0C23A2F57A7208FB21
:1046200002F283EACC0C8EFB026E80FB01600FFA73
:104630008CFCC917D217C2EBAE12C1EBA0034FF02E
:10464000000B08A98CF0C80ECDED0A7AADF8322027
:10465000ADF83030CDF820B0CDF82CB088468EEAD9
:104660000E1E5FFA8EFE0291CCF3072CB8E80F0005
:104670008CEA1E1C4CEA0E2C8CEACE0EDFF8B4C27B
:10468000D8F8008084F80490ACE80F000FFA8EFE92
:104690008EF04A0383EA0313DBB2CEF3072181EAEB
:1046A0001311624641EA032109F1010981EAC303BA
:1046B000142042F810894FF0FE0E4FF04A080021F6
:1046C00084F85A914FF0C809E07023800CF1040C73
:1046D00084F8078084F802E0617184F80690184637
:1046E00012F8011B414081EA0111C9B20B0983EAAA
:1046F000102343EA012383EAC10109B288B262456B
:104700002080EDD181F0140181EA0111C9B24FEA94
:10471000111E8EEA102E8EEA012E8EEAC10E7E4BFD
:104720000FFA8EFE1FFA8EFC1E464FEA1C2B5FFA14
:104730008EFE84F81DB084F81CE059689A683068D1
:10474000DB68A4F800C006F5C17CACE80F00306956
:104750007169B6F818900396ACE8030004F2831868
:10476000ACF8009084F89FB1C14684F89EE104F251
:104770009F1B19F8011F3868F4F708FFCB45F8D1E3
:10478000664B674A1B781278013B12F00100DBB2DE
:1047900014BFC0214021172B03D8624A134493F859
:1047A00008A0614B1A8896071ABF002341F0100138
:1047B000012312F4027F18BF022312F0100F18BF5A
:1047C000062312F0200F18BF1023002840F029867E
:1047D0004FF0030994F85AE108938EF0460383EAF8
:1047E0000313DAB2130983F0920343EA022383EA44
:1047F000C2031BB283EA0310C0B2C3F3072282EAEA
:10480000101242EA002282EAC00212B282F0C80C00
:104810008CEA0C1C5FFA8CFCC2F3072282EA1C12A1
:1048200000238DF82790032042EA0C29029A8DF884
:1048300024A08DF825308DF826108DF8280007CAA1
:1048400089EACC0C0FFA8CFCDFF8E890E3718CEA73
:104850000C1AA9E803005FFA8AFACCF3072C8CEA59
:104860001A1C4CEA0A2181EACA0A94F808C089F89D
:1048700000200FFA8AFA8CEA0A0C8CEA0C1C5FFA08
:104880008CFCCAF3072282EA1C1242EA0C22607AEC
:10489000A17A94F80BA0637182EACC0212B2504064
:1048A00080EA001C5FFA8CFCC2F3072080EA1C102F
:1048B00040EA0C2080EACC0000B2414081EA0111BC
:1048C000C9B2C0F3072282EA111242EA012282EA47
:1048D000C10212B28AEA020A8AEA0A1A5FFA8AFA5C
:1048E000C2F3072282EA1A1242EA0A2294F80CC0A2
:1048F000607BA17B84F804E01EE000BF64A0002080
:10490000406D00200AD7233C646D00206C6D0020B0
:10491000CC540020676666661E200020FC7D0020C7
:104920007197002014080408BC6D00209F2100200E
:10493000D34D62102420002082EACA0212B28CEA0F
:10494000020C8CEA0C1C5FFA8CFCC2F3072282EA90
:104950001C1242EA0C2282EACC0212B2504080EAD7
:104960000010C0B2C2F3072282EA101242EA00220B
:1049700082EAC00212B2514081EA0111C9B2C2F307
:10498000072282EA111242EA012282EAC102E17B95
:1049900094F810A013B281EA030282EA0212D2B2A2
:1049A000C3F3072383EA121343EA022383EAC20311
:1049B0001BB28AEA030282EA0212D2B2C3F30723CD
:1049C00083EA121343EA022383EAC2031BB283F091
:1049D000320282EA0212D2B2C3F3072383EA12132D
:1049E00043EA022383EAC2031BB29AB24FF0FE0CE1
:1049F0000920C8210EF1010EDBB284F802C04FEA93
:104A0000122CE070A17184F85AE1228084F812C05F
:104A10006374039E30687168B268B6F80CB009F52B
:104A2000BA7EAEE8070009F5C2798EF802A0AEF8AA
:104A300000B084F894C184F8933118F8011F3868E5
:104A4000F4F7A4FDC145F8D1019BC4F84431FEF749
:104A500073BCDA4BDA491868F4F760FD0023237061
:104A6000FEF7E9BC94F89832D64AC4F8945202EBA7
:104A70008302126A42B310AD04F29F23D24E45F86E
:104A8000203D002104F2B1233180099380211523B8
:104A9000A52784F89E32284684F89D1284F89C72DB
:104AA000904728463188F5F77DFF089DC74804F5F3
:104AB00027716D1A152DA8BF15252A4629F086F9EC
:104AC000C34A94F898321570C24A013382FB03122C
:104AD000A2EBE37202EB42029B1A84F89832FEF7D3
:104AE0003BBCDFF828E3BC4ABC4BD4F82011DEF80D
:104AF00000001B8892F80BC0B94A401A4FF47A7133
:104B0000DFB201FB0CF11B0A9777177588424FF053
:104B10000007D37753759770177180F00C82B14BF3
:104B2000B14E1B68B149DFF8E89208688968DFF880
:104B3000E4E2DFF8E482DEF800E086FB036CDB17DA
:104B4000C3EB6C1303F5FA739BB293761B0AD3760F
:104B500089FB003AC01789FB0139CB17C0EBAA01CA
:104B600011770912DFF8B4C251779F499CF800C051
:104B7000C3EBA9030EF5EA4081FB0E1982F8203041
:104B80004FEAEE711B12C1EB6911303082F821300F
:104B9000974B98F8009083F81A90001278310EF134
:104BA000300E1CF0020F82F8230082F8241082F8E5
:104BB00022E000F0BD81D8F804C08E49D8F808A0E2
:104BC000DFF85CB28C4A81FB0C604FEAEC7E81FB23
:104BD0000A61CEEBA05E4FEAEA70C0EBA1510BFB7D
:104BE0000EC00BFB01AB0BEB4B0B4FEA4B0600EB84
:104BF00040000196400082FB007B01EB810182FBBB
:104C00000672019E92140EEB8E0E01EB81014FEAAB
:104C1000AB4B04920EEB8E07B8F8122005914FEAC9
:104C2000E67EC117B8F80C80744E03974FEADC7C1F
:104C300083F809C0ABEB010C06FB1C0108F5FA7800
:104C4000049E03981FFA88F70297A6EB0E086B4F95
:104C5000019EDFF8D0E1B9F1050F4FFA8CF909EBAD
:104C60008009404607FB1868059EDFF8BCC140B2CA
:104C700000EB860002EBC2025B4E4FEA82024FEA73
:104C8000DA7A8CFB02BC83F80EA086FB017A86FBE5
:104C900008B74FEAE27B9DF808205A75CBEBAC12BF
:104CA0000192029ABEF80060DFF880E14FEAE878EE
:104CB0004FEAE1711FFA89F980B2C8EB6717C1EBBF
:104CC0006A114FEA1228019A83F80A904FEA102BD2
:104CD0004FEA192C4FEA212A4FEA272983F810B00E
:104CE000BEF800E083F80BC0D873C2F3072C4FEA7C
:104CF000162034BF4FF0320B4FF0330B197383F88B
:104D00000DA05F7483F8129083F816809DF804203C
:104D1000DA7183F808C0DE74187583F81BB083F865
:104D20001CE0C4F81C51FEF770BA354F38680368B0
:104D30005B69984700283EF4EDAA386803680121B2
:104D40009B6998470222002388F800202370FEF711
:104D5000E1BA94F8381194F83931D8F800004A1CB7
:104D6000013384F8382184F83931F4F70FFCFEF769
:104D7000B0BAF9F773FE234B1A6840F6B833801ABD
:104D8000984200F2EE80204F3B793A2B00F0CB8224
:104D900000232370FEF7BEBAC4F82C3184F8243106
:104DA000DFF88C801AF090FC94F83031FEF776BA78
:104DB000013A84F84B21FEF7B7BF00BFDC6E00203C
:104DC000F86D002014080408A86B0020EC290020CE
:104DD000012A00205655555530A800202CA8002047
:104DE000586E0020646D00201F85EB51AC6B0020D5
:104DF000846E00206BCA5F6B83DE1B4340420F0052
:104E0000D02C00201866002000660020C4B80020C6
:104E100067666666686D0020406D00203D6D00206D
:104E2000806967FF302E0020D34D6210322E0020A3
:104E3000C86D00200AF1FF3A84F853A104E60CF192
:104E4000FF3C84F852C1FFF791BBB94A1288D705DD
:104E500015D4D00600F1D882910600F19A83570646
:104E600000F18A84100700F18B84D10700F1AE8431
:104E700012F0020F0CBF4FF004084FF00C08AD49C0
:104E8000AD4A0F78D27807F001070AB147F0020760
:104E90005320019325F0D4FEA84A128802EB820227
:104EA00002EB8202900080B225F0AEFE002025F0D9
:104EB000ABFEA34AA3491288D9F80000C2EBC21284
:104EC000520081FB02311144D217C2EB61225FFA1A
:104ED00082FA5146F4F75AFB9BF80020D9F80000FB
:104EE0008AEA020248EA070700218BF80020F4F75B
:104EF0004DFB3946D9F80000F4F748FB9BF8002039
:104F0000D9F800007A40D2B211468BF80020F4F7AD
:104F10003DFB94F84071019BFEF773BC013B84F8A4
:104F20004A31FEF7C8BD013B84F84E31FFF72BBA7A
:104F30002D22DA76F5E6844BDEF800101B78C4F8F3
:104F40002011013B012B3FF6EAAD102102239170A5
:104F50001371E4E51AF0A8FB7C4B01221A70FEF7EE
:104F60006FB97B4AB2F8423100210133A2F84231D5
:104F70002170FEF7CFB901468046864683460290EF
:104F8000814603900246FEF7CDBD9FED727A13F085
:104F9000140F08BFF0EE477A7FF404ABFFF70BBBAA
:104FA0006D4B664909930DF14008A3F1210048F8C3
:104FB000200D4FF0080E4FF000090A2003F822ECF4
:104FC00003F8230C03F8249C40460988F5F7C4FC39
:104FD000624B63491B6881FB0321DB17C3EBA10113
:104FE000404689B2F5F7B8FC5E4BB3F806A015F061
:104FF000A5FE089B5A1C089283F80090089B4FEA74
:105000001A22591C08911A70089B5A1C089283F89E
:1050100000A0089B5A1C0892187040461AF002FC27
:10502000FEF71EBADFF850919FED4F8AB9F90230B2
:10503000494A099207EE903AF8EEE77A0DF14008F6
:1050400067EE887AA2F12403FDEEE77AA2F121014E
:10505000002048F8201D02F8240C0822CDED017A2A
:105060005A701E229A70BDF804104046F5F774FC81
:10507000B9F9003007EE903AF8EEE77A404667EE6D
:10508000887AFDEEE77ACDED017ABDF80410F5F7E8
:1050900063FCB9F9043007EE903AF8EEE77A40463F
:1050A00067EE887AFDEEE77ACDED017ABDF804105F
:1050B000F5F752FC40461AF0B5FBFEF7CEB92B4A85
:1050C000254B12680993A3F12408002103F8241C3E
:1050D0002123D10088F8023040F1008224490326C0
:1050E000134B1B885A0500F1F681D80700F1F582B1
:1050F00003F002031F4A002B1CBF03261146DFF8F2
:105100007C903246484628F061FE06EB090310A861
:105110000133A9F1020140F8203D00225B1A06F894
:10512000092088F801301AF07DFBFEF79CB900BF1A
:10513000BC6D002071970020682D00202CA8002055
:10514000622D002003082080652D002035000020FE
:105150001C20002000000000F86D0020AC6B002037
:1051600067666666586D002058A08B41107C002051
:1051700064360408743604086C6D0020D76D002076
:1051800002201AF0E5FAFF2025F008FC0278FF2A39
:1051900000F0E98290F901004FEAE0785FFA88F8C0
:1051A000C0B21AF0ABFA40461AF0A8FA03201AF07F
:1051B000CFFAFF2025F0F2FB0278FF2A00F0CF8221
:1051C000B0F908805FFA88F0C8F30728DFF898A3E1
:1051D0001AF094FA40461AF091FA9AF80420002A3C
:1051E00040F0E781D14A1268900640F11081DFF863
:1051F0007CA3DFF87C839AF80020910700F170828D
:105200004FF0000B01201AF0A3FA38461AF076FA94
:1052100058461AF073FA09201AF09AFA00201AF088
:105220006DFA00201AF06AFAB8F8161098F80030F3
:10523000B1F5967F0AD994F8142102F00F02072ADB
:1052400004D842F20F738B4228BF0B46DFF824B319
:10525000019305201AF07CFA9BF80820019B002A94
:1052600000F0A482203B07EE903A9FEDB17AF8EE71
:10527000E77AF6EE006A67EE877ABEEE007AF5EE20
:10528000C07AF1EE10FA58BFB0EE667A77EE877A00
:10529000FDEEE77ACDED017ABDF904300193D8B285
:1052A0001AF02CFA019BC3F307201AF027FA9AF898
:1052B0000020002306930793930700F16D8194F873
:1052C0001831012B00F06881BBF90030DFED996ADD
:1052D00007EE103ABBF9023007EE903AB8EEC77A03
:1052E000F8EEE77A27EE267A67EEA67ABDEEC77A61
:1052F000FDEEE77A08A88DED087ACDED097A1AF06F
:1053000039FA5E21D9F80000F4F740F994F8142135
:10531000FEF790B9884A1068FEF759BAC4F82851C8
:105320001F70FDF78DBFBB78DBB103F1FF3C5FFA67
:105330008CFC0CF1010CBC44BE4600221EF8013B63
:10534000534083EA0313DBB2120AD90042EA032274
:10535000F44581EA131382EA0302EFD1002A7FF4B5
:1053600017AD764BDFF810E21968734BD1F830C0F7
:105370001B68734ADFF8EC81CEF83830714BB8F80F
:105380000080CEF86800B3F8423110689268CEF819
:105390001880CEF82800CEF84820CEF85830BCF15E
:1053A000000F00F01782DCF80430886C83423BBFAA
:1053B000CA681B1A1B1A9B18002B7DF4A4AF0B683C
:1053C000DFF8B8819B690846022198470423F878E2
:1053D00088F8003028F074FB03232370FDF795BF95
:1053E0000127FEF7C9B90221D8F80000F4F7B6F892
:1053F00094F83031FDF752BF4F4B1B6803EB83032A
:105400004FEA430EFEF79CBD4FF0340837E54E4B94
:1054100093E8030008AB83E8030018461AF0AAF9E2
:105420006FE74A4AD278002A0CBF4FF004094FF0C8
:105430000509FFF7CFB9DFF800B1DFF844A110206C
:105440001AF086F9DBF800208AFB0238D217C2EB8B
:1054500068185FFA88F01AF051F9C8F307201AF0BB
:105460004DF921201AF074F9DBF800108AFB013A9B
:10547000CA17C2EB6A12642000FB1212002AD8BFBE
:10548000524212B2D0B21AF039F900201AF036F9AD
:10549000FEF7A5B80122D8F800001A70F4F76AF8F0
:1054A0000746D8F80000F4F765F87F067DF4C8AE2B
:1054B0008A2800F069818E287DF4C2AE94F82431E8
:1054C000002B7DF4DAAE224BC4F82C312D2384F866
:1054D0003031FDF7BCBE03261E4910E61E4B1F4AA5
:1054E0001B681F4903F48003002B16BF11460426D6
:1054F0000326F5E54FF00109FEF734BC19495A7946
:105500000B8803EB830303EB83034FEA83091FFA42
:1055100089F9002A00F09A81094B1B681BB202939B
:1055200015F00CFC029B40B2FEF7F2B964A000201B
:10553000E4380E3F0050C347646D0020D02C00209B
:10554000AC6B00201C20002014080408682D0020EB
:10555000586E0020683604081836002064360408A7
:105560005C3604082CA80020586D00203D6D0020FA
:10557000406D002030A8002060020020D1020020F1
:105580001F85EB5111469046964693460292FEF7D0
:10559000C9BA4FF0240872E40121D8F80420D8F8E1
:1055A000083084F8181106A8069207931AF0E2F85A
:1055B000A7E6DFF8C0B29BF80020002A3FF412AE45
:1055C000A449B4F81681088802914FEA08184FF0F0
:1055D000640E1FFA88F80EFB00204FEA420EB0FB63
:1055E000FEF048EA00281FFA88F8C0F3032048EAD2
:1055F0000008062001921AF0ABF85FFA88F01AF062
:105600007DF84FEA18201AF079F8B4F81601019ADB
:10561000914B0299013080B290FBF2FC02FB1C021C
:10562000587AB1F80080A4F81621012800F0E4802F
:105630005A7B6E2303FB08F8152198FBF1F8002A2A
:1056400040F0D3803A201AF083F81FFA88F84FF020
:10565000640BB8FBFBF291B2C8B2029201911AF04E
:105660004DF80199080A1AF049F83B201AF070F831
:10567000029A0BFB128080B20A22053090FBF2F0F6
:10568000C0B21AF03BF800201AF038F8DFF8E0B1A9
:1056900028201AF05DF84FF00A08DBF8002092FB92
:1056A000F8F85FFA88F01AF029F8C8F307201AF022
:1056B00025F804201AF04CF8BAF80620002A7DD10B
:1056C000DBF8082082F310085FFA88F01AF016F869
:1056D000C8F307201AF012F884E5604904260EE5A5
:1056E00011201AF035F8B8F812205D494FF4F36B29
:1056F0000BFB02F281FB0231D217C2EB6132D0B256
:10570000019219F0FBFF019AC2F3072019F0F6FF8E
:1057100019201AF01DF8B8F8122052490BFB02F2BA
:1057200081FB0230D217C2EB601281FB0230D1172D
:10573000C1EB6011642000FB1120C0B219F0DEFF44
:10574000002019F0DBFF9AF80020B8F80CB092079F
:105750007FF556AD5FFA8BF74FEA1B2B52E54FF002
:105760000008404632E540461BE5938907EE903A33
:10577000F8EE677AFEF71FBF4FF01008FFF77FBB08
:105780004FF02008FFF77BBB374B1B6898067DF571
:1057900057AD94F82431002B7DF46FAD334BC4F832
:1057A0002C312D2384F83031FDF751BDD8B219F0DA
:1057B000A5FF019B180A19F0A1FF78E515F0BEFAC4
:1057C00019F09CFF002019F099FF0BE54FF0080835
:1057D000FFF755BBCA690B6A9A423CBFC8681218EA
:1057E000D31AE9E51146FEF79DB91FFA88F89BF830
:1057F000002098FBF2F825E7392019F0A9FF5FFA9D
:1058000088F019F07BFF4FEA182019F077FF3DE789
:10581000114690469646934602929146FEF782B90B
:10582000134B9146B3F900306420FEF771B811466E
:105830009046FEF777B9114690469646FEF772B944
:105840001146904696469346FEF76CB94FF0FF33EB
:1058500064E600BF2CA8002030A800206C360408A5
:1058600089B5F8141F85EB5164A00020846E0020D8
:10587000AC6B00203EA800202DE9F04F2DED028BEF
:10588000C74B1B7891B0072B089001F0F6810023DD
:105890000793C44B1B6805935D0500F1DE86C24B80
:1058A000D3F8008018F0080F40F07586BF4BC04D4C
:1058B000B3F800B0DFF81CA30693BE4BBE491E68C8
:1058C000B1F906907289914580F2A484BB4B4FF0E8
:1058D0007E521A60BA4F9AF90420B1F900C03C8B8D
:1058E0009AF800009AF801E0002AACEB040314BF18
:1058F00001224FF0FF32002B40F3EE84B3F5FA7F24
:10590000C0F2F0844FF4FA731B1A07EE903AF8EEE7
:10591000E77AA445C5ED007A03DAF1EE677AC5EDC2
:10592000007AB1F902C0ACEB0403002B40F3E18430
:10593000B3F5FA7FC0F2E3844FF4FA731B1A07EE53
:10594000903AF8EEE77AA445C5ED017A03DAF1EE74
:10595000677AC5ED017AB1F90430191B0029D8BF67
:10596000E11AB1F5FA7F80F24F847145D8BF4FF04C
:10597000000E00F34B8402FB0EF207EE902AF8EEC5
:10598000E77AA342059BC5ED027ABCBFF1EE677AC8
:10599000C5ED027A13F48053049300F0ED80B9F55D
:1059A000FA6F4A46A8BF4FF4FA62B2F57A7FB8BFE1
:1059B0004FF47A72A2F57A728249DFF81CE281FB19
:1059C0000230D317C3EB6013581C6FF0630C3EF921
:1059D00010003EF913E00CFB0323A0EB0E0003FBC9
:1059E00000F381FB0321DB17C3EB61139E440FFA25
:1059F0008EFE07EE90EA049BB8EEE78A85ED038AF7
:105A0000002B40F071861BF0400F40F034856E4C47
:105A100018F0140F03D01BF4027F40F0ED866B4B9F
:105A20001B781BB17B8B4B4580F2078594F82630A1
:105A30001BB11BF0030F41F0098094F82C20FB7F71
:105A4000002A40F07E86B97F002900F0C980022933
:105A500000F0CD87032940F0B28797F82010C1EB02
:105A6000411001EB8001C90089B20233DBB2002A88
:105A700000F0AC87002900F0A98755480068B1FB09
:105A8000F0F10FFA81F9A4F85C90ABB307EE909AAD
:105A9000F8EEE77AF7EE006A86EEA77A012BD5EDED
:105AA000007AD4ED1C6A77EEE67A67EE877AC4ED69
:105AB000187A21D0D5ED017AD4ED1D6A77EEE67A19
:105AC000022B67EE877AC4ED197A15D0D5ED027AEC
:105AD000D4ED1E6A77EEE67A032B67EE877AC4ED83
:105AE0001A7A09D0D5ED037AD4ED1F6A77EEE67AFB
:105AF00067EE877AC4ED1B7A29490978092901F0F4
:105B0000B385B9F1000F71DD93B394ED1C7AD4ED38
:105B1000187A77EE877A012BC4ED1C7AC5ED007AEE
:105B200021D094ED1D7AD4ED197A77EE877A022B85
:105B3000C4ED1D7AC5ED017A15D094ED1E7AD4ED31
:105B40001A7A77EE877A032BC4ED1E7AC5ED027AB6
:105B500009D0D4ED1F7A94ED1B7A77EE877AC4EDE5
:105B60001F7AC5ED037A013B022BB8BF0223DBB2DB
:105B7000002A18BF02233AE0798B8945C0F26C8471
:105B8000B9F5FA6FD4BFC1EB0903C1F5FA634FF45D
:105B90007A7202FB03F2C1F5FA61B2FBF1F20BE794
:105BA00055A700201836002064A00020BC6D0020FE
:105BB00040A80020C46D0020CC540020A824002060
:105BC000E83500201F85EB51D4220020040200207C
:105BD000F87D0020C47D002040BC00200AD7233C73
:105BE000A4F85C108946002A00F072810223327802
:105BF0005FED066AB17807EE902AF8EEE77AB0EE2C
:105C0000007A67EEA67ADB4AF4EEC77AF1EE10FA74
:105C1000107840F3BC84DFEDD86A37EEC77AB0EE77
:105C2000676AA7EE266AF0EE466A95ED007A9FED68
:105C3000D36ADFF870E3DFF870C327EE066AF0EE90
:105C4000C65ACEED005A8CED006A99B107EE101AD3
:105C5000B8EEC75A9FEDCA7A66EE064A25EE075A95
:105C6000B7EE007A37EE457A64EEA54AA5EE247ABF
:105C700026EE076A9FEDC37A727926EE877A27EEC1
:105C8000067AAAB1DFEDBE6A9FEDBF6A65EEA65A3D
:105C900006EE902AF8EEE66A66EEA56AF4EEC66AAB
:105CA000F1EE10FA40F35F869FEDB86A27EE067AB0
:105CB0000C289FEDB78ADFEDB76ADFF8F08200F0BD
:105CC0002D86B4EEC87AF1EE10FA98BFB0EE478A8E
:105CD000B4EEE68AF1EE10FAB8BFB0EE668A88ED4F
:105CE000008A002B00F0E680B0EE007AF4EEC77A6E
:105CF000F1EE10FA05DD37EEC77ADFED9F6AE7EEC9
:105D0000267A95ED017ADFED9D6A27EE267AF0EE90
:105D1000C75A8CED017ACEED015A99B106EE901A70
:105D20009FED976AF8EEE66A27EE075A66EE866AF6
:105D3000B7EE006A36EE666A25EE255AA5EE266AAB
:105D400027EE067ADFED8F6AB27967EEA67A67EE04
:105D5000877AFAB107EE102AB8EEC77A9FED886A03
:105D6000DFED896A27EE257A27EE067AB4EEE67A29
:105D7000F1EE10FA00F3F385B5EEC07AF1EE10FA09
:105D800001F1DF80B7EE006A36EE477AC6EE076AA9
:105D900067EEA67A0C2800F0A285DFED7D6A9FED04
:105DA0007D7AF4EEE67AF1EE10FA88BFF0EE667ACC
:105DB000F4EEC77AF1EE10FAB8BFF0EE477A012B95
:105DC000C8ED017A76DD7378DFED6D6A07EE903A03
:105DD000F8EEE77AB0EE007A67EEA67A737AF4EE20
:105DE000C77AF1EE10FA05DD37EEC77ADFED626AA9
:105DF000E7EE267A95ED027ADFED606A27EE267AE5
:105E0000F0EEC75A8CED027ACEED025A9BB106EE47
:105E1000903A9FED5B6AF8EEE66A27EE075A66EE67
:105E2000866AB7EE006A36EE666A25EE255AA6EE59
:105E3000856A27EE067ADFED536AF37967EEA67A74
:105E400067EE877AFBB107EE103AB8EEC77A9FED9E
:105E50004C6ADFED4D6A27EE257A27EE067AB4EE1E
:105E6000E67AF1EE10FA00F37685B5EEC07AF1EE3F
:105E700010FA01F16280B7EE006A36EE477AC6EE9C
:105E8000076A67EEA67A0C2800F02185DFED406AEC
:105E90009FED407AF4EEE67AF1EE10FA88BFF0EE6C
:105EA000667AF4EEC77AF1EE10FAB8BFF0EE477AF0
:105EB000C8ED027A092800F0008597F82150002DDE
:105EC00040F0B584344BD3F80080002384F82C30A4
:105ED00018F0200F06D0069B1B8803F03003002B20
:105EE00040F03C822D4D2E4F95F82420DFF8C080E5
:105EF000DFF8C0A0531E082B00F20781DFE813F083
:105F000020019E01A90005015C000900A001050116
:105F1000B30198F80030002B40F02D852B68297ACA
:105F20004FF4807203EB0121002025F0FBFD2B7A5A
:105F30000133DBB2022B2B7240F05581002025F09B
:105F400031FE002025F02EFEFF2025F02BFE00F074
:105F50001F00052801F03C8422F00CF9EE68002EA9
:105F600000F0468400222B6969680120B04795F84B
:105F70002420BFE755A70020D7A368416F12033B39
:105F80000AD7233C00004843A4707D3F0000C8426C
:105F900000C0F94400C0F9C464A0002018530020D8
:105FA000C4B80020D8240020CC240020B024002035
:105FB000442D0020706002404FF40071286810F0FA
:105FC00081FE012800F01985C0F02E86022840F0DD
:105FD0000A8122F007F922F0CDF8EE68002E00F0D9
:105FE0000784002210462B696968B04795F8242081
:105FF00080E71021CD4810F065FE8346002840F070
:10600000F08001217F2014F01FFA0128814640F022
:10601000E8805846022114F017FA002801F0A982FE
:10602000012840F0DE8016213A2014F00DFA431CBE
:106030009B02EB6322F0D6F83068F3F71BFD0021DA
:106040000A2022F067F8002840F07386032385F8C1
:10605000243010210CA810F035FE002840F0C38039
:106060009DF83A209DF839009DF83C109DF83D3090
:106070009DF83B60120442EA00620A431B019DF84E
:106080003E109DF83100DBB243EA111342EA0622CA
:1060900003F5FA636A632B879DF832209DF8383048
:1060A00042EA002201F00F01180903F00F0385F8FE
:1060B0003A106A859DF830109DF8332085F832300B
:1060C0009DF8343085F8281085F82C209DF835107F
:1060D0009DF8362085F82D309DF8373085F8303022
:1060E00085F8310085F82E1085F82F2022F07AF8F7
:1060F000AB7E002B00F00A818D4825F0C7FD002300
:1061000004222B6285F824200323DBB2022B70D9F2
:10611000042A00F0BB80082A00F0B880854B1B7869
:1061200023B9854EB378002B40F09285834B1B78C2
:10613000072B00F0148511B0BDEC028BBDE8F08F89
:106140007F4E3068F3F796FC0021084621F0E2FF0D
:10615000814622F047F8B9F1010F44D130684FF081
:10616000000B85F819B0F3F785FC40F2AB1108205D
:1061700021F0D0FF052800F0A584012800F0BC859F
:1061800022F030F86B7E002B01F03683022385F875
:1061900024303068F3F76EFC6B7E022B14BF4FF097
:1061A00000094FF080490021372021F0B3FF494614
:1061B000292021F0AFFF814622F014F8B9F1000F39
:1061C00011D16B7E022B00F0A48585F81A903068FF
:1061D000F3F750FC0021092021F09CFF00283FF438
:1061E00008AF21F0FFFF95F82420531EDBB2022BED
:1061F0008ED8544B69691B685B1AC82B8BD921F068
:10620000B9FF95F8242083E74FF4FA71A1EB0E0E45
:10621000FFF7B1BBB9F5FA6FC0F22181337AC3F150
:10622000640307EE903A9FED487A484BF8EEE77A20
:1062300067EE877AC3ED007AFFF74CBB404EA8E7C4
:106240000826FF2025F0AEFCFF2800F09384013ED5
:10625000F7D16B693A68FA339342C4D221F08AFFCE
:1062600095F8242046E6FF2025F09CFCFF284FF0FF
:10627000080606D0013EECD0FF2025F093FCFF2855
:10628000F8D121F0AFFF042385F82430304D10F011
:1062900079FB6B78022B00F0F584032B7FF43EAF83
:1062A00041F2B813EB5C002B41F0848141F2A4036E
:1062B000EB5C002B41F0798141F2E803EB5C002BB1
:1062C00041F07D8141F22C13EB5C002B3FF426AFB3
:1062D000204825F09FFA21E7A4EB0C03B3F5FA7FE1
:1062E000BFF610AB9842FFF60FABDFED1B7AFFF75E
:1062F00010BBA4EB0C03B3F5FA7FBFF61DAB9842BD
:10630000FFF61CABDFED147AFFF71DBB0C4E3068B7
:10631000F3F7B0FB4FF40071102021F0FBFE0646AE
:1063200021F060FF002E3FF4E7AE97E758530020BE
:1063300000380040F62700200188002055A70020E3
:10634000402D0020C4B800200AD7233CA8240020F8
:10635000903E0020BC4F002000000000C54B1B7881
:10636000D8077FF5BFADC44BC44AB3F90430DFEDA5
:10637000C47A82FB0312DB17C3EBA2031BB208EE45
:10638000103AB8EEC88A28EE278AB0EE480AF4F729
:10639000D3FDF0EE408AB0EE480AF4F753FDB94B56
:1063A000D878002800F0F285B749B4F98A20B1F90D
:1063B000023044F250659B1AAB4241F31F81A3F5B2
:1063C0000C43A03B45429D4201F315818342A8BF87
:1063D0000346B1F90010B4F9886013448A1B44F2F3
:1063E00050611BB28A42A4F88A3041F30F81A2F5B2
:1063F0000C42A03A954203DC9042A8BF10460546E5
:10640000721912B207EE902A07EE103AF8EEE77A08
:10641000F8EEC76A27EEE87A60EE277AA0EE267AD1
:106420009A49A4F88820E8EEA67ADFED996A27EE6B
:10643000267A67EEA67A00F0C5BD964B1B78012B35
:1064400000F08283192B00F07F830E2B3FF4EEAA1D
:10645000082B3FF4EBAA7CE31A46FFF79CBB307A8B
:10646000A9EB020303FB00F3C2F5FA6293FBF2F31C
:10647000C3F16403D5E6804B8049B3F90430864C00
:10648000DFED7F6A22889FED857A81FB0301DB17B0
:10649000C3EBA1039B1A1BB207EE903AF8EEE77A22
:1064A00067EEA67A77EE876ABDEEE66A16EE103AD8
:1064B0002033402B40F27183DFED796ABDEEE77A3D
:1064C00017EE103A2033402B00F264839FED757A6B
:1064D000F4EEC77AF1EE10FA41F38980DFED725ADB
:1064E0009FED726A01E0F0EE477AF4EEC67AF1EEC3
:1064F00010FA37EEE57AF6DCDFED6D7AB4EEE77A86
:10650000F1EE10FA41F16F80DFED675A9FED696A95
:1065100001E0B0EE677AB4EEC67AF1EE10FA77EEEB
:10652000257AF6D49FED5D7AF4EEC77AF1EE10FA93
:1065300000F3C3829FED607AF4EEC77AF1EE10FAB1
:1065400044BF9FED5B7A77EE677A67EEA75A9FEDBF
:106550005B5A9FED5B6A9FED5B7AA5EE856A27EE3D
:10656000A55AA5EE867AE5EE077A95ED016AD5ED96
:10657000005A27EEC67A65EEA77AA5EEA67AE6EE71
:10658000267A85ED007AC5ED017AFFF741BAF0EE83
:10659000676AFFF74ABB4C4D4C4BD5ED027A069328
:1065A000B2EE0E7AF0EEE76AF4EEC76AF1EE10FA98
:1065B000B3F800B0304B42D51BF0040F3FD0B3F915
:1065C00004302E4A4249DFF81CA1098882FB0302ED
:1065D000DB17C3EBA2035B1A9BB21AB212F1B30F23
:1065E000BCBF03F5B4731AB2B32AC8BFA2F5B47323
:1065F0002049C8BF1AB29AF804300978002B4FF628
:10660000FF7318BF01230C077FF557A931490968AB
:1066100012FB03F3097E304A9BB211FB03F382FBAA
:1066200003121A44DB17C3EB221307EE103AB8EE3D
:10663000C77A77EEC77AC5ED027AFFF73EB9B3F9AC
:1066400004300E49224ADFF89CA081FB0301DB17CE
:10665000C3EBA1031380FFF730B920488368002BF8
:106660003FF41DA900F1440198471D4B1B68059399
:10667000FFF715B93D6D00206C6D002067666666FA
:1066800035FA8E3C802E0020DC2E0020C82400200D
:10669000CDCCCC3DFC7D0020D4220020DB0FC93FB7
:1066A00000000000DB0F4940DB0FC940E4CB16417E
:1066B000DB0F49C0E4CB16C1DB0FC9BF92E741B97C
:1066C0009730083C15A82ABE40A80020BC6D0020C9
:1066D000FC2E0020C06D0020898888882898002022
:1066E00018360020C47D00201D21C848F4F7FCFCAA
:1066F00000283FF488A9C64BDB78002B7FF483A9E0
:10670000DFEDC47AC44938EE678AC4F5FA62FDEE5B
:10671000C87A12B2CDED097ABDF924301B0381FB92
:106720000301DB17C3EBA11302FB03F343F30F33A6
:10673000234407EE903AB8EEE78A85ED038AFFF727
:1067400062B9B649B148D1F8EC10006844F6206E41
:106750007145A8BF7146B1F57A7FB8BF4FF47A7121
:1067600089B2C006E18540F1B1810498002840F06B
:10677000EC83AB48D0F800A0BAF936B0DFF898E265
:10678000206BD5ED037AAEFB01E14FEA911E642147
:1067900091FBFEF11429BDEEE77A04EB400CA8BF93
:1067A000142101308842206317EE109AA4BF002004
:1067B000206304EB4000ACF83490B0F9341007EEDD
:1067C000101AB8EEC77A77EEC77AFDEEE77ACDED0C
:1067D000047ABDF9100080EAE071A1EBE07159453F
:1067E00000F3F2868F494FF07E500860FFF72BB917
:1067F00095F82420FFF77EBB8B4B1B7813F010031A
:1068000000F074812279A36895ED017A002A0CBF0B
:1068100001224FF0FF3203FB02F307EE903AF8EE4D
:10682000E77A77EE877AC5ED017AFFF7F8B81E218F
:106830007648F4F759FC00283FF444AB069B1B88CC
:106840005E063FF53FAB94F88030AB4240F02E87B8
:10685000764BD4ED217AD3ED006A98ED025ADFED44
:10686000745A9FED746A27EEC57A68EE277AA8EE0F
:10687000267AE5EE267AB4EEE57AF1EE10FA88BFD4
:10688000B0EE657AB4EEC67AF1EE10FAF4EEE57A7F
:10689000B8BFB0EE467AF1EE10FA88BFF0EE657A36
:1068A000F4EEC67AF1EE10FAB8BFF0EE467A88ED53
:1068B000007AC8ED027AFFF705BBFDEEC87A5E4AA2
:1068C00017EE903AA2F80490D380FFF7F6BABDEE27
:1068D000E77A594B17EE102A9A80FFF7D7BA9FED47
:1068E000547ADFED546A5449F4EEC77AF1EE10FAA7
:1068F00098BFB0EE677AFDEEE77AB4EEE67AF1EE95
:1069000010FA17EE902AB8BFB0EE667A012B88ED28
:10691000017A4A803FF757AAFFF7CFBAB4EEC87A98
:10692000F1EE10FA98BFB0EE478ABDEEC77AB4EE2A
:10693000E68ADFF804A1F1EE10FA17EE102AB8BFCC
:10694000B0EE668A88ED008AAAF80020002B7FF45A
:10695000CBA9FFF7B2BADFED396AFFF792BADFEDE4
:10696000376AFFF715BAF7EE005A75EEE66A85EE5C
:10697000A66AFFF79BB9324B596889067FF5CBAB06
:106980002022DA60DAF800202E4B22F00102CAF849
:1069900000201A89D20700F19F801EF03FF90028DD
:1069A000FBD1284A938823F002031B041B0C93801D
:1069B00098F80030002B7FF4C1AAFFF7AFBA224944
:1069C00002334988DBB2002A7FF454A8B4F85C9003
:1069D00009F1FF390FFA89F9B9F1000FA4F85C90B9
:1069E0003FF792A8002A7FF401A9FFF771BAE18D61
:1069F00001F57A7189B2FFF738B86B693A68643388
:106A00009342FFF4E6AAFFF7EEBB00BF107C002024
:106A1000682D002000007A44D34D62103C03002012
:106A2000C06D00203C0000203D6D0020380000209B
:106A300000C0F94400C0F9C458A700200000C842B3
:106A400000600240003800405C280020C74ADFEDAB
:106A5000C87A92ED080A0993B4EEE70AF1EE10FA4B
:106A600040F2618227F0BCFBD4ED0A7A20EE270ABF
:106A700027F020FBB0F5617F099B00F36E8207EEE3
:106A8000900AF8EEE76ADFEDBB7A66EEA76A07EEDA
:106A9000903AB8EEE77AFDEEE67A17EE903A2033B8
:106AA000402B40F2AF869FEDB40A27F003FB00B203
:106AB00007EE900AB8EEE77A37E29FEDB07A77EE0C
:106AC000677A42E585F81990FFF75ABB0598C00030
:106AD0003FF54BAEFEF7B7BF9A891A89D207FBD4B0
:106AE0001EF09CF800287FF458AF5AE79AF803206C
:106AF000002A40F07382B4F90CE09AF80210A9EB76
:106B00000E0383EAE370A0EBE370884240F3A085B4
:106B100003EBD37301225B10E36184F8202022751C
:106B2000A3689E44BEF5FA6FA8BF4FF4FA6EBEF597
:106B30007A7FB8BF4FF47A7E07EE90EAF8EEE77AF4
:106B4000C5ED037AFEF76BBF8D4B9B7B002B7EF46C
:106B50006DAF8C4A0023AB609360FEF767BFF7F719
:106B60007DFF079A884B801A988011B0BDEC028B8C
:106B7000BDE8F08F2B6A0022012B2A7641F2D480E7
:106B8000EA69013B01322B620823EA6185F824306F
:106B9000FFF77CBBDFED787AE7E4F4EEC77AF1EE3D
:106BA00010FA40F30D86DFED795A9FED796A01E026
:106BB000F0EE476AF4EEC66AF1EE10FA36EEE57AC8
:106BC000F6DCDFED746AB4EEE67AF1EE10FA40F12D
:106BD000FB85DFED6E5A9FED706A01E0B0EE667ADC
:106BE000B4EEC67AF1EE10FA77EE256AF6D49FED90
:106BF0006B7AF4EEC76AF1EE10FA40F3AB809FEDCA
:106C00005F7A77EE666A66EEA65A9FED655A9FED4B
:106C1000656A9FED657AA5EE856A26EEA55AA5EE12
:106C2000867AE5EE076A49E421F0DCFAEE6804238F
:106C3000002085F824302876002E3FF427AB2B69FE
:106C40002A686968B04795F82420531EFFF7CEBA2A
:106C5000564F3A78013A0D2A38D8DFE812F0AD00E5
:106C60000C031A02F901DC0142031A032F03E802A4
:106C700023008F02850256024D02F7F7EFFE0790C0
:106C8000FEF707BEAB784FF0010B072B3FF646AA85
:106C9000DFE813F045034B04A2034004AE038C036A
:106CA00096034103424B1B78002B00F071861A209B
:106CB0000AF05EFF002840F06B8694F88C30002BC1
:106CC00040F0668609233B701BF03CFF1FF056FE28
:106CD000002800F083803B780C3B022B7FF626AA2D
:106CE00094F88C3001223A70002B3FF41FAA002345
:106CF00084F88C30FFF71ABA594604220CA824F005
:106D000011FF9DF83330AB2B04BF02236B76FFF7E6
:106D100037BA3068F2F7AEFE49463A2021F0FAF968
:106D20004946834604220CA824F0FCFEBBF1000F68
:106D300007D021F057FA21F01DFA95F82420FFF72B
:106D4000D9B821F04FFA0C9B1BBAC3F38073AB7612
:106D5000FFF73DBA9FED177AF4EEC76AF1EE10FA2D
:106D600044BF9FED0C7A77EE666A4CE7F470002022
:106D70008FC2753CD06D393A00000000DB0F4940EE
:106D800010A60020B024002058A70020DB0FC94027
:106D9000E4CB1641DB0F49C0E4CB16C1DB0FC93F82
:106DA00092E741B99730083C15A82ABE0088002018
:106DB000507E0020DB0FC9BFD84B1B78DB0700F1EA
:106DC000CD871F200AF0D4FE00283FF47FAF0C23AC
:106DD0003B701FF0D3FD00287FF4A8A9F378002BA7
:106DE0003FF4A4A9CE4B1B68D90440F1C585CD4B17
:106DF0009B8807EE903AF8EEE77ACB4A92ED012AAB
:106E0000D2ED022A92ED033AD2ED043A92ED054A10
:106E1000D2ED064A92ED075AD2ED085A92ED096A70
:106E2000D2ED0A6A92ED0B7AB4EE672AF1EE10FA0F
:106E3000F4EE672A14BF01230023F1EE10FAB4EE3A
:106E4000673A18BF43F00103F1EE10FAF4EE673A27
:106E500018BF43F00103F1EE10FAB4EE674A18BF11
:106E600043F00103F1EE10FAF4EE674A18BF43F065
:106E70000103F1EE10FAB4EE675A18BF43F00103B4
:106E8000F1EE10FAF4EE675A18BF43F00103F1EE89
:106E900010FAB4EE676A18BF43F00103F1EE10FA7E
:106EA000F4EE676A18BF43F00103F1EE10FAB4EE96
:106EB000677A18BF43F00103F1EE10FA18BF43F0F0
:106EC0000103002B40F0618492ED007AB4EE677A02
:106ED000F1EE10FA40F05984944DD4F890202B68CC
:106EE0009A4200F259843B78012B3FF41FA994F891
:106EF0008C20002A3FF41AA90B2B0ED801229A40AD
:106F000040F6030112EA01067FF4F1AE12F4C06FFD
:106F100003D0093B012B40F2EB87854B2A685A606E
:106F20000B233B70E3E69FED837AD5ED037A77EE92
:106F3000877AC5ED037AFEF780BDF7EE006AFEF7AB
:106F4000A0BFF7EE006AFEF723BF7B48D0F800A091
:106F5000BAF836B04FEA5B0B10E407EE903ADFED7B
:106F6000776AB8EEE77A66EEA65A9FED755A9FEDFE
:106F7000756ADFED757AA5EE856A26EEA55AE5EE0F
:106F8000867AE5EE276A26EE870A8EE56F4B9FED3F
:106F9000706AB3F90020B3F902306E4907EE902A07
:106FA00006EE903AF8EEE77AF8EEE66A27EEE87A2F
:106FB00060EE277AA0EE267AE8EEA67A27EE067A29
:106FC00067EE867ABDEEC77AFDEEE77A17EE102AF5
:106FD00017EE903A0A804B80FEF784BFB4F90C207C
:106FE0009AF80210A9EB020E8EEAEE70A0EBEE709A
:106FF000884240F313839145C8BF494207EE901A77
:10700000F8EEE77A012037EE888A2361207585ED56
:10701000038AFEF704BD1FF06DFC4F4B00210220D8
:107020008DE80300A3F10802029148201CF060FAE9
:1070300000287FF44BAE3E4B4FF0FF310622186024
:1070400059603A701FF09AFC00283FF4C7AE47E63B
:107050001FF050FC414A0292A2F10C032921019336
:107060000091A2F10A035021163A49201CF040FA7F
:1070700000287FF42BAE2A4B1B6813F0800300F02E
:107080007C862B4B4FF0FF310522186059603A7017
:10709000D8E7274D1FF02EFC244A6B681268643332
:1070A0009342BFF413AE40201FF0F6FB00287FF49C
:1070B0000DAE2B68DFF8A8A0DFF8A8904FF04008CD
:1070C0000DE01FF03BFDD9F800202B68013A013399
:1070D000B8F10108C9F800202B6000F0DD861AF82D
:1070E00003301846002BECD100234FF0FF322B6009
:1070F00004236A603B70A5E71F200AF039FD0028D1
:107100007FF467AE01233B709CE7012B00F01F86E4
:107110000E2313203B7017F0ABFAD7E571970020D0
:1071200018360020F4790020FC780020C4B8002034
:10713000B47D002000000000C06D002084F9223FD3
:1071400092E741B99730083C15A82ABEDC2E0020F2
:10715000CDCCCC3DC8240020940A0408B60804080D
:107160004008040880960020012B01D1F4F77EFA34
:107170000D2313203B7017F07BFAA7E5022B38D1C3
:10718000B84BDFF830831B78002B40F00986D8F825
:10719000005045B32B7833B395F82820002A7FF4AC
:1071A00051AF2B7EAA6385F83C20042285F8282065
:1071B00013F008036A6AEA622A6303D0AA4A41F21A
:1071C0009413D3586B634FF00009C5F82490C5F8A9
:1071D0000890C5F80C90284613F0E8F80523C5F888
:1071E000409085F8283000220423C8F8002088F851
:1071F00014309E4B9E4A5B681268C833934204D396
:107200001FF0DCFB00283FF461ADB378032B7FF463
:1072100079AF984D286814F0A9FD974B1B78002290
:10722000022B2A607FF46EAF14F028F86AE71A2068
:107230000AF09EFC00283FF447AD904B1B88002BC2
:107240007FF442AD8E4B45201D681FF077FC0E2069
:107250001FF074FC28461BF075F8089D28461BF0AB
:1072600071F8884A4FF480510A23284611803B70F8
:107270001BF018F928E5022B00F0E9837C4B7B4AD0
:107280001B68536080490023136003220B603A702F
:10729000D8E61FF02FFB7D4B002105208DE8030071
:1072A000A3F10802029153201CF022F900287FF478
:1072B0000DAD6E4A082310603B70C3E61FF01AFB49
:1072C0001BF060FC00283FF401AD1FF077FB0028A5
:1072D0003FF4FCAC6B4A4FF480510A2311803B70A1
:1072E000B0E61FF007FB6A4A0292A2F10C030725E1
:1072F00001930095A2F108030021143A47201CF0E5
:10730000F7F800287FF4E2AC584B3D704FF0FF32A5
:1073100083E8050096E603236B70FEF7FFBE0023AB
:107320000DF130094946184609220EF057FA012896
:107330007EF4F4AE0C9B93F8FE21552A00F0DA821D
:1073400041F2B41202210123A9546B70FEF7E6BE8C
:107350002B690622652BAA7032D92A78032A14BF1A
:107360006FF0FF026FF07F02A3F1650303EA0203EF
:1073700003F1010314BF4FF4807280229A422B6103
:107380001ED23268EE6802329F19974280F0F08474
:10739000404A6E60D16FAF60490203FB01F30521E3
:1073A000166042F81C3C42F8183CA970AA683A4999
:1073B00001200EF08DFC012840F0E8840623AB701C
:1073C000002136480EF0B6FB012840F0DF84AB7890
:1073D0000133DBB2AB7058E4314B00930320A8704B
:1073E000302305222F492D480FF03AFAFEF796BEBA
:1073F0002A782B7D2C4EDFF8A0A0032A14BF4FF46F
:1074000080778027002B70D0012BFBD1274B32686F
:1074100019686B684FEA412E4FF000094FF0FF31B9
:10742000B1FBFEFE1EEB030049F100014FF0000925
:10743000494502F1020208BF904238BF03EB0E0239
:107440001B4902200EF07CFD032800F2D98101A324
:1074500053F820F01D610108B97401081D6101088D
:10746000B97401089C7D0020903E0020B47D00206E
:10747000C4B8002084960020F47D0020187C0020F1
:107480001C7C0020047C002080960020F80A040860
:10749000B00A040824500020943E00200050002030
:1074A000A15402087836040898500020A05000200B
:1074B000983E0020E49500206968D5F808E02B6923
:1074C000AEEB01029A4284BFE9602A6103283FF4CF
:1074D0003FAF0EF10103B3FBF7F207FB12320AB123
:1074E0003B449B1A00226B602A7532685146023277
:1074F00000200EF025FD032800F2828101A353F83D
:1075000020F000BF1D610108677501081D610108B9
:107510005173010841F27013EB5C002B3EF4FEAD99
:10752000DB4824F077F9FEF7F9BD0DF1300941F29F
:10753000FC164946A859002309220EF04FF90128EC
:107540007EF4ECAD00230C9A2B70B2F80B30B3F53F
:10755000007F00F02F8441F2B41203210123A954CB
:107560006B70FEF7DBBD6B6885F814B00133AB6060
:107570004CE704212C2012F067FF032183464E20A4
:1075800012F062FF0C210490362012F05DFF049B84
:10759000421C02339A4009FA0BF9A2FB0901420A84
:1075A00042EAC152EA63FEF745BDBA4824F032F917
:1075B000FEF782BEB84824F02DF9FEF777BEB74833
:1075C00024F028F9FEF77EBEBAF838109FEDB47AA1
:1075D00007EE901AF8EEE77AB24967EE877AC1EDC6
:1075E000007AFEF730BAF0EE477AFEF79BBFB0EEB6
:1075F000677AFEF781BF2B46FEF7EBBEAA4DAB4282
:10760000BCBF03F50C43A033FEF7DCBEA6498A429B
:10761000BCBF02F50C42A032FEF7ECBE217D19B1D1
:10762000A24923750B68A361A3681344B3F5FA6FED
:10763000A8BF4FF4FA63B3F57A7FB8BF4FF47A73FB
:1076400007EE903AF8EEE77AC5ED037AFEF7E7B970
:10765000237D002B3FF464AA944B84F820201B6800
:107660002275A361FFF75CBA95ED000A04930592B9
:1076700026F020FD8E49DFF874E2D1F8EC10DFF837
:1076800070C2059AACF800008EFB013EC917C1EB31
:10769000AE1107EE901AF8EEE77A049BFDEEE77A5A
:1076A00017EE901AACF80210FEF72BBA07EE905ABC
:1076B000DFED806A9FED807A84F88050F8EEE77AFB
:1076C00067EEA67A77EE876ABDEEE66A16EE103AA6
:1076D0002033402B40F26481DFED786A784BBDEEB9
